:100000000C94250F0C94560F0C94560F0C94560F0D
:100010000C94560F0C94560F0C94560F0C94560FCC
:100020000C94560F0C94560F0C94560F0C94560FBC
:100030000C94560F0C9421AD0C94560F0C94560F43
:100040000C94560F0C94FA8B0C94560F0C94560F7C
:100050000C94560F0C94560F0C9439260C94E7A868
:100060000C94560F0C940D890C94560F0C94560F4B
:100070000C94560F0C94560F0C94560F0C94560F6C
:100080000C94560F0C94560F0C94560F0C94560F5C
:100090000C94560F0C94560F0C94560F0C9419A6F2
:1000A0000C94560F0C94560F0C94560F0C94560F3C
:1000B0000C94560F0C94560F0C94560F0C94560F2C
:1000C0000C94560F0C94560F0C94560F0C94560F1C
:1000D0000C94560F0C94560F0C94560F0C94560F0C
:1000E0000C94560F86269426B026BE26D826E626E1
:1000F0000027042706270A2712276BA770A775A7D2
:100100007FA7F8A789A791A799A7A3A7ADA7B7A786
:10011000C6A7D0A7F8A7DAA7E4A7EEA716A819A83C
:100120000CA810A850A81DA821A827A82BA82FA864
:1001300035A839A83DA850A843A847A84BA8084A05
:10014000D73B3BCE016E84BCBFFDC12F3D6C7431EB
:100150009ABD56833DDA3D00C77F11BED9E4BB4C42
:100160003E916BAAAABE000000803F05A84CCDB20C
:10017000D44EB93836A9020C50B9918688083CA6ED
:10018000AAAA2ABE000000803F007C3C3E5E2B3DB8
:100190003F2F5B5D3B2C2A225C004572723A204D5A
:1001A000415854454D50204245440054656D70659A
:1001B000726174757265206865617465642062653A
:1001C00064207377697463686564206F66662E20A7
:1001D0004D415854454D502074726967676572658A
:1001E00064202121004572723A204D494E54454DFC
:1001F00050003A204578747275646572207377698F
:100200007463686564206F66662E204D494E5445C0
:100210004D502074726967676572656420210045DE
:1002200072723A204D415854454D50003A2045785D
:10023000747275646572207377697463686564208D
:100240006F66662E204D415854454D50207472699A
:10025000676765726564202100202D20496E7661F4
:100260006C6964206578747275646572206E756D52
:10027000626572202100504944204175746F747585
:100280006E652066696E69736865642120507574B7
:1002900020746865206C617374204B702C204B694E
:1002A00020616E64204B6420636F6E7374616E74A2
:1002B000732066726F6D2061626F766520696E745F
:1002C0006F20436F6E66696775726174696F6E2E19
:1002D0006800504944204175746F74756E652066DE
:1002E00061696C6564212074696D656F75740020A7
:1002F000403A006F6B20543A006F6B20423A005036
:100300004944204175746F74756E65206661696C2F
:100310006564212054656D70657261747572652025
:10032000746F6F206869676800204B643A20002072
:100330004B693A2000204B703A200020436C6173D7
:100340007369632050494420002054753A200020EE
:100350004B753A2000206D61783A2000206D696E5F
:100360003A200020643A200020626961733A20003C
:1003700070012C0190012701B0012201C0011D0173
:10038000F00118011002130130020E016002090190
:1003900090020401C002FF000003FA004003F500D0
:1003A0008003F000D003EB002004E6007004E100BD
:1003B000E004DC004005D700C005D2004006CD00B7
:1003C000D006C8008007C3003008BE00F008B9009E
:1003D000C009B400B00AAF00B00BAA00D00CA50051
:1003E000000EA000500F9B00C0109600501291000C
:1003F00000148C00C0158700B0178200B0197D0072
:10040000D01B7800001E730040206E00902269000F
:10041000F024640040275F0090295A00E02B55002B
:10042000102E500020304B0010324600E0334100C7
:1004300090353C001037370070383200A0392D005D
:10044000B03A2800A03B2300603C1E00103D19007C
:10045000903D1400103E0F00703E0A00C03E0500A3
:10046000003F00004D383420582059205A204500C4
:1004700043616E6E6F7420656E7465722073756271
:100480006469723A20004D3234004D3233202573B6
:10049000006175746F25692E67006572726F722036
:1004A00077726974696E6720746F2066696C650085
:1004B0004E6F74205344207072696E74696E6700C9
:1004C0002F005344207072696E74696E67206279E0
:1004D000746520002E0044656C6574696F6E20663B
:1004E00061696C65642C2046696C653A2000466938
:1004F0006C652064656C657465643A002E006F70ED
:10050000656E206661696C65642C2046696C653A8D
:10051000200057726974696E6720746F2066696C79
:10052000653A20002E006F70656E206661696C650B
:10053000642C2046696C653A20002E006F70656E51
:10054000206661696C65642C2046696C653A200000
:1005500046696C652073656C65637465640020533F
:10056000697A653A200046696C65206F70656E6532
:10057000643A20002E006F70656E206661696C65BC
:10058000642C2046696C653A20004E6F77206672B5
:100590006573682066696C653A20004E6F77206449
:1005A0006F696E672066696C653A20002220706F63
:1005B00073002220706172656E743A2200535542B6
:1005C000524F5554494E452043414C4C2074617262
:1005D0006765743A2200747279696E6720746F20BF
:1005E00063616C6C207375622D67636F6465206650
:1005F000696C6573207769746820746F6F206D6112
:100600006E79206C6576656C732E204D4158206C98
:100610006576656C2069733A0053442063617264A7
:10062000206F6B006F70656E526F6F74206661692A
:100630006C656400766F6C756D652E696E697420EB
:100640006661696C656400534420696E6974206654
:1006500061696C0000002110422063308440A55085
:10066000C660E770088129914AA16BB18CC1ADD1F8
:10067000CEE1EFF13112100273325222B5529442A0
:10068000F772D662399318837BB35AA3BDD39CC348
:10069000FFF3DEE36224433420040114E664C774EC
:1006A000A44485546AA54BB528850995EEE5CFF598
:1006B000ACC58DD55336722611163006D776F66640
:1006C0009556B4465BB77AA719973887DFF7FEE7E8
:1006D0009DD7BCC7C448E5588668A778400861180C
:1006E00002282338CCC9EDD98EE9AFF94889699938
:1006F0000AA92BB9F55AD44AB77A966A711A500AE0
:10070000333A122AFDDBDCCBBFFB9EEB799B588B87
:100710003BBB1AABA66C877CE44CC55C222C033C2B
:10072000600C411CAEED8FFDECCDCDDD2AAD0BBDD7
:10073000688D499D977EB66ED55EF44E133E322E7F
:10074000511E700E9FFFBEEFDDDFFCCF1BBF3AAF27
:10075000599F788F8891A981CAB1EBA10CD12DC185
:100760004EF16FE18010A100C230E320045025401B
:1007700046706760B9839893FBA3DAB33DC31CD37B
:100780007FE35EF3B1029012F322D232354214526B
:1007900077625672EAB5CBA5A89589856EF54FE5C7
:1007A0002CD50DC5E234C324A014810466744764BB
:1007B00024540544DBA7FAB79987B8975FE77EF71B
:1007C0001DC73CD7D326F2369106B016576676760B
:1007D000154634564CD96DC90EF92FE9C899E989E7
:1007E0008AB9ABA94458654806782768C018E1085B
:1007F0008238A3287DCB5CDB3FEB1EFBF98BD89BBB
:10080000BBAB9ABB754A545A376A167AF10AD01AAA
:10081000B32A923A2EFD0FED6CDD4DCDAABD8BAD06
:10082000E89DC98D267C076C645C454CA23C832CFA
:10083000E01CC10C1FEF3EFF5DCF7CDF9BAFBABF5A
:10084000D98FF89F176E367E554E745E932EB23E4A
:10085000D10EF01E53544F505045442E200050727C
:10086000696E7465722073746F707065642064754E
:100870006520746F206572726F72732E20466978DE
:1008800020746865206572726F7220616E642075D5
:100890007365204D39393920746F20726573746126
:1008A00072742E202854656D70657261747572655E
:1008B0002069732072657365742E205365742069F6
:1008C00074206166746572207265737461727469F4
:1008D0006E6729004B494C4C45442E2000507269EC
:1008E0006E7465722068616C7465642E206B696C2F
:1008F0006C28292063616C6C656421006F6B005269
:100900006573656E643A20002200556E6B6E6F77DA
:100910006E20636F6D6D616E643A2022004D32323D
:100920003020532569005A204F6666736574203A5B
:1009300020007A5F6D61783A20007A5F6D696E3AC7
:1009400020005A204F6666736574005A204F666611
:10095000736574206F6B002200556E6B6E6F776E3F
:1009600020636F6D6D616E643A2022007A5F6D6165
:10097000783A20007A5F6D696E3A2000795F6D6188
:10098000783A2000795F6D696E3A2000785F6D617A
:10099000783A2000785F6D696E3A2000205A3A005C
:1009A00020593A0020436F756E7420583A20002079
:1009B000453A00205A3A0020593A00583A00464930
:1009C000524D574152455F4E414D453A4D61726C13
:1009D000696E2056312E302E323B20537072696E74
:1009E0007465722F6772626C206D61736875702018
:1009F000666F722067656E36204649524D574152E8
:100A0000455F55524C3A68747470733A2F2F67697A
:100A1000746875622E636F6D2F4D61726C696E46DE
:100A200069726D776172652F4D61726C696E2050CD
:100A3000524F544F434F4C5F56455253494F4E3AD5
:100A4000312E30204D414348494E455F5459504561
:100A50003A50727573612069332045585452554499
:100A600045525F434F554E543A3120555549443A0B
:100A700030303030303030302D303030302D30307C
:100A800030302D303030302D30303030303030306C
:100A9000303030300A005072757361206933204F56
:100AA00066662E005072757361206933207265612D
:100AB00064792E0042656420646F6E652E002042CA
:100AC0003A0020453A00543A004265642048656186
:100AD00074696E672E0048656174696E6720646F83
:100AE0006E652E0020573A0020453A00543A0048DF
:100AF000656174696E672E2E2E002042403A0020F8
:100B0000403A00202F003A00205400202F002042BD
:100B10003A00202F006F6B20543A002569206D6940
:100B20006E2C2025692073656300456E642066691C
:100B30006C65206C69737400426567696E20666934
:100B40006C65206C697374004E6F206D6F76652E36
:100B50000050727573612069332072656164792E6B
:100B600000526573756D696E67207072696E7400EE
:100B70005761697420666F7220757365722E2E2E10
:100B800000536C6565702E2E2E00256920686F75E8
:100B90007273202569206D696E7574657300446FEA
:100BA0006E65207072696E74696E672066696C6527
:100BB0000053544F505045442E20005072696E74BB
:100BC00065722073746F707065642064756520743D
:100BD0006F206572726F72732E2046697820746878
:100BE00065206572726F7220616E64207573652076
:100BF0004D39393920746F20726573746172742EA7
:100C0000202854656D706572617475726520697312
:100C10002072657365742E20536574206974206199
:100C2000667465722072657374617274696E672987
:100C3000004E6F204C696E65204E756D62657220A6
:100C40007769746820636865636B73756D2C204CDD
:100C5000617374204C696E653A20004E6F204368C2
:100C600065636B73756D2077697468206C696E6558
:100C7000206E756D6265722C204C617374204C6916
:100C80006E653A2000636865636B73756D206D69EE
:100C9000736D617463682C204C617374204C696EB1
:100CA000653A20004C696E65204E756D6265722054
:100CB0006973206E6F74204C617374204C696E658B
:100CC000204E756D6265722B312C204C617374203F
:100CD0004C696E653A20004D31313000446F6E65CD
:100CE00020736176696E672066696C652E006F6B94
:100CF000004D3239002020506C616E6E6572427575
:100D00006666657242797465733A200020467265A2
:100D100065204D656D6F72793A200044656320321D
:100D200033203230313500436F6D70696C65643A41
:100D30002000286E6F6E652C2064656661756C748A
:100D400020636F6E6669672900207C204175746896
:100D50006F723A20004465632032332032303135DF
:100D60002031353A34373A323200204C61737420E6
:100D7000557064617465643A2000312E302E320063
:100D80004D61726C696E0020536F66747761726595
:100D900020526573657400205761746368646F67DF
:100DA000205265736574002042726F776E206F75F4
:100DB00074205265736574002045787465726E61A5
:100DC0006C20526573657400506F776572557000C2
:100DD0007374617274002200656E717565696E6767
:100DE0002022002200656E717565696E6720220001
:100DF000FFFFFF0000A0400000A0400000004000F6
:100E0000005643000046431FC54843000000000051
:100E10000000001F856B3E00005643000046430063
:100E200000494300000000000000001F856B3E6584
:100E300063686F3A004572726F723A004361726480
:100E40002072656D6F766564004361726420696E1F
:100E50007365727465640047312045343020463133
:100E60003030004731204536352046343030004D93
:100E7000383300473120452D38302046343030009B
:100E80004D3833002D2D3A2D2D002D2D2D0053449E
:100E9000000120000120004D363030004368616EB3
:100EA00067652066696C616D656E7400466C6F776E
:100EB00000466C6F770046616E2073706565640054
:100EC00046616E207370656564004265640042652A
:100ED00064004E6F7A7A6C65004E6F7A7A6C6500AA
:100EE0005370656564005370656564004D61696E9B
:100EF00000436F6F6C646F776E00464C4558202D31
:100F000020203235302F35300050502020202D2029
:100F1000203235342F3130300048495053202D20B5
:100F2000203232302F3130300050455420202D20D7
:100F3000203234302F393000504C4120202D2020D9
:100F40003232302F35300041425320202D202032C4
:100F500038352F313030004D61696E004D38340026
:100F60004D383420582059205A2045004D32340045
:100F70004D323320257300052E2E004D61696E0021
:100F800046616E2073706565640046616E20737003
:100F90006565640042656400426564004E6F7A7A5C
:100FA0006C65004E6F7A7A6C650053657474696E77
:100FB000677300580059005A00457874727564656B
:100FC00072004578747275646572004D6F766520A5
:100FD0005A004D6F76652059004D6F766520580098
:100FE00053657474696E67730047323800417574D5
:100FF0006F20686F6D65004D38340044697361621D
:101000006C652073746570706572730047323820A8
:101010005A0043616C696272617465205A004D6FB9
:10102000766520617869730054656D7065726174CE
:10103000757265004D61696E005265763A203330F5
:10104000302D316100686F77746F2E707275736127
:1010500033642E636F6D00666F72756D2E707275DE
:10106000736133642E636F6D0070727573613364E6
:101070002E636F6D004669726D77617265202D2059
:10108000322E322E31004D61696E00537570706FD3
:1010900072740053657474696E677300556E6C6F7B
:1010A00061642066696C616D656E74004C6F61648B
:1010B0002066696C616D656E74004E6F205344202C
:1010C00063617264005072696E742066726F6D2085
:1010D00053440053746F70207072696E74005265CF
:1010E00073756D65207072696E74005061757365FB
:1010F000207072696E740050726568656174005486
:10110000756E6500496E666F2073637265656E006B
:1011100048617264636F6465642044656661756CE0
:10112000742053657474696E6773204C6F616465D5
:10113000640046696C616D656E74207365747469D2
:101140006E67733A2044697361626C6564002020A5
:10115000204D32303020440046696C616D656E74FC
:101160002073657474696E67733A002020204D32D5
:1011700030392053004175746F2D5265747261636C
:10118000743A20533D3020746F2064697361626C3F
:10119000652C203120746F20696E746572707265E1
:1011A0007420657874727564652D6F6E6C79206D2E
:1011B0006F766573206173207265747261637473F6
:1011C000206F72207265636F7665726965730020A7
:1011D00046002020204D3230382053005265636F86
:1011E0007665723A20533D4578747261206C656E65
:1011F00067746820286D6D2920463A5370656564D0
:1012000020286D6D2F6D2900205A002046002020D7
:10121000204D323037205300526574726163743A46
:1012200020533D4C656E67746820286D6D292046FB
:101230003A537065656420286D6D2F6D29205A3AE8
:10124000205A4C69667420286D6D290020440020C6
:1012500049002020204D3330312050005049442097
:1012600073657474696E67733A00205A00205900E0
:1012700020204D323036205800486F6D65206F6653
:101280006673657420286D6D293A00204500205A48
:101290000020580020420020540020204D323035DC
:1012A000205300416476616E6365642076617269E3
:1012B00061626C65733A20533D4D696E20666565C9
:1012C000647261746520286D6D2F73292C20543D44
:1012D0004D696E2074726176656C20666565647216
:1012E00061746520286D6D2F73292C20423D6D6936
:1012F0006E696D756D207365676D656E74207469B8
:101300006D6520286D73292C20583D6D6178696DBD
:10131000756D205859206A65726B20286D6D2F738A
:10132000292C20205A3D6D6178696D756D205A20F9
:101330006A65726B20286D6D2F73292C2020453D26
:101340006D6178696D756D2045206A65726B202826
:101350006D6D2F73290020540020204D3230342031
:101360005300416363656C65726174696F6E3A2006
:10137000533D616363656C65726174696F6E2C20A7
:10138000543D7265747261637420616363656C655A
:10139000726174696F6E00204500205A0020590068
:1013A00020204D3230312058004D6178696D756DC7
:1013B00020416363656C65726174696F6E20286D8E
:1013C0006D2F7332293A00204500205A0020590021
:1013D00020204D3230332058004D6178696D756D95
:1013E0002066656564726174657320286D6D2F7366
:1013F000293A00204500205A0020590020204D396C
:101400003220580053746570732070657220756EB9
:1014100069743A0045303A20005A3A2000593A207F
:1014200000583A20004D53312C4D53322050696EF4
:10143000730A00656E6473746F7073206869743A20
:10144000205A00205A3A00656E6473746F707320DE
:101450006869743A20590020593A00656E647374C3
:101460006F7073206869743A20580020583A0065FC
:101470006E6473746F7073206869743A200024F48A
:10148000D43050C38E20C2A24017828B7011127AC2
:10149000910D816CD90AA861E108C75866076151AE
:1014A00043061E4B5D05C145A7041A411104093DC1
:1014B0009803713931034036DB0265339102D43031
:1014C0005402802E1D02632CEE01752AC501B0283E
:1014D000A001102781018F2564012B244B01E022FC
:1014E0003401AC211F018D200D01801FFC00841EE2
:1014F000ED00971DDF00B81CD200E61BC600201BC4
:10150000BC00641AB200B219A8000A19A0006A1837
:101510009900D117910040178B00B5168400311641
:101520007E00B31579003A157300C7146F00581484
:101530006A00EE1366008813630025135E00C7126D
:101540005B006C12570015125400C111510070114C
:101550004F0021114B00D61049008D104700461056
:10156000440002104200C00F4000800F3E00420FB6
:101570003C00060F3B00CB0E3800930E37005C0E8C
:101580003500270E3400F30D3200C10D3100900DEF
:101590003000600D2E00320D2D00050D2C00D90CF1
:1015A0002B00AE0C2900850C29005C0C2700350CA3
:1015B00027000E0C2600E80B2400C40B2400A00B0F
:1015C00023007D0B23005A0B2100390B2100180B3F
:1015D0002000F80A1F00D90A1E00BB0A1E009D0A3F
:1015E0001D00800A1D00630A1C00470A1B002C0A0C
:1015F0001B00110A1A00F7091A00DD091900C409B5
:101600001900AB091900920917007B09180063093A
:1016100017004C09160036091600200916000A09A1
:101620001500F5081500E0081400CC081400B808EF
:101630001400A4081400900813007D0812006B0821
:10164000130058081200460812003408110023083D
:1016500011001208110001081100F0071000E00746
:101660001000D0071000C0071000B0070F00A1073E
:10167000100091070E0083070F0074070F00650725
:101680000E0057070E0049070E003B070D002E07FE
:101690000E0020070D0013070D0006070D00F906C8
:1016A0000C00ED060D00E0060C00D4060C00C80688
:1016B0000C00BC060C00B0060C00A4060B0099063A
:1016C0000C008D060B0082060B0077060B006C06E3
:1016D0000B0061060A0057060B004C060A00420682
:1016E0000A0038060A002E060A0024060A001A0616
:1016F0000A001006090007060A00FD050900F405A6
:101700000900EB050900E2050900D9050900D0052B
:101710000900C7050900BE050900B5050800AD05AB
:101720000800A50509009C050800940508008C0523
:101730000800840508007C050800740508006C0595
:101740000700650508005D050700560508004E0501
:101750000700470507004005080038050700310568
:1017600007002A050700230507001C0506001605CB
:1017700007000F0507000805060002050700FB0427
:101780000600F5040700EE040600E8040600E20483
:101790000700DB040600D5040600CF040600C904D8
:1017A0000600C3040600BD040600B7040600B10429
:1017B0000500AC040600A6040600A00405009B0476
:1017C000060095040500900406008A0405008504BF
:1017D0000500800406007A04050075040500700405
:1017E00005006B04050066040500610405005C0447
:1017F000050057040500520405004D040500480487
:101800000500430405003E0404003A0405003504C5
:101810000500300404002C04050027040400230400
:1018200005001E0404001A04040016040500110437
:1018300004000D040400090405000404040000046D
:101840000400FC030400F8030400F4030400F003A4
:101850000400EC030400E8030400E4030400E003D4
:101860000400DC030400D8030400D4030400D00304
:101870000400CC030400C8030300C503030024F4E0
:1018800004D9201BC40C5C0E9804C4095F026507D0
:101890007101F405F900FB04B30048048700C1039B
:1018A00069005803550003034500BE023A00840254
:1018B000310053022A002902250004022000E4011D
:1018C0001C00C8011900AF01170098011400840121
:1018D0001300710110006101100051010E0043015D
:1018E0000D0036010B002B010B0020010B00150130
:1018F00009000C01090003010800FB000800F300C7
:101900000800EB000700E4000600DE000600D80037
:101910000600D2000600CC000500C7000500C2008A
:101920000500BD000400B9000400B5000400B100CA
:101930000400AD000400A9000400A5000300A200FB
:1019400003009F0004009B00030098000300950023
:10195000020093000300900003008D0002008B0042
:10196000030088000200860002008400030081005A
:1019700002007F0002007D0002007B00020079006F
:10198000020077000100760002007400020072007D
:101990000100710002006F0002006D0001006C0088
:1019A00002006A0001006900020067000100660091
:1019B0000100650001006400020062000100610096
:1019C0000100600001005F0002005D0001005C009A
:1019D00001005B0001005A0001005900010058009D
:1019E000010057000100560001005500010054009D
:1019F000010053000000530001005200010051009B
:101A00000100500001004F0001004E0000004E0098
:101A100001004D0001004C0001004B0000004B0094
:101A200001004A0001004900010048000000480090
:101A3000010047000100460000004600010045008B
:101A40000000450001004400010043000000430085
:101A5000010042000000420001004100000041007E
:101A60000100400001003F0000003F0001003E0077
:101A700000003E0001003D0000003D0001003C0070
:101A800000003C0000003C0001003B0000003B0067
:101A900001003A0000003A0001003900000039005E
:101AA0000100380000003800000038000100370055
:101AB000000037000100360000003600000036004C
:101AC0000100350000003500000035000100340041
:101AD0000000340000003400010033000000330037
:101AE000000033000100320000003200000032002C
:101AF0000100310000003100000031000100300021
:101B0000000030000000300001002F0000002F0016
:101B100000002F0000002F0001002E0000002E000A
:101B200000002E0001002D0000002D0000002D00FF
:101B300000002D0001002C0000002C0000002C00F3
:101B400000002C0001002B0000002B0000002B00E7
:101B500000002B0001002A0000002A0000002A00DB
:101B600000002A00010029000000290000002900CF
:101B700000002900000029000100280000002800C2
:101B800000002800000028000000280001002700B5
:101B900000002700000027000000270000002700A9
:101BA000010026000000260000002600000026009C
:101BB000000026000100250000002500000025008F
:101BC0000000250000002500000025000100240081
:101BD0000000240000002400000024000000240075
:101BE0000100230000002300000023000000230068
:101BF0000000230000002300000023000100220059
:101C0000000022000000220000002200000022004C
:101C1000000022000100210000002100000021003E
:101C20000000210000002100000021000000210030
:101C30000100200000002000000020000000200023
:101C40000000200000002000000020000000200014
:101C500001001F0000001F0000001F0000001F0007
:101C600000001F0000001F0000001F0001001E00F8
:101C700000001E0000001E0000001E000000207476
:101C80006F6F206C6F6E6720657874727573696F03
:101C90006E2070726576656E7465640020636F6C8B
:101CA0006420657874727573696F6E2070726576E2
:101CB000656E746564000000090A02080B0C0D07CC
:101CC0000603040100000000000000000000000006
:101CD0000000000000000000000000000000000004
:101CE000000011100F0000000000000000000000C4
:101CF00000000000000000000000000000000000E4
:101D000000000000000000000000000001021020A0
:101D10002008081020401020408002010201080421
:101D200002010102040810204080804020100804B5
:101D3000020180040201804020100804020108040E
:101D40000201010204081020408001020408102052
:101D5000408010080408801020400440801020407B
:101D600004800505050507050808080802020202A7
:101D70000A0A080804040404010101010101010127
:101D80000303030303030303040707070C0C0C0CF2
:101D90000C0C0C0C020202020606060606060606DB
:101DA0000B0B0B0B0B0B0B0B07070A0A0A0A0A0A91
:101DB000050505040404080800002000230026008F
:101DC00029002C002F003200000100000301060151
:101DD000090100002200250028002B002E00310000
:101DE000340002010000050108010B010000210080
:101DF000240027002A002D003000330001010000DC
:101E0000040107010A01024E414E494E4954594905
:101E10004E46CDCCCC3D0AD7233C17B7D13877CC32
:101E20002B329595E6241FB14F0A00002041000097
:101E3000C84200401C4620BCBE4CCA1B0E5AAEC550
:101E40009D749D63FF7DEDA5A16311241FBECFEF9F
:101E5000D1E2DEBFCDBF00E00CBF15E0A0E0B2E0F4
:101E6000E2E6F2E701E00BBF02C007900D92A23E4E
:101E7000B107D9F724E1A2EEB5E001C01D92AD3B58
:101E8000B207E1F71EE1C8E4DEE100E006C02297F8
:101E90000109FE010BBF0E94D8B2C234D10780E015
:101EA0000807A9F70E94F1A90C9420B90C9400002E
:101EB000CF93DF93EC019C012C5F3F4F41E050E05A
:101EC00060E070E0898D9A8D0E94FA19882399F05C
:101ED0004D895E896F89788D452B462B472B59F4A8
:101EE0004C815D816E817F814D8B5E8B6F8B788F96
:101EF000998190689983DF91CF910895CF92DF9275
:101F0000EF92FF920F931F93CF93DF93EC01898998
:101F10009A89AB89BC89803E9F4FAF41B10510F0D3
:101F200080E06BC0CE01C4DF8823D1F30E940E187D
:101F3000182F8823A9F3E98DFA8DCC80DD80EE80FF
:101F4000FF8032E0C31AD108E108F108058404C01B
:101F5000CC0CDD1CEE1CFF1C0A94D2F786859785FD
:101F6000A089B189C80ED91EEA1EFB1E81E08093AC
:101F7000E805C092EB07D092EC07E092ED07F092F3
:101F8000EE0780E092E0EBEEF5E0DF019C011D92B0
:101F900021503040E1F701E0E98DFA8D8481081786
:101FA00090F42BEE35E0B701A601400F511D611DE5
:101FB000711D8091E9059091EA050E94E73B882315
:101FC000E1F00F5FE9CFC12C82E0D82EE12CF12C9B
:101FD000058404C0CC0CDD1CEE1CFF1C0A94D2F757
:101FE00049895A896B897C894C0D5D1D6E1D7F1D49
:101FF000498B5A8B6B8B7C8B812FDF91CF911F91FB
:102000000F91FF90EF90DF90CF900895CF93DF93E3
:10201000EC0141E0611101C040E06C857D858E8559
:102020009F850E944E18882341F0888920E2829F74
:10203000C001112485519A4F02C080E090E0DF91E9
:10204000CF91089530E020E04EE2DC015C91503207
:1020500071F0383029F4FB01E20FF11D40832F5F4E
:10206000FB01E20FF11DDC015C9150832F5F3F5FAC
:1020700001963B3051F7FB01E20FF11D10820895EC
:10208000CF93DF93EB01FC012381211102C080E09B
:102090000EC02250223020F48FE28883198206C0BD
:1020A00060E0B4DF009799F3BE01CCDF81E0DF91FF
:1020B000CF910895FB012BE030E231932150E9F7F5
:1020C000DC0190E027E03A2FEB2F8D9181110AC0BF
:1020D000DA013C931196EC9381E0FB019081903200
:1020E00039F525C08F32A1F38E3219F0EAE8F1E01C
:1020F00008C02A30E1F098E02AE0E5CF31963817A1
:10210000B1F034913111FACF291788F03FED380F33
:102110003E3568F431E0390FFB01E90FF11D9FE90D
:10212000980F9A3108F480528083932FCCCF80E0AF
:1021300008950F931F93CF93DF93EC018B018B8155
:10214000882311F080E042C0FB018789803139F19A
:102150008032C1F783E08B83F801428D538D648D0B
:10216000758D4D8B5E8B6F8B788F9E012F5E3F4FF1
:10217000C8010E940519882329F31A8F098F81E06D
:1021800089831C821D821E821F82188619861A86E8
:102190001B861C861D861E861F86188A17C082E035
:1021A0008B831D8A1E8A1F8A188EFB01408D518DDC
:1021B00060E070E095E0440F551F661F771F9A9509
:1021C000D1F7498B5A8B6B8B7C8BD7CFDF91CF911B
:1021D0001F910F9108952F923F924F925F926F92AD
:1021E0007F928F929F92AF92BF92CF92DF92EF92A7
:1021F000FF920F931F93CF93DF93EC015B016A0172
:102200008B81811103C08FEF9FEFC7C0898180FF51
:10221000FACF49895A896B897C8988859985AA85ED
:10222000BB852601612C712C8A019B01081B190BAF
:102230002A0B3B0B401651066206730618F06A0122
:10224000C81AD90A76013E0124E0620E711CE1141D
:10225000F10409F476C0488559856A857B854A0171
:1022600081E098222B811A012B01E9E056944794D2
:1022700037942794EA95D1F7898D9A8DFC01223005
:1022800049F4628D738D848D958D620D731D841D4F
:10229000951D3CC014811150122181149104C1F488
:1022A000111116C0452B462B472B49F48D899E8969
:1022B000AF89B88D8C839D83AE83BF8309C04C8169
:1022C0005D816E817F81930121D7882309F49BCFA3
:1022D000E98DFA8D6C817D818E819F8162507109BB
:1022E00081099109058404C0660F771F881F991F13
:1022F0000A94D2F72685378540895189620F731F6A
:10230000841F951F610F711D811D911D20E032E01A
:102310002819390987012E153F0508F4890101158F
:10232000F2E01F0769F52091EB073091EC0740912F
:10233000ED075091EE07621773078407950719F4AC
:102340001FC0C6012AC09501AB01BC018091E905FF
:102350009091EA050E94723B882309F454CFA00EA5
:10236000B11E88859985AA85BB85800F911FA11D07
:10237000B11D88879987AA87BB87E01AF10A67CFC2
:1023800040E08CD6882309F43ECFB40165517A4FE2
:10239000A801C5010E94F5B5E2CFDF91CF911F9151
:1023A0000F91FF90EF90DF90CF90BF90AF909F90F4
:1023B0008F907F906F905F904F903F902F900895F7
:1023C000CF93DF931F92CDB7DEB741E050E0BE015F
:1023D0006F5F7F4F00DF019719F4898190E002C0A1
:1023E0008FEF9FEF0F90DF91CF910895CF92DF9203
:1023F000EF92FF920F931F93CF93DF936C01EB014A
:102400007A01FC018381823060F00085118522858C
:1024100033850F71112722273327012B022B032B22
:1024200011F08FEF5CC04115510511F0F7011082DA
:102430001DE040E250E0BE01C601CDDE80329105D4
:1024400039F021E0892B09F420E0822F819547C0E3
:1024500028812223C1F0253E61F32E3251F33B85C2
:102460003F733F3061F4E114F10449F04A8D5B8D14
:10247000452B29F42F713FEF320F343030F02B858C
:1024800023FDD7CF2CC080E02AC030E02150310995
:10249000129FC001139F900D1124F701E80FF91F3F
:1024A000298120832B8121832D8122832F812383E6
:1024B000298524832E852583288926832A892783B5
:1024C0002C8920872E892187288D22872C8D238790
:1024D0002E8D2487288126FFD2CF1586D0CFDF917D
:1024E000CF911F910F91FF90EF90DF90CF900895C3
:1024F0001F93CF93DF93EC018B81823018F480E03F
:1025000090E023C0488559856A857B85A5E076954E
:10251000679557954795AA95D1F7142F1F70CE014F
:102520004FDF97FDECCF488559856A857B85415EF5
:102530005F4F6F4F7F4F488759876A877B8720E2BD
:10254000129FC001112485519A4FDF91CF911F91A5
:1025500008954F925F926F927F92AF92BF92CF9207
:10256000DF92EF92FF920F931F93CF93DF93EC01D3
:102570006A017B012B81222349F089899A89AB89E1
:10258000BC8984179507A607B70710F480E06BC0D5
:10259000223009F463C0C114D104E104F10449F408
:1025A0001C821D821E821F82188619861A861B862F
:1025B00059C088859985AA85BB85E98DFA8DE58501
:1025C000F0E03996AC01BD01415051096109710932
:1025D0000E2E04C076956795579547950A94D2F7C5
:1025E00097018601015011092109310904C036956E
:1025F000279517950795EA95D2F70417150726072B
:10260000370720F0892B8A2B8B2B49F48D899E89E3
:10261000AF89B88D8C839D83AE83BF8304C0041BB8
:10262000150B260B370B280139015E0184E0A80E3B
:10263000B11C411451046104710481F04C815D812D
:102640006E817F819501898D9A8D60D591E0491ABF
:102650005108610871088111ECCF05C0C886D98680
:10266000EA86FB8681E0DF91CF911F910F91FF9069
:10267000EF90DF90CF90BF90AF907F906F905F9082
:102680004F9008950F931F93CF93DF93EC018B81AD
:102690008823D1F1898187FF32C061E0CE01B6DCA9
:1026A0008C01009789F1FC018081853E69F18B8165
:1026B000823040F449895A896B897C89448F558FCF
:1026C000668F778F4D895E896F89788DF801538F7A
:1026D000428F758B648BE091E205F091E3053097B2
:1026E00059F0B8016A5E7F4FC80148961995F80104
:1026F000808D918D938B828B89818F778983DF91F8
:10270000CF911F910F918AC481E0888380E0DF918F
:10271000CF911F910F910895CF93DF93EC01B2DF1A
:102720001B82DF91CF910895FC0123812111F4CF09
:1027300008954F925F926F927F92AF92BF92CF9225
:10274000DF92EF92FF920F931F93CF93DF9300D00E
:102750001F92CDB7DEB75C016A017B01FC0183816A
:102760008130E9F4818181FF1AC0F5018189928964
:10277000A389B48984179507A607B70780F0892B2A
:102780008A2B8B2B09F472C0F5014084518462843A
:102790007384B701A601C501DCDE811102C080E0AF
:1027A00066C0F501818D928DC114D104E104F1045C
:1027B00069F4458956896789708D25D7882379F30F
:1027C000F501158A168A178A108E37C0F5014481E3
:1027D0005581668177819E012F5F3F4F97D4882373
:1027E000F1F249815A816B817C81F501818D928D55
:1027F000FC012789203139F4483FFFEF5F0761056D
:102800007105D8F407C0483F2FEF520762072FE049
:10281000720798F4F8D6882309F4C1CFF5014481F2
:102820005581668177810FEF1FEF2FEF3FE0818D9C
:10283000928D51D5882309F4B2CFF501C18AD28A8D
:10284000E38AF48A818180688183C5011BDF882344
:1028500009F4A5CFB701A6014C145D046E047F04F2
:1028600010F4B301A201C50174DE01C081E00F9034
:102870000F900F900F90DF91CF911F910F91FF90CC
:10288000EF90DF90CF90BF90AF907F906F905F9070
:102890004F900895FF920F931F93CF93DF93EC0116
:1028A000F42E80E2689FF0011124E551FA4F8385F0
:1028B000817121F0842F827109F04EC08091EB0765
:1028C0009091EC07A091ED07B091EE078C879D8762
:1028D000AE87BF87688B4489558960E070E0BA0194
:1028E00055274427028D138D20E030E0402B512BDB
:1028F000622B732B4D8B5E8B6F8B788F83858871EA
:1029000051F4048D158D268D378D098B1A8B2B8BE9
:102910003C8B81E00BC08031F9F49E012F5E3F4F6C
:10292000898D9A8D72D48823B9F084E08B838F2DA2
:102930008F7089831C821D821E821F8218861986D1
:102940001A861B86F4FE0BC040E050E0BA01CE01AF
:10295000F0DE811104C011C01B8280E00EC0F5FEC4
:102960000BC049895A896B897C89CE01DF91CF914F
:102970001F910F91FF90EDCD81E0DF91CF911F91DD
:102980000F91FF900895AF92BF92CF92DF92EF9296
:10299000FF920F931F93CF93DF937C01EB016A01AA
:1029A000B22E898D9A8DF701928F818F40E050E091
:1029B000BA01CE01CEDDA12C088519852A853B857B
:1029C00089899A89AB89BC89081719072A073B07A7
:1029D000A0F585E036952795179507958A95D1F747
:1029E0000F70CE0185DD009709F481C0FC012081C4
:1029F000222311F0253EB9F4A1100EC04091EB073F
:102A00005091EC076091ED077091EE07F701448754
:102A1000558766877787008BFC018081AA24A39461
:102A20008111CACF0AC04BE050E0BC01C6010E9430
:102A3000E8B5892B09F0C0CF58C08B2D8274823441
:102A400009F055C0AA2049F0F701008961E0C701EB
:102A5000DDDAEC01009769F44AC08B81823009F419
:102A600046C0CE014BDA882309F441C0CBEED5E055
:102A700000E080E2FE0111928A95E9F78BE0F60111
:102A8000DE0101900D928A95E1F7E091E205F09167
:102A9000E305309739F0BE01625F7F4FCE0140966B
:102AA000199508C081E298E2998B888B80E098E0C4
:102AB0009F878E87888999899B8B8A8B998F888F2E
:102AC0008E859F859F8B8E8BA9D2882381F04B2D7D
:102AD000602FC701DF91CF911F910F91FF90EF9071
:102AE000DF90CF90BF90AF90D5CEB7FEF0CF80E013
:102AF000DF91CF911F910F91FF90EF90DF90CF90DA
:102B0000BF90AF9008953F924F925F926F927F92E5
:102B10008F929F92AF92BF92CF92DF92EF92FF92ED
:102B20000F931F93CF93DF93CDB7DEB7C354D10973
:102B30000FB6F894DEBF0FBECDBF5C016B012496CB
:102B40005FAF4EAF2497522E1C8E1F8E19821C82AF
:102B50006115710511F410E073C0FC0183818111CE
:102B6000FACF2496EEADFFAD249780818F3211F01D
:102B700076011DC02496EEADFFAD249780818F3283
:102B800031F431962496FFAFEEAF2497F3CFF601E0
:102B900083818250823060F3F601618D728DCE01A7
:102BA0000196C7DA8823B9F2CE0101967C018E0125
:102BB000045E1F4F3801FE0131964F01402E312E29
:102BC00019C08823A9F121E0AE01495C5F4FB7012C
:102BD000C801D9DE882309F4BECFEC14FD0411F03E
:102BE000C7019ADD0615170501F1942D832D780193
:102BF000092F182FAE014E5B5F4FBE01695C7F4FFE
:102C000024968EAD9FAD249755DA882309F4A3CF7F
:102C10002496EEADFFAD249780818F3291F63196E8
:102C20002496FFAFEEAF2497F3CF982D892DDFCFF9
:102C3000252DAE01495C5F4FB701C501A4DE182FF9
:102C4000CE01019671DDCE014C966EDD812FCD5BFC
:102C5000DF4F0FB6F894DEBF0FBECDBFDF91CF912F
:102C60001F910F91FF90EF90DF90CF90BF90AF90AA
:102C70009F908F907F906F905F904F903F900895BE
:102C8000CF93DF93EC0140E050E0BA0152DD88239E
:102C900061F061E0CE01BAD9009739F025EEFC0170
:102CA00020831B82DF91CF91B9C180E0DF91CF916A
:102CB00008951F93CF93DF93CDB7DEB76B970FB611
:102CC000F894DEBF0FBECDBFAB0119821C8222E09B
:102CD000BC01CE01019617DF182F882321F0CE0109
:102CE0000196CEDF182FCE0101961EDD812F6B9647
:102CF0000FB6F894DEBF0FBECDBFDF91CF911F910D
:102D000008952F923F924F925F926F927F928F928F
:102D10009F92AF92BF92CF92DF92EF92FF920F936A
:102D20001F93CF93DF9300D01F921F92CDB7DEB7D2
:102D30008C015B013A01DC0113968C911397813071
:102D4000C1F411968C9181FF14C082FF18C0F80164
:102D5000418952896389748980859185A285B3856B
:102D600084179507A607B70751F0C801F2DB811158
:102D700006C081E0F80180838FEF9FEF37C16301C8
:102D800083C0D80159968D919C915A97FC01F4818A
:102D9000F1501A012B0169E0569447943794279417
:102DA0006A95D1F7F221FD834A0121E09222FF23A7
:102DB00009F476C080E092E08819990976018C15B3
:102DC0009D0508F47C01D8015996ED91FC915A9724
:102DD00014962D903D904D905C901797B2E02B1A71
:102DE000310841085108058404C0220C331C441CDE
:102DF000551C0A94D2F786859785A089B189280E3B
:102E0000391E4A1E5B1EED812E0E311C411C511CC9
:102E1000E114F2E0FF0609F089C08091EB07909180
:102E2000EC07A091ED07B091EE0782159305A4057C
:102E3000B50569F41092E8058FEF9FEFDC018093F0
:102E4000EB079093EC07A093ED07B093EE07950185
:102E5000B201A1018091E9059091EA050E94E73B4A
:102E6000882309F486CFF80180859185A285B385F2
:102E70008E0D9F1DA11DB11D80879187A287B387ED
:102E8000AE0CBF1CCE18DF08D80118964D915D918D
:102E90006D917C911B97C114D10409F072CF7AC057
:102EA0008114910409F086CF14964D915D916D9136
:102EB0007C911797411551056105710559F4559697
:102EC0008D919D910D90BC91A02D0097A105B1050C
:102ED00039F520C09E012F5F3F4F18D1882309F498
:102EE00048CF89819A81AB81BC81F801218D328DD7
:102EF000F9012789203139F4883FFFEF9F07A105A9
:102F0000B10540F40DC0883F2FEF9207A2072FE0D4
:102F1000B20730F0C8010E94580F81114BCF29CF62
:102F2000F80184839583A683B78344CF81149104E9
:102F300011F5D80118964D915D916D917C911B977B
:102F400051968D919D910D90BC91A02D48175907D8
:102F50006A077B0780F062D0882309F40ACF81E0FA
:102F60008093E8052092EB073092EC074092ED0742
:102F70005092EE0707C041E0C201B1018FD0882313
:102F800009F4F7CEA701B501C40185519A4F0E94FB
:102F9000F5B569CF51968D919D910D90BC91A02D65
:102FA000F801218184179507A607B70738F4418BEC
:102FB000528B638B748B206821830CC08091E20557
:102FC0009091E305892B31F06114710419F02068A8
:102FD000F8012183D80111968C9183FD02C0C301B1
:102FE00005C0C8014FDB8111FACFC3CE0F900F90FF
:102FF0000F900F900F90DF91CF911F910F91FF9045
:10300000EF90DF90CF90BF90AF909F908F907F9088
:103010006F905F904F903F902F900895CF93809145
:10302000E8058823B9F14091EB075091EC076091D6
:10303000ED077091EE072BEE35E08091E905909158
:10304000EA050E94E73BC82F811102C0C0E023C0FF
:103050004091E4055091E5056091E6057091E70522
:10306000411551056105710591F02BEE35E0809118
:10307000E9059091EA050E94E73B882339F3109215
:10308000E4051092E5051092E6051092E70510920E
:10309000E80501C0C1E08C2FCF910895CF92DF9257
:1030A000EF92FF92CF936B017C01C42F8091EB07CD
:1030B0009091EC07A091ED07B091EE078C159D055E
:1030C000AE05BF05C9F0AADF811102C080E018C0BB
:1030D0002BEE35E0B701A6018091E9059091EA0554
:1030E0000E94723B882391F3C092EB07D092EC07C9
:1030F000E092ED07F092EE0781E0C1118093E805C0
:10310000CF91FF90EF90DF90CF9008958F929F9294
:10311000AF92BF92CF92DF92EF92FF920F931F93E5
:10312000CF93DF93EC016A017B01890189859A8540
:10313000AB85BC850196A11DB11D84179507A60717
:10314000B70710F480E054C08F89803129F49927A3
:10315000872F762F652F0BC08032A1F7CB01BA01E4
:1031600027E096958795779567952A95D1F78B886F
:103170009C88AD88BE88680D791D8A1D9B1D809036
:10318000EB079090EC07A090ED07B090EE07681564
:1031900079058A059B0581F48F89803191F4DD24BE
:1031A000EE24FF24F601EE0FFF1FE551FA4F808158
:1031B0009181A0E0B0E016C040E070DF8111ECCF5B
:1031C000C1CFE894C7F8DD24EE24FF24F601EE0F0A
:1031D000FF1FEE0FFF1FE551FA4F80819181A28101
:1031E000B381BF70F80180839183A283B38381E0B0
:1031F000DF91CF911F910F91FF90EF90DF90CF90D3
:10320000BF90AF909F908F9008954F925F926F9272
:103210007F92AF92BF92CF92DF92EF92FF920F9385
:103220001F93CF93DF9300D01F92CDB7DEB78C01F1
:1032300049835A836B837C835901C12CD12C76013D
:10324000412C42E0542E612C712C49815A816B81B2
:103250007C819E012F5F3F4FC80158DF882341F1D9
:10326000D301C201F801058404C0880F991FAA1F69
:10327000BB1F0A94D2F7C80ED91EEA1EFB1E498155
:103280005A816B817C818789803139F481E0483FA4
:103290005F4F6105710538F4D8CF81E0483F5F4F3B
:1032A0006F4F7F4090F2F501C082D182E282F382BB
:1032B0000F900F900F900F90DF91CF911F910F9172
:1032C000FF90EF90DF90CF90BF90AF907F906F9086
:1032D0005F904F9008954F925F926F927F928F927E
:1032E0009F92AF92BF92CF92DF92EF92FF920F9395
:1032F0001F93CF93DF93EC014A015B012801390151
:10330000423051056105710508F462C049855A854E
:103310006B857C854F5F5F4F6F4F7F4F4815590519
:103320006A057B0508F454C08F89803129F4FF2495
:10333000EB2CDA2CC92C0CC0803209F049C0750185
:10334000640177E0F694E794D794C7947A95D1F71F
:103350004B895C896D897E89C40ED51EE61EF71ED9
:1033600041E0C701B6019ADE882391F19F8990312F
:1033700059F49924AA24BB24F401EE0FFF1FE55150
:10338000FA4F5182408210C0E89487F89924AA2409
:10339000BB24F401EE0FFF1FEE0FFF1FE551FA4FA4
:1033A00040825182628273829A89923090F04D817C
:1033B0005E816F8178854C0D5D1D6E1D7F1D409374
:1033C000E4055093E5056093E6057093E70501C0B9
:1033D00080E0DF91CF911F910F91FF90EF90DF90F0
:1033E000CF90BF90AF909F908F907F906F905F90A5
:1033F0004F9008952F923F924F925F926F927F92DB
:103400008F929F92AF92BF92CF92DF92EF92FF92F4
:103410000F931F93CF93DF93CDB7DEB72F970FB6E0
:10342000F894DEBF0FBECDBF1C014C875D876E8751
:103430007F873B872A87DC0119960D911D912D917D
:103440003C911C970F5F1F4F2F4F3F4F0D831E83E3
:103450002F833887EA85FB8580809180A280B380A6
:1034600081149104A104B10431F0FFEF8F1A9F0A77
:10347000AF0ABF0A10C0DC018D909D90AD90BC904A
:10348000B1E0B9870C851D852E853F85013011057A
:103490002105310509F0198675016401412C512C73
:1034A0003201F10181859285A385B48548165906BC
:1034B0006A067B0608F04EC00D811E812F8138857B
:1034C0000C151D052E053F0550F4F2E0CF2ED12C32
:1034D000E12CF12CA2E08A2E912CA12CB12C9E0182
:1034E0002F5F3F4FB701A601C10110DE882391F184
:1034F00049815A816B817C81D701C6010196A11D4A
:10350000B11D452B462B472B19F04C015D010FC017
:10351000AC01BD01481959096A097B090C851D8553
:103520002E853F85401751076207730741F01FEF53
:10353000411A510A610A710A6C017D01B2CF0FEF85
:103540001FEF2FEF3FE0B701A601C101C4DE8D835D
:10355000811113C01D823DC02601370121E0421AAE
:1035600051086108710897018601B301A201C101E8
:10357000B2DE882379F3730162018C149D04AE04DA
:10358000BF0450F3AA85BB854D915D916D917C91EF
:103590004115510561057105A9F4EA85FB85808215
:1035A0009182A282B382F985FF2399F00FEF801AEE
:1035B000900AA00AB00AD1018D929D92AD92BC9260
:1035C000139707C095018401C10185DE8111E5CF04
:1035D000C1CF8D812F960FB6F894DEBF0FBECDBF41
:1035E000DF91CF911F910F91FF90EF90DF90CF90DF
:1035F000BF90AF909F908F907F906F905F904F9013
:103600003F902F900895AF92BF92CF92DF92EF92AA
:10361000FF920F931F93CF93DF9300D01F92CDB7EC
:10362000DEB75C016A017B0182E090E0A0E0B0E0DF
:10363000F50180839183A283B3839E012F5F3F4F67
:10364000B701A601C50162DD811102C080E023C07F
:1036500000E010E09801B701A601C5013CDE882317
:10366000A9F3C980DA80EB80FC80F501878980317D
:1036700049F481E0F8EFCF16FFEFDF06E104F10433
:1036800050F4DBCF81E098EFC9169FEFD906E90629
:103690009FE0F90690F20F900F900F900F90DF913E
:1036A000CF911F910F91FF90EF90DF90CF90BF903F
:1036B000AF9008957F928F929F92AF92BF92CF92D8
:1036C000DF92EF92FF920F931F93CF93DF93EC0162
:1036D000142F7093EA056093E9051F8A82E090E059
:1036E000A0E0B0E088839983AA83BB831092E805A9
:1036F0001092E4051092E5051092E6051092E70598
:103700008FEF9FEFDC018093EB079093EC07A09382
:10371000ED07B093EE07442349F1453008F0DEC0D1
:1037200040E060E070E0CB01B9DC882309F4D6C04A
:1037300020E1129FF0011124E756F84F80818F7726
:1037400009F0CCC084859585A685B785843691051A
:10375000A105B10508F4C2C0C084D184E284F38419
:10376000C114D104E104F10421F4B8C0C12CD12C5E
:10377000760140E0C701B60191DC782E882309F478
:10378000ADC08091F6059091F7058115924009F042
:10379000A5C03091FB05332309F4A0C08091F90541
:1037A0009091FA05892B09F499C02091F8052223FC
:1037B00009F494C03A8B2C831D8630E041E050E040
:1037C0006D85062FCA01062E02C0880F991F0A9424
:1037D000E2F72817390731F081E0860F8D876830CE
:1037E00078F37CC020910106309102062115310545
:1037F00019F040E050E008C020910F06309110060B
:1038000040911106509112062D833E834F835887B5
:103810008091F9059091FA0546015701880E991E8D
:10382000A11CB11C8B8A9C8AAD8ABE8AE091FC05E2
:10383000F091FD05F98FE88FA091FB05B0E00E94A3
:10384000C8B2680D791D8A1D9B1D6A8F7B8F8C8F76
:103850009D8FB5E0EE0FFF1FBA95E1F7E150FE4FE7
:10386000EF2FFF27E695DC01CB018E0F9F1FA11DD7
:10387000B11D8E879F87A88BB98B8090FE05909095
:10388000FF058114910419F0A12CB12C08C080907F
:103890000B0690900C06A0900D06B0900E06A701A6
:1038A0009601281B390B4A0B5B0BDA01C901880D05
:1038B000991DAA1DBB1D04C0B695A7959795879520
:1038C0000A95D2F789879A87AB87BC87853F3FE007
:1038D0009307A105B10520F48CE08F8B712C15C0E6
:1038E000853F9F4FA105B10510F480E10DC0809187
:1038F000170690911806A0911906B0911A068A8FA2
:103900009B8FAC8FBD8F80E28F8B872DDF91CF9106
:103910001F910F91FF90EF90DF90CF90BF90AF90ED
:103920009F908F907F9008954F925F926F927F92B9
:103930008F929F92AF92BF92CF92DF92EF92FF92BF
:103940000F931F93CF93DF932C0124E733E081E0A3
:1039500090E0F90145915491441655060CF062C06F
:10396000AC0141505109DA01AA0FBB1FAA0FBB1FBE
:10397000AE58BC4FFD0165917491440F551F440F23
:10398000551F40595C4FFA0165907490FC01EE0F91
:10399000FF1FEE0FFF1FEE58FC4FA590B490FD01E6
:1039A00005911491F901C591D491FA0185909490F3
:1039B000882777FD8095982F0E9442AF6B017C018C
:1039C000B20166197709882777FD8095982F0E94A4
:1039D00042AF2B013C01B501601B710B882777FDBD
:1039E0008095982F0E9442AF9B01AC01C301B201A8
:1039F0000E9475B12B013C01BE0168197909882725
:103A000077FD8095982F0E9442AF9B01AC01C301C6
:103A1000B2010E94A7AE9B01AC01C701B6010E9492
:103A2000C7AD11C001962C5F3F4F8D33910509F052
:103A300090CFE2E6F4E065917491882777FD809558
:103A4000982F0E9442AFDF91CF911F910F91FF906D
:103A5000EF90DF90CF90BF90AF909F908F907F902E
:103A60006F905F904F9008954F925F926F927F9208
:103A70008F929F92AF92BF92CF92DF92EF92FF927E
:103A80000F931F93CF93DF932C01662371F1E5E32E
:103A9000FEE08491882341F09091C00095FFFCCF17
:103AA0008093C6003196F5CF70E04AE050E08CE993
:103AB0009DE00E945A8AE9E5F2E08491882341F072
:103AC0009091C00095FFFCCF8093C6003196F5CF52
:103AD0008091C00085FFFCCF8AE08093C6000E94E1
:103AE000224560E070E0CB017EC024E733E081E056
:103AF00090E0F90145915491441655060CF062C0CE
:103B0000AC0141505109DA01AA0FBB1FAA0FBB1F1C
:103B1000AE58BC4FFD0165917491440F551F440F81
:103B2000551F40595C4FFA0165907490FC01EE0FEF
:103B3000FF1FEE0FFF1FEE58FC4FA590B490FD0144
:103B400005911491F901C591D491FA018590949051
:103B5000882777FD8095982F0E9442AF6B017C01EA
:103B6000B20166197709882777FD8095982F0E9402
:103B700042AF2B013C01B501601B710B882777FD1B
:103B80008095982F0E9442AF9B01AC01C301B20106
:103B90000E9475B12B013C01BE0168197909882783
:103BA00077FD8095982F0E9442AF9B01AC01C30125
:103BB000B2010E94A7AE9B01AC01C701B6010E94F1
:103BC000C7AD11C001962C5F3F4F8D33910509F0B1
:103BD00090CFE2E6F4E065917491882777FD8095B7
:103BE000982F0E9442AFDF91CF911F910F91FF90CC
:103BF000EF90DF90CF90BF90AF909F908F907F908D
:103C00006F905F904F90089560E08091440890918C
:103C100045082ADF6093400870934108809342086A
:103C20009093430880913E0890913F087DDE609319
:103C30003A0870933B0880933C0890933D088FB7F7
:103C4000F894109232088FBF089520911402309199
:103C50001502409116025091170260E070E08FE764
:103C600093E40E94A7AE60931208709313088093A8
:103C7000140890931508089597FF03C080913908A0
:103C800004C0FC01E45FF74F808190E00895CF937A
:103C9000DF93D82FC62FC19561E00E9451A86C2FE9
:103CA0008D2F0E948AA86C2F70E08D2FDF91CF910D
:103CB0000C9447A7CF93C1E020E030E048E452E401
:103CC00060914008709141088091420890914308AA
:103CD0000E94A3B018160CF0C0E06C2F86E090E0B4
:103CE000CF91D5CF2F923F924F925F926F927F925A
:103CF0008F929F92AF92BF92CF92DF92EF92FF92FC
:103D00000F931F93CF93DF93CDB7DEB728970FB6EE
:103D1000F894DEBF0FBECDBF80913208882309F42E
:103D2000F8C172DF8090400890904108A09042084E
:103D3000B09043080091480810914908B8018827BD
:103D400077FD8095982F0E9442AFA50194010E94B3
:103D5000C6AD6B017C0160931A0870931B088093B9
:103D60001C0890931D0820E030E040E251E40E94DE
:103D7000A3B0181624F481E080931108F7C020E066
:103D800030E040E251ECC701B6010E94A0AE87FDD1
:103D900002C0012B21F481E0809311080CC18091B5
:103DA0001108882351F010922E0810922F081092BB
:103DB00030081092310810921108209118023091A9
:103DC000190240911A0250911B02C701B6010E94CC
:103DD00075B169837A838B839C8360932608709383
:103DE0002708809328089093290820912E08309165
:103DF0002F084091300850913108C701B6010E9448
:103E0000C7AD2B013C012090160830901708109187
:103E10001808009119089101412F502F0E94A0AE5F
:103E200087FD14C0209012083090130810911408D8
:103E3000009115089101412F502FB201C3010E943A
:103E4000A3B018161CF01201162D072DC101A12FC9
:103E5000B02F80932E0890932F08A0933008B09332
:103E600031082091140230911502409116025091B0
:103E70001702B101812F902F0E9475B16D837E834F
:103E80008F83988760932208709323088093240877
:103E90009093250820912A0830912B0840912C08F6
:103EA00050912D08C501B4010E94C6AD20911002A9
:103EB0003091110240911202509113020E9475B18B
:103EC00020ED3CEC4CE45DE30E9475B12B013C011C
:103ED00023E333E343E75FE360911E0870911F081B
:103EE00080912008909121080E9475B19B01AC013E
:103EF000C301B2010E94C7AD2B013C0160931E08B3
:103F000070931F0880932008909321082D813E8193
:103F10004F81588569817A818B819C810E94C7ADD0
:103F2000A30192010E94C6AD2B013C0120E030E0CC
:103F30004FE753E40E94A3B020E030E0A901181637
:103F4000E4F4C701B6010E94A3B018167CF4A701DF
:103F50009601B101812F902F0E94C6AD60932E086B
:103F600070932F088093300890933108412C512C86
:103F70009FE7692E93E4792E21C0C301B2010E940C
:103F8000A0AE87FF1BC020E030E0A901C701B60149
:103F90000E94A0AE87FF0FC0A7019601B101812F3B
:103FA000902F0E94C6AD60932E0870932F088093C7
:103FB000300890933108412C512C320180922A080C
:103FC00090922B08A0922C08B0922D0860910408C2
:103FD00070910508882777FD8095982F0E9442AF41
:103FE0009B01AC01C501B4010E94A3B01816DCF41A
:103FF0006091080270910902882777FD8095982FBB
:104000000E9442AF9B01AC01C501B4010E94A0AE69
:1040100087FF09C0C301B2010E940FAF7595679574
:1040200060930C0802C010920C080E9431A9009104
:1040300008081091090820910A0830910B08601BAC
:10404000710B820B930B653C79408105910558F00B
:1040500031DE0E9431A960930808709309088093AB
:104060000A0890930B080E9431A900910D08109145
:104070000E0820910F0830911008601B710B820B05
:10408000930B683873418105910508F442C00E9482
:1040900031A960930D0870930E0880930F089093D8
:1040A0001008C0903A08D0903B08E0903C08F0908F
:1040B0003D0820E030E040E751E4C701B6010E942E
:1040C000A3B018161CF520E030E046E153E4C70128
:1040D000B6010E94A0AE87FF19C06091460870919A
:1040E0004708882777FD8095982F0E9442AF9B0153
:1040F000AC01C701B6010E94A3B087FD03C01092B6
:10410000390807C08FE78093390803C01092390837
:10411000A59828960FB6F894DEBF0FBECDBFDF91ED
:10412000CF911F910F91FF90EF90DF90CF90BF90B4
:10413000AF909F908F907F906F905F904F903F9047
:104140002F900895CF93DF931092160810921708BE
:10415000109218081092190820911402309115023B
:10416000409116025091170260E070E08FE793E4EF
:104170000E94A7AE609312087093130880931408EE
:10418000909315086D9A80910101806180930101DF
:104190009D9A8091010180628093010187ED809357
:1041A0007A0010927E0010927D0080917E008160E6
:1041B00080937E0080917E00826080937E0080915B
:1041C0007E00846080937E0080E888BD80916E00D0
:1041D000846080936E006AEF70E080E090E00E945F
:1041E00060A98FE090E0909305088093040860E058
:1041F00080910A0290910B0237DC20E030E040E72A
:1042000051E40E94A0AE87FF0AC080910A029091FB
:104210000B02409790930B0280930A02E8CF8BE346
:1042200091E0909309028093080260E08091060873
:104230009091070819DC20E030E84DE953E40E9432
:10424000A3B0181654F48091060890910708409680
:104250009093070880930608E8CFC0910208D09198
:104260000308CE0161DB20E030E046E153E40E9428
:10427000A3B0181634F46096D0930308C0930208D4
:10428000ECCFDF91CF9108950895109249081092D4
:104290004808109247081092460810920C0875982A
:1042A000109247081092460810923908A598089570
:1042B0002F923F924F925F926F927F928F929F9236
:1042C000AF92BF92CF92DF92EF92FF920F931F9324
:1042D000CF93DF93CDB7DEB7AE970FB6F894DEBFBE
:1042E0000FBECDBF6B8F7C8F8D8F292E5A8749874C
:1042F0003CA72BA70E9431A96F8F78A389A39AA30B
:104300000E9431A96FA378A789A79AA729853A8522
:10431000121613061CF0E4E2F3E017C0E7E3F3E043
:104320008191882339F09091C00095FFFCCF809354
:10433000C600F6CF8091C00085FFFCCF1BC29091D4
:10434000C00095FFFCCF8093C60081918111F7CF0B
:104350008091C00085FFFCCF8AE08093C60095DF86
:1043600049855A858FE7452B99F1809339088F8DC0
:1043700098A1A9A1BAA1898B9A8BAB8BBC8B8D8795
:104380009E87AF87B88B1D8290E4988FACE1A98F90
:10439000B6E4BA8F1DA61D8A1E8A1F8A2FE730E059
:1043A00040E050E029833A834B835C83EFE74E2E55
:1043B000512C612C712C1BA21CA21DA21EA231E04B
:1043C0003E8F1C861B86312C00E010E01EA605C027
:1043D00080930C08CCCF0E949C7680913208882371
:1043E00009F4F6C011DC49855A85452B51F030900F
:1043F0003A0800913B0810913C0850913D085EA797
:1044000009C0309040080091410810914208809105
:1044100043088EA7232D302F412F5EA56DA57D89E2
:104420008E899F890E94A3B018162CF03DA60D8B93
:104430001E8B9EA59F8B232D302F412F5EA56D8156
:10444000788D898D9A8D0E94A0AE87FD05C03D8232
:10445000088F198FAEA5AA8F0E9431A92FA138A568
:1044600049A55AA5621B730B840B950B653C7940DB
:104470008105910538F01EDC0E9431A96FA378A751
:1044800089A79AA74E8D442309F44FC02B8D3C8DEC
:104490004D8D522D632D702F812F9EA50E94A3B0AC
:1044A00018160CF095C00E9431A929893A894B89C8
:1044B0005C89621B730B840B950B69387341810512
:1044C000910508F485C0D301C20129813A814B814D
:1044D0005C81821B930BA40BB50B49855A85B5955E
:1044E000A79597958795452B19F08093390802C0B9
:1044F00080930C080E9431A96D877E878F87988BE7
:10450000DC01CB0129893A894B895C89821B930B99
:10451000A40BB50B8BA39CA3ADA3BEA33B8D3DA762
:104520004C8D4D8B5D8D5E8B2F8A2B8D3C8D4D8DF3
:10453000522D632D702F812F9EA50E94A0AE87FF64
:10454000EEC20E9431A92D853E854F855889621B98
:10455000730B840B950B693873418105910508F441
:10456000DEC20E9431A9698B7A8B8B8B9C8BDC011C
:10457000CB012D853E854F855889821B930BA40B5B
:10458000B50B4B855C85452B09F010C189819A815B
:10459000AB81BC81840D951DA61DB71D29853A856B
:1045A000B595A79597958795232B09F4B5C2809368
:1045B00039084B855C854F5F5F4F5C874B875B8D10
:1045C0005D838C8D888F9D8D998F2A8EA1E0AE8F13
:1045D00020E030E040EA51E46B8D7C8D8D8D922D92
:1045E0000E94C7AD9B01AC01632D702F812F9EA54A
:1045F0000E94A3B0181694F4EFEFF2E084918823A0
:1046000041F09091C00095FFFCCF8093C600319699
:10461000F5CF8091C00085FFFCCFACC00E9431A9CE
:104620002F8D38A149A15AA1621B730B840B950BE6
:10463000613D77408105910508F44FC049855A8551
:10464000452B81F0E0903908F12CE9EFF2E08491FC
:104650008823C1F09091C00095FFFCCF8093C600E5
:104660003196F5CFE0900C08F12CE3EFF2E0849165
:10467000882341F09091C00095FFFCCF8093C60045
:104680003196F5CF22E030E0432D502F612F7EA5EB
:104690008CE99DE00E94308BEFEEF2E0849188235C
:1046A00041F09091C00095FFFCCF8093C6003196F9
:1046B000F5CF4AE050E0B7018CE99DE00E945A8AAC
:1046C0008091C00085FFFCCF8AE08093C6000E94E5
:1046D00031A96F8F78A389A39AA30E9431A96B0196
:1046E0007C010E9431A989889A88AB88BC882D8575
:1046F0003E854F855889820E931EA41EB51EC8188C
:10470000D908EA08FB08C60ED71EE81EF91E31E8D4
:10471000C3163FE4D30632E1E306F10490F0E2ED84
:10472000F2E08491882341F09091C00095FFFCCF86
:104730008093C6003196F5CF8091C00085FFFCCFF5
:1047400019C04B855C858BA59CA5841795070CF03B
:1047500042CEE6E7F2E08491882341F09091C000D8
:1047600095FFFCCF8093C6003196F5CF8091C000B5
:1047700085FFFCCF8AE08093C600AE960FB6F89412
:10478000DEBF0FBECDBFDF91CF911F910F91FF9084
:10479000EF90DF90CF90BF90AF909F908F907F90E1
:1047A0006F905F904F903F902F9008958BA09CA0AA
:1047B000ADA0BEA0880E991EAA1EBB1E2BA13CA1B7
:1047C0004DA15EA1281B390B4A0B5B0BCA01B90135
:1047D00029813A814B815C810E943BB2A501940101
:1047E0000E94A0B2240D351D461D571D24313105F0
:1047F0004105510504F129013A013CEE43165104EB
:10480000610471042CF06BEE462E512C612C712C3E
:1048100040E84416510461047104DCF08EEF90E02E
:10482000A0E0B0E084199509A609B70989839A83A5
:10483000AB83BC8312C054E1452E512C612C712CEA
:1048400024E130E040E050E029833A834B835C83ED
:1048500004C049825A826B827C82E8E6F3E084914C
:10486000882341F09091C00095FFFCCF8093C60053
:104870003196F5CF2AE030E0B301A2018CE99DE04A
:104880000E94378AE3E6F3E08491882341F0909117
:10489000C00095FFFCCF8093C6003196F5CF2AE08B
:1048A00030E049815A816B817C818CE99DE00E94D6
:1048B000378AECE5F3E08491882341F09091C000C1
:1048C00095FFFCCF8093C6003196F5CF22E030E013
:1048D0004D81588D698D7A8D8CE99DE00E94308BD9
:1048E000E5E5F3E08491882341F09091C00095FFC5
:1048F000FCCF8093C6003196F5CF22E030E04DA585
:104900005D896E897F898CE99DE00E94308B809162
:10491000C00085FFFCCF8AE08093C6002B853C85D4
:10492000233031050CF432CE69817A818B819C81F0
:104930000E9442AF20E030E040E850E40E9475B1B0
:104940006B017C012D81388D498D5A8D6DA57D8936
:104950008E899F890E94C6AD20ED3FE049E450E476
:104960000E9475B120E030E040E05FE30E9475B145
:104970009B01AC01C701B6010E94A7AE6B017C018F
:10498000C501B4010E9442AF20E030E04AE754E4A0
:104990000E94A7AE4B015C01EFE4F3E08491882311
:1049A00041F09091C00095FFFCCF8093C6003196F6
:1049B000F5CF22E030E0B701A6018CE99DE00E942E
:1049C000308BE9E4F3E08491882341F09091C000BA
:1049D00095FFFCCF8093C6003196F5CF22E030E002
:1049E000B501A4018CE99DE00E94308B8091C0004C
:1049F00085FFFCCF8AE08093C6002AE939E949E1C6
:104A00005FE3C701B6010E9475B16B017C019B0198
:104A1000AC010E94C7ADA50194010E94A7AE6D83B1
:104A20007E838F839887A5019401C701B6010E94F8
:104A300075B120E030E040E05EE30E9475B14B01CB
:104A40005C01EBE3F3E08491882341F09091C00096
:104A500095FFFCCF8093C6003196F5CF8091C000C2
:104A600085FFFCCF8AE08093C600E5E3F3E0849104
:104A7000882341F09091C00095FFFCCF8093C60041
:104A80003196F5CF22E030E0B701A6018CE99DE038
:104A90000E94308B8091C00085FFFCCF8AE080931C
:104AA000C600EFE2F3E08491882341F09091C000CA
:104AB00095FFFCCF8093C6003196F5CF22E030E021
:104AC0004D815E816F8178858CE99DE00E94308BFD
:104AD0008091C00085FFFCCF8AE08093C600E9E2A8
:104AE000F3E08491882341F09091C00095FFFCCFC2
:104AF0008093C6003196F5CF22E030E0B501A401E5
:104B00008CE99DE00E94308B8091C00085FFFCCF36
:104B10008AE08093C6003ACD80930C084ACD1E8E61
:104B200057CDCF93C82FB1DB0E94E949811134C022
:104B3000E5E3FEE09491992341F08091C00085FF68
:104B4000FCCF9093C6003196F5CF6C2F70E04AE011
:104B500050E08CE99DE00E945A8A8091C00085FF58
:104B6000FCCF8AE08093C600ECE2F2E084918823D7
:104B700041F09091C00095FFFCCF8093C600319624
:104B8000F5CF8091C00085FFFCCF8AE08093C600FE
:104B90008FE192E00E940D76CF910C94AA49CF93B9
:104BA000C82F73DB0E94E949811134C0E5E3FEE0C0
:104BB0009491992341F08091C00085FFFCCF9093A0
:104BC000C6003196F5CF6C2F70E04AE050E08CE9DA
:104BD0009DE00E945A8A8091C00085FFFCCF8AE048
:104BE0008093C600E2EFF1E08491882341F0909138
:104BF000C00095FFFCCF8093C6003196F5CF809121
:104C0000C00085FFFCCF8AE08093C60085EE91E06E
:104C10000E940D76CF910C94AA49A5980E94E9496B
:104C2000811125C0E5E3FEE08491882341F0909155
:104C3000C00095FFFCCF8093C6003196F5CFEBEA1C
:104C4000F1E08491882341F09091C00095FFFCCF62
:104C50008093C6003196F5CF8091C00085FFFCCFD0
:104C60008AE08093C6008AE991E00E940D760C9458
:104C7000AA491F920F920FB60F9211240BB60F92F2
:104C80000F931F932F933F934F935F936F937F9354
:104C90008F939F93AF93BF93CF93DF93EF93FF9344
:104CA00080910702811112C080910C088093010845
:104CB000882311F0759A01C0759880913908809306
:104CC0000008882311F0A59A01C0A59890910108C9
:104CD00080910702981708F47598909100088091C8
:104CE0000702981708F4A598809107028F5F8F77C5
:104CF000809307028091060290E08B30910508F0C6
:104D000093C0FC01EE58FF4F0C94BCB210927B0094
:104D100080E480937C0080917A00806480937A00A4
:104D20000E94167681E019C02091780030917900B8
:104D30008091FC079091FD07A091FE07B091FF07BD
:104D4000820F931FA11DB11D8093FC079093FD0757
:104D5000A093FE07B093FF0782E08093060264C031
:104D600010927B0082E480937C0080917A008064C2
:104D700080937A000E94167683E0EFCF209178002E
:104D8000309179008091F8079091F907A091FA0786
:104D9000B091FB07820F931FA11DB11D8093F807EF
:104DA0009093F907A093FA07B093FB0784E0D5CF5F
:104DB00010927B0081E480937C0080917A00806473
:104DC00080937A000E94167685E0C7CF2091780004
:104DD000309179008091F4079091F507A091F60742
:104DE000B091F707820F931FA11DB11D8093F407A7
:104DF0009093F507A093F607B093F70786E0ADCF41
:104E00000E94167687E0A9CF88E0A7CF0E94167689
:104E100089E0A3CF109206028091F3078F5F809301
:104E2000F30702C0109206028091F307803108F464
:104E300063C080913208811110C08091FC0790916D
:104E4000FD0790934508809344088091F80790915E
:104E5000F90790933F0880933E0881E080933208E1
:104E60001092F3071092FC071092FD071092FE07B4
:104E70001092FF071092F4071092F5071092F607B0
:104E80001092F7071092EF071092F0071092F107B7
:104E90001092F2071092F8071092F9071092FA0791
:104EA0001092FB0720914408309145088091060834
:104EB000909107088217930714F080E032DE20916A
:104EC00044083091450880910A0290910B022817FE
:104ED000390714F080E063DE20913E0830913F08EE
:104EE0008091020890910308821793072CF010928A
:104EF00047081092460891DE00E010E0E801CC0F70
:104F0000DD1FCD5CD74F888199811816190644F4AE
:104F100061E0802F0E94D59388819981019709C013
:104F2000892B49F060E0802F0E94D5938881998178
:104F30000196998388830F5F1F4F03301105F1F6A7
:104F4000FF91EF91DF91CF91BF91AF919F918F91A1
:104F50007F916F915F914F913F912F911F910F9191
:104F60000F900BBE0F900FBE0F901F9018952CEA5C
:104F700035EC47E25EE30C9475B12CEA35EC47E280
:104F80005EE30C94A7AE2CEA35EC47E25EE30C94AA
:104F9000A7AE2CEA35EC47E25EE30C9475B1CF93F3
:104FA000DF93EC0160E08E810E948AA881E090E0AE
:104FB0000E9484A961E08E810E948AA881E090E02D
:104FC0000E9484A960E08E810E948AA884E690E015
:104FD000DF91CF910C9484A9CF92DF92EF92FF9250
:104FE0000F931F93CF93DF937C01C0E0D0E0C62ED8
:104FF000D12C87010C0F1D1F61E0F80187810E94F1
:1050000051A8B6010C2E02C0759567950A94E2F777
:105010006170F80187810E948AA82196C430D10569
:1050200041F7C701DF91CF911F910F91FF90EF9052
:10503000DF90CF90B4CFCF92DF92EF92FF920F9399
:105040001F93CF93DF937C01C0E0D0E0C62ED12C1C
:1050500087010C0F1D1F61E0F80187810E9451A894
:10506000B6010C2E02C0759567950A94E2F761703F
:10507000F80187810E948AA82196C830D10541F79E
:10508000C701DF91CF911F910F91FF90EF90DF90BB
:10509000CF9085CF1F93CF93DF93EC01162F642F12
:1050A0008C810E948AA88D818F3F19F060E00E9458
:1050B0008AA88F85612F84FF05C0CE01DF91CF9133
:1050C0001F91B9CF70E084E0759567958A95E1F7F7
:1050D000CE0182DF612FCE01DF91CF911F917CCF76
:1050E00040E0D8CF61E0FCDF80E496E00C9484A936
:1050F00062E0F6DF80E496E00C9484A9CF93DF931E
:10510000CDB7DEB728970FB6F894DEBF0FBECDBF80
:1051100028E0E7EAF2E0DE01119601900D922A956F
:10512000E1F7FC012389421710F04FEF420FFE0117
:105130003196E40FF11DE40FF11D2081260F206848
:10514000622F28960FB6F894DEBF0FBECDBFDF9159
:10515000CF91C6CFFC016089262F2460208B6C6024
:10516000BFCFCF93DF93EC01423018F08F8588607A
:105170008F874B8B1C8A222329F0413019F48F85AD
:1051800084608F8780E593EC0E9484A960E08C8125
:105190000E948AA860E08E810E948AA88D818F3F3C
:1051A00019F060E00E948AA86F8564FD19C063E071
:1051B000CE0112DF84E991E10E9484A963E0CE016F
:1051C0000BDF84E991E10E9484A963E0CE0104DF52
:1051D00086E990E00E9484A962E0CE01FDDE13C062
:1051E0006062CE017DDF84E991E10E9484A96F8530
:1051F0006062CE0175DF86E990E00E9484A96F8528
:105200006062CE016DDF6F856062CE0169DF84E090
:10521000888BCE019FDFCE0165DF82E0898B66E05F
:10522000CE01DF91CF915CCF6F927F928F92AF9240
:10523000CF92EF920F931F93CF93DF93CDB7DEB74B
:105240003C01162F842F5E854F8538899989F3019B
:10525000848325830683E782C086A186828653875E
:1052600044873587968761E00E9451A8F3018581C4
:105270008F3F19F061E00E9451A861E0F30186813F
:105280000E9451A8112319F0F301178603C080E191
:10529000F301878720E041E060E1C301DF91CF9116
:1052A0001F910F91EF90CF90AF908F907F906F9064
:1052B00058CF8F92AF92CF92EF920F93DC0113965B
:1052C0001C921E921297E5E6F3E0ED93FC931F9279
:1052D0001F921F921F928C2CAE2CC02EE22E042FF8
:1052E0002FEF462F61E0A0DF0F900F900F900F90EF
:1052F0000F91EF90CF90AF908F900895CF93DF9361
:10530000EC01423018F08F8588608F874B8B1C8AA8
:10531000222329F0413019F48F8584608F8780E53E
:1053200093EC0E9484A960E08C810E948AA860E0CE
:105330008E810E948AA88D818F3F19F060E00E94C3
:105340008AA86F8564FD19C063E0CE0145DE84E95B
:1053500091E10E9484A963E0CE013EDE84E991E1FF
:105360000E9484A963E0CE0137DE86E990E00E94C6
:1053700084A962E0CE0130DE13C06062CE01B0DEEF
:1053800084E991E10E9484A96F856062CE01A8DE64
:1053900086E990E00E9484A96F856062CE01A0DE5C
:1053A0006F856062CE019CDE84E0888BCE01D2DE08
:1053B000CE019EDE82E0898B66E0CE0191DE40E088
:1053C00068E0CE019BDE6EE873E0CE010E94BEADC8
:1053D00041E068E0CE0192DE6EE873E0CE010E940B
:1053E000BEAD42E066E0CE0189DE6CE873E0CE013E
:1053F000DF91CF910C94BEADCF92DF92EF92FF92EE
:105400000F931F93CF93DF931F921F92CDB7DEB7F9
:105410008C01677088E0689FB00111246064C80146
:1054200049835A835DDE4981C42E5A81D52EE12CF1
:10543000F12CD6016D916D01D801ED91FC91019097
:10544000F081E02DC8011995BFEFEB1AFB0AE8E0E7
:10545000EE16F10471F70F900F90DF91CF911F912D
:105460000F91FF90EF90DF90CF90089541E012DE12
:1054700081E090E008952F923F924F925F926F9259
:105480007F928F929F92AF92BF92CF92DF92EF92D4
:10549000FF920F931F93CF93DF93CDB7DEB7CF5417
:1054A000D1090FB6F894DEBF0FBECDBF1C017E8FB1
:1054B0006D8F4A012FAB09AF2896EFAE28972C9637
:1054C000ACAEBDAECEAEDFAE2C9734E0239F500124
:1054D0001124FC01EA0DFB1D80819181A281B38121
:1054E000898F9A8FAB8FBC8FDA01AA0DBB1DBCAF21
:1054F000ABAF4D905D906D907C90A3019201698D52
:105500007A8D8B8D9C8D0E94C7AD21966CAF7DAF3F
:105510008EAF9FAF2197B4E00B9F80011124F10162
:10552000E00FF11F20813181428153812F8F38A3F9
:1055300049A35AA3A401400F511F23965FAF4EAF5A
:105540002397DA01CD90DD90ED90FC90A7019601B4
:105550006F8D78A189A19AA10E94C7AD27966CAFE3
:105560007DAF8EAF9FAF27972896EFAD2897B4E019
:10557000EB9FC0011124F101E80FF91F2081318157
:10558000428153812BA33CA34DA35EA3ED8DFE8DE1
:10559000E80FF91F60817181828193810E94C6ADFD
:1055A0006FA378A789A79AA7AD8DBE8D1C968D9104
:1055B0009D910D90BC91A02D60968CAF9DAFAEAF2C
:1055C000BFAF6097D1011C962D913D914D915C919B
:1055D0001F972BA73CA74DA75EA7A3019201505888
:1055E0002D8B3E8B4F8B588FD701C601B058898BBE
:1055F0009A8BAB8BBC8BED8DFE8DEA0DFB1D208154
:105600003181428153812FA738AB49AB5AAB2196E8
:105610002CAD3DAD4EAD5FAD21976FA578A989A9A1
:105620009AA90E94C6AD6B017C01ED8DFE8DE00F45
:10563000F11F80819181A281B3818BAB9CABADAB1B
:10564000BEAB27962CAD3DAD4EAD5FAD2797BC01EF
:10565000CD010E94C6AD4B015C01A70196016D8989
:105660007E898F89988D0E9475B12B013C01A5011F
:10567000940169897A898B899C890E9475B19B0103
:10568000AC01C301B2010E94C7AD2B013C01A501D1
:1056900094016D897E898F89988D0E9475B14B0127
:1056A0005C01A701960169897A898B899C890E948E
:1056B00075B19B01AC01C501B4010E94C6ADA30147
:1056C00092010E943AAE6B017C0120E030E0A9011A
:1056D0000E94A0AE87FF0AC02BED3FE049EC50E4EA
:1056E000C701B6010E94C7AD6B017C01AA968FADC0
:1056F000AA97882351F02BED3FE049EC50E4C70115
:10570000B6010E94C6AD6B017C012FA538A949A93D
:105710005AA9698D7A8D8B8D9C8D0E94A0AE8111C6
:105720001FC02BA93CA94DA95EA96F8D78A189A1A5
:105730009AA10E94A0AE811113C020E030E0A9011F
:10574000C701B6010E94A0AE81110AC02BED3FE057
:1057500049EC50E4C701B6010E94C7AD6B017C0162
:10576000A9962CAD3DAD4EAD5FADA997C701B60171
:105770000E9475B12FA138A549A55AA55F770E944F
:10578000B0B04B015C012FE632E143E85AE30E94DE
:10579000A0AE87FDC8C1C501B4010E947DAF0E94C3
:1057A00014AF7A8F698FDB01AB2B21F4E1E0F0E0DD
:1057B000FA8FE98F298D3A8DB90180E090E00E943F
:1057C00040AF4B015C019B01AC01C701B6010E94D7
:1057D000A7AE2B013C01A50194016FA178A589A575
:1057E0009AA50E94A7AE6FA778AB89AB9AAB2BA501
:1057F0003CA54DA55EA560966CAD7DAD8EAD9FAD13
:1058000060970E94C6ADA50194010E94A7AE6BAB44
:105810007CAB8DAB9EAB20E030E040E05FE3C301AA
:10582000B2010E9475B1A30192010E9475B19B0162
:10583000AC0160E070E080E89FE30E94C6AD6FA31A
:1058400078A789A79AA7CE010196FC0128964FADAB
:10585000289734E0439FE00DF11D11242BA13CA1BA
:105860004DA15EA120833183428353832BA53CA5A8
:105870004DA55EA52D873E874F87588BB12C41E003
:1058800050E058A34F8F1C01BFA9A4E0BA9F800D20
:10589000911D112498AF8FAB910159AD44E0549FF5
:1058A000200D311D11243AAF29AFFCA7EBA74F8D76
:1058B00058A1898D9A8D4817590708F01AC188E1B7
:1058C0008B150CF444C02FA138A549A55AA56989A8
:1058D0007A898B899C890E9475B16B017C01A30137
:1058E00092016D897E898F89988D0E9475B1A7017B
:1058F00096010E94C7ADA62E172F982E892E2FA194
:1059000038A549A55AA56D897E898F89988D0E94F1
:1059100075B16B017C01A301920169897A898B8938
:105920009C890E9475B19B01AC01C701B6010E9420
:10593000C6AD6D8B7E8B8F8B988FB3948A2D912FF4
:10594000A92DB82D898B9A8BAB8BBC8B6CC0AF8D7E
:10595000B8A1BD0180E090E00E9440AFA301920198
:105960000E9475B16B017C010E94A4AE698B7A8B99
:105970008B8B9C8BC701B6010E94D8B14B015C0197
:10598000EBADFCADC080D180E280F380F7FAF094FB
:10599000F7F8F0942396AEADBFAD23972D913D91CE
:1059A0004D915C912BA33CA34DA35EA329893A8919
:1059B0004B895C89C701B6010E9475B16D8B7E8BE6
:1059C0008F8B988FA50194016BA17CA18DA19EA1C5
:1059D0000E9475B19B01AC016D897E898F89988D7C
:1059E0000E94C7AD6D8B7E8B8F8B988FA501940124
:1059F000C701B6010E9475B16B017C0129893A8902
:105A00004B895C896BA17CA18DA19EA10E9475B17F
:105A10009B01AC01C701B6010E94C6AD698B7A8BB0
:105A20008B8B9C8BB12C2D893E894F89588D21966B
:105A30006CAD7DAD8EAD9FAD21970E94C7ADEFA936
:105A4000F8AD608371838283938329893A894B8976
:105A50005C8927966CAD7DAD8EAD9FAD27970E947A
:105A6000C7ADA9ADBAAD6D937D938D939C931397FC
:105A70002FA538A949A95AA9EBA5FCA56081718178
:105A8000828193810E94C7ADABA5BCA56D937D9328
:105A90008D939C9313972BA93CA94DA95EA96D8565
:105AA0007E858F8598890E94C7AD6D877E878F8799
:105AB000988BC1010E946A41FE01E659FF4F6F01B8
:105AC0002C96ECACFDAC0EAD1FAD2C979E01235F68
:105AD0003F4FAE01475F5F4FBE016B5F7F4FC1011C
:105AE0000E94779A2F8D38A12F5F3F4F38A32F8FB9
:105AF000DECE2D8D3E8D245F3F4F4D8D5E8D485FF8
:105B00005F4F6D8D7E8D6C5F7F4FDE01A659BF4F5D
:105B10006D012C96ECACFDAC0EAD1FAD2C978D8DB0
:105B20009E8D0E94779AC15BDF4F0FB6F894DEBF5F
:105B30000FBECDBFDF91CF911F910F91FF90EF90DE
:105B4000DF90CF90BF90AF909F908F907F906F909D
:105B50005F904F903F902F900895FC011482178220
:105B6000138212828AEB95E09183808308952AEB59
:105B700035E0FC01318320832781222319F004962C
:105B80000C948C130895CF92DF92EF92FF920F93B3
:105B90001F93CF93DF93EC01875B9F4FDEDFCE0136
:105BA00086599F4FDADF7E0129E8E20EF11C87015A
:105BB0006E0131E4C31A3EEFD30AC801CEDF015EA5
:105BC0001F4F0C151D05C9F7FE01EF53FE4F89E16C
:105BD000818314823596178ACE018C519E4FBDDF8A
:105BE000FE01EB56FD4F108211821282138238960D
:105BF00010821182128213821A821B8218821982E9
:105C00006E0187E6C81A8DEFD80AF601108211825C
:105C100012821382F80111821082FE01ED5FFD4FA6
:105C2000108286E391E0F7019C01119221503040EF
:105C3000E1F7FE01EF55FD4F81E08083C95BDF4F47
:105C4000198218820E9431A968577C4E8F4F9F4F4E
:105C5000F6016083718382839383DF91CF911F91DB
:105C60000F91FF90EF90DF90CF900895FC0120E01E
:105C70003EE2DB014C91403241F0283011F4308398
:105C80003196DB014C91408331962F5F6F5F7F4FE0
:105C90002B3079F7108208952F923F924F925F92A6
:105CA0006F927F928F929F92AF92BF92CF92DF922C
:105CB000EF92FF920F931F93CF93DF93CDB7DEB791
:105CC000CA58D1090FB6F894DEBF0FBECDBF8C0104
:105CD0006B017A014901CA57DF4F1882C658D0407C
:105CE00084E0E80EF11C180191E1290E311CF80145
:105CF000EA5BFF4FC957DF4FF983E883C758D040AD
:105D00003801FEE56F1AFDEF7F0A58018CE5A81AED
:105D10008DEFB80A80E4482E512C4C0E5D1E94E0A5
:105D2000490E511CA101BE016F5F7F4FC7010E9448
:105D3000F61118160CF03CC12C85322F3871303119
:105D400009F09EC0F301808191810197029708F4C8
:105D500097C0BE016F5F7F4FCE0187589F4F86DF90
:105D6000A0961FAEA097F6018081811107C069E659
:105D700073E0CE01815A9F4F0E9418B6B601CE0142
:105D8000815A9F4F0E9418B6BE0167587F4FCE01BF
:105D9000815A9F4F0E9418B669E673E0CE01815A7E
:105DA0009F4F0E9418B6CE01805C9F4FD6DE21E047
:105DB000AE0147585F4FB701C2010E9483158111A0
:105DC00039C0F30180819181892BA1F5EFE2FEE0DA
:105DD0008491882341F09091C00095FFFCCF80937F
:105DE000C6003196F5CFEBE6F3E08191882339F0D8
:105DF0009091C00095FFFCCF8093C600F6CF8091B4
:105E0000C00085FFFCCF8AE08093C600FE01E75802
:105E1000FF4F8191882339F09091C00095FFFCCF0E
:105E20008093C600F6CF8091C00085FFFCCF8AE04A
:105E30008093C6008BE1FE01EC5BFF4FDE0195967F
:105E400001900D928A95E1F724968EAD9FAD24972F
:105E50009CA38BA38AEB95E09AA389A320E030E072
:105E6000AE014F5D5F4FBE01615A7F4FC80114DF25
:105E7000CE0181967CDECE01805C9F4F78DE52CFD2
:105E80008981882309F494C08E3209F44BCF8F3571
:105E900009F448CFF80181898E3209F443CF8F3558
:105EA00009F440CF23FD3ECF81E0303109F080E09E
:105EB000C957DF4FE881F981C758D04080838111ED
:105EC00008C08985873409F02DCF8A858E3709F47B
:105ED00029CF98012C5F3F4FBE016F5F7F4FC901F3
:105EE000C757DF4F2883C958D040C657DF4F388384
:105EF000CA58D040BBDEF30180819181C757DF4F84
:105F00002881C958D040C657DF4F3881CA58D04081
:105F10000097F1F4F6018191882339F09091C00047
:105F200095FFFCCF8093C600F6CFF90181918823BD
:105F300039F09091C00095FFFCCF8093C600F6CF5A
:105F40008091C00085FFFCCF8AE08093C600EACE36
:105F50008130910539F4F501808191810196918319
:105F60008083E0CE029709F0DDCE8114910439F0F0
:105F7000B901C4010E9405B6892B71F419C0CA5732
:105F8000DF4FF881C658D0402F2F30E0F5018081D7
:105F900091812817390761F0CA57DF4FF881C65839
:105FA000D040FF5FCA57DF4FF883C658D040BACE03
:105FB000C657DF4F0FB6F894DEBF0FBECDBFDF91DF
:105FC000CF911F910F91FF90EF90DF90CF90BF90F6
:105FD000AF909F908F907F906F905F904F903F9089
:105FE0002F9008950F931F93CF93DF93CDB7DEB714
:105FF0006F970FB6F894DEBF0FBECDBF8C01FC01CA
:10600000EE55FD4F1182108240E050E0BA01835BF3
:106010009F4F0E94A912C801875B9F4F2BE1FC0193
:106020003496DE01159601900D922A95E1F7FC0158
:10603000828193819C838B838AEB95E09A83898309
:1060400020E030E0AE014F5F5F4F62E973E0C801CE
:1060500023DECE0101968BDD6F960FB6F894DEBF7E
:106060000FBECDBFDF91CF911F910F9108952BE10E
:10607000FB013496DC01149601900D922A95E1F70C
:10608000FB0122813381FC01338322830895EF9247
:10609000FF920F931F93CF93DF93EC011B82FC01C0
:1060A000E05BFF4F8081882329F0CE01835B9F4F07
:1060B0000E948C137E018FE3E81A8EEFF80A45E305
:1060C00060E0C7010E94BF3A81111FC0EFE2FEE00D
:1060D0008491882341F09091C00095FFFCCF80937C
:1060E000C6003196F5CFE7E4F6E08491882341F0CD
:1060F0009091C00095FFFCCF8093C6003196F5CFFC
:106100008091C00085FFFCCF77C08E010A531E4FDF
:1061100041E0B701C8010E945A1B811126C040E02E
:10612000B701C8010E945A1B81111FC0E5E3FEE0C0
:106130008491882341F09091C00095FFFCCF80931B
:10614000C6003196F5CFE4E3F6E08491882341F070
:106150009091C00095FFFCCF8093C6003196F5CF9B
:106160008091C00085FFFCCF47C0B801CE01835BA2
:106170009F4F0E94991081111FC0E5E3FEE08491BA
:10618000882341F09091C00095FFFCCF8093C6001A
:106190003196F5CFE4E2F6E08491882341F09091C6
:1061A000C00095FFFCCF8093C6003196F5CF80915B
:1061B000C00085FFFCCF20C081E08B83EFE2FEE0D2
:1061C0008491882341F09091C00095FFFCCF80938B
:1061D000C6003196F5CFE9E1F6E08491882341F0DD
:1061E0009091C00095FFFCCF8093C6003196F5CF0B
:1061F0008091C00085FFFCCF8AE08093C6008E01AD
:10620000075B1F4FB801CE0186599F4F30DFC85939
:10621000DF4F19830883DF91CF911F910F91FF907A
:10622000EF900895FC01128213820895FC012381EE
:10623000222311F021E022830895FC012281211103
:1062400012820895AF92BF92CF92DF92EF92FF92A7
:106250000F931F93CF93DF931F92CDB7DEB78C01BF
:106260008FE2FB0181935F01D12C41E07801F1E4E1
:10627000EF1AFEEFFF0A9FE1C92E2D2D30E0F70146
:106280008081918128173907D8F4C29EC001C39E2E
:10629000900D112483579F4FB501800F911F4983A3
:1062A0000E944010C50149815C010196F5012081E1
:1062B000222321F04D3810F44F5FF6CFD394DDCF79
:1062C00047FD11C0B501C80188519E4F0F90DF9165
:1062D000CF911F910F91FF90EF90DF90CF90BF90E3
:1062E000AF900C944010F50110820F90DF91CF9188
:1062F0001F910F91FF90EF90DF90CF90BF90AF90E4
:1063000008953F924F925F926F927F928F929F92E9
:10631000AF92BF92CF92DF92EF92FF920F931F93B3
:10632000CF93DF93CDB7DEB7AC970FB6F894DEBF4F
:106330000FBECDBF7C015B01FC018381882309F482
:1063400008C1C70188519E4F0E948C13F701128229
:10635000CE0101966C0101DC270198E6490E511C23
:10636000C701875B9F4FF20191838083F501808194
:106370008F3209F084C06FE270E0C5010E9423B63D
:106380008C010F5F1F4F2AE0322E0115110509F411
:106390007CC06FE270E0C8010E9423B64C010097F8
:1063A00009F474C00817190708F070C03C01601A9E
:1063B000710AA301B801CE0180960E944CB6E0E2BA
:1063C000F0E0EC0FFD1FE60DF71D1082FE01B09608
:1063D0008191882339F09091C00095FFFCCF809384
:1063E000C600F6CF8091C00085FFFCCF3092C6007A
:1063F000F201608171816115710519F06C5F7F4F49
:1064000002C060E070E021E0AE01405E5F4FCE016F
:1064100005960E94831581112BC0EEEFF4E0849164
:10642000882341F09091C00095FFFCCF8093C60077
:106430003196F5CFFE01B0968191882339F0909185
:10644000C00095FFFCCF8093C600F6CFECEFF4E0E0
:106450008491882341F09091C00095FFFCCF8093F8
:10646000C6003196F5CF8091C00085FFFCCF6CC08F
:10647000F201D182C08284010F5F1F4F86CFC70116
:1064800086599F4FF201918380838501F2018081BB
:106490009181009711F0049602C080E090E0B8016D
:1064A0000E945916882339F1EEEEF4E08491882396
:1064B00041F09091C00095FFFCCF8093C6003196CB
:1064C000F5CFF8018191882339F09091C00095FFB4
:1064D000FCCF8093C600F6CF8091C00085FFFCCF33
:1064E0008AE08093C600F701E356FD4F10821182C7
:1064F000128213822CC0E6EDF4E08491882341F0EF
:106500009091C00095FFFCCF8093C6003196F5CFE7
:10651000F8018191882339F09091C00095FFFCCF5C
:106520008093C600F6CFE4EDF4E08491882341F037
:106530009091C00095FFFCCF8093C6003196F5CFB7
:106540008091C00085FFFCCF8AE08093C600C60121
:106550000EDBAC960FB6F894DEBF0FBECDBFDF9159
:10656000CF911F910F91FF90EF90DF90CF90BF9050
:10657000AF909F908F907F906F905F904F903F90E3
:106580000895CF93DF93EC018B818823C1F1E2EC76
:10659000F4E08491882341F09091C00095FFFCCFF6
:1065A0008093C6003196F5CFFE01E356FD4F408142
:1065B0005181628173812AE030E08CE99DE00E9484
:1065C000868AE0ECF4E08491882341F09091C00049
:1065D00095FFFCCF8093C6003196F5CFCB56DD4FAB
:1065E000488159816A817B812AE030E08CE99DE015
:1065F0000E94868A8091C00085FFFCCF11C0E0EB2D
:10660000F4E08491882341F09091C00095FFFCCF85
:106610008093C6003196F5CF8091C00085FFFCCFF6
:106620008AE08093C600DF91CF910895AF92BF9228
:10663000CF92DF92EF92FF920F931F93CF93DF934E
:106640005C01EB01FB0101900020E9F78F01015093
:106650001109061B170B6C01F8E1CF1AFEEFDF0AD8
:10666000F60110826EE470E0CE010E9423B67C0138
:10667000009729F4F8013197EC0FFD1F0DC060E27F
:1066800070E00E9423B6EC0121966AE270E0C70137
:106690000E9423B6FC0131978DE081838AE08283DA
:1066A0001382BE01C5018C519E4F0E94438BF6019F
:1066B0008081882309F1E5E3FEE08491882341F09D
:1066C0009091C00095FFFCCF8093C6003196F5CF26
:1066D000EAE9F4E08491882341F09091C00095FFAD
:1066E000FCCF8093C6003196F5CF8091C00085FF26
:1066F000FCCF8AE08093C600DF91CF911F910F916C
:10670000FF90EF90DF90CF90BF90AF9008952F92C1
:106710003F924F925F926F927F928F929F92AF9231
:10672000BF92CF92DF92EF92FF920F931F93CF937E
:10673000DF93CDB7DEB7CC55D1090FB6F894DEBFE5
:106740000FBECDBF4C018C010F551D4F662339F094
:10675000F8011082F401838181111DC015C0F80178
:106760008081882309F4AFC0F401E756FD4FC08053
:10677000D180E280F3800E9431A9C616D706E806D0
:10678000F90608F4A0C0E4CFC40181DCF4018381E0
:10679000882309F498C07401F7E4EF0EF11CF701A7
:1067A00081818F9380818F9381E994E09F938F9370
:1067B0008E01015C1F4F1F930F930E945BB60F90D9
:1067C0000F900F900F900F900F90B12CF801019047
:1067D0000020E9F73197E01BF10BBE1684F4680145
:1067E000CB0CD11CB7FCDA94F6018081992787FD88
:1067F00090950E9498B5F6018083B394E7CFFDE4AD
:106800008F0E911C40E050E0BA01C4010E94A91211
:10681000512CCE0101966C013AE8632E34E0732EC0
:106820005E0191E2A90EB11C40E050E0B601C40146
:106830000E94F6111816DCF5412CF601019000209B
:10684000E9F73197EC19FD094E1674F41601240C82
:10685000311C47FC3A94F101808190E00E9498B588
:10686000F10180834394E9CF8A858E37E9F245E0D0
:1068700050E0B801C6010E943EB6892BA9F61F93CD
:106880000F937F926F92BF92AF920E945BB6C50149
:106890000E94C03D86E894E00E94333E0F900F9026
:1068A0000F900F900F900F9055245394BDCF51101F
:1068B00004C08FEF9FEFF70104C0F7018081918141
:1068C000019691838083C45ADF4F0FB6F894DEBFE0
:1068D0000FBECDBFDF91CF911F910F91FF90EF9031
:1068E000DF90CF90BF90AF909F908F907F906F90F0
:1068F0005F904F903F902F9008950F931F93CF93E9
:10690000DF93EC018C0108511E4FC8010E94421315
:10691000C8010E948C1318821982DF91CF911F91B8
:106920000F910895CF92DF92EF92FF920F931F93F2
:10693000CF93DF93CDB7DEB76F970FB6F894DEBF76
:106940000FBECDBF8C016A017C0188E6E80EF11C08
:10695000C80186599F4FF70191838083E65CFD4F04
:1069600022E030E03183208332967183608340E0FF
:1069700050E0BA0104960E94A912F701808191812A
:106980002BE1FC013496DE01159601900D922A95BB
:10699000E1F7FC01828193819C838B838AEB95E0F4
:1069A0009A8389839601AE014F5F5F4F62E973E07E
:1069B000C80172D9CE010196DAD86F960FB6F89455
:1069C000DEBF0FBECDBFDF91CF911F910F91FF9022
:1069D000EF90DF90CF9008952F923F924F925F9269
:1069E0006F927F928F929F92AF92BF92CF92DF92DF
:1069F000EF92FF920F931F93CF93DF93CDB7DEB744
:106A0000AC970FB6F894DEBF0FBECDBF8C016B0103
:106A1000342EDC0113968C91882309F4EEC2F80120
:106A2000E551FE4F8081882309F4F5C02111C1C0D2
:106A30007801BDEFEB1AFB0AF7018081882361F131
:106A4000E5E3FEE08491882341F09091C00095FF3A
:106A5000FCCF8093C6003196F5CFE6EDF5E084914A
:106A6000882341F09091C00095FFFCCF8093C60031
:106A70003196F5CF4AE050E061E070E08CE99DE0AE
:106A80000E945A8A8091C00085FFFCCF8AE08093E3
:106A9000C6000E942245B1C2EFE2FEE08491882345
:106AA00041F09091C00095FFFCCF8093C6003196D5
:106AB000F5CFEDEBF5E08491882341F09091C00093
:106AC00095FFFCCF8093C6003196F5CFF6018191FA
:106AD000882339F09091C00095FFFCCF8093C600C9
:106AE000F6CFE2EBF5E08491882341F09091C0006D
:106AF00095FFFCCF8093C6003196F5CFD7018C91DE
:106B00005DE8B52EB801B89E600D711D1124685F57
:106B10007D4FC80197DBF7018081F801B89EE00D39
:106B2000F11D1124E85FFD4F8191882339F0909188
:106B3000C00095FFFCCF8093C600F6CFECEAF5E0ED
:106B40008491882341F09091C00095FFFCCF809301
:106B5000C6003196F5CF5801F3E6AF1AFDEFBF0A34
:106B6000D5014D915D916D917C912AE030E08CE9E9
:106B70009DE00E94868A8091C00085FFFCCF8AE05C
:106B80008093C600F7012081F80184E0289FE00D82
:106B9000F11D1124EC5FFD4FD5014D915D916D917B
:106BA0007C9140835183628373832F5FF70120833D
:106BB0002CC0EFE2FEE08491882341F09091C00068
:106BC00095FFFCCF8093C6003196F5CFEBE9F5E059
:106BD0008491882341F09091C00095FFFCCF809371
:106BE000C6003196F5CFF6018191882339F0909156
:106BF000C00095FFFCCF8093C600F6CF8091C00007
:106C000085FFFCCF8AE08093C600C80188519E4F63
:106C10000E948C1330C0F801ED5FFD4F1082EFE24F
:106C2000FEE08491882341F09091C00095FFFCCF55
:106C30008093C6003196F5CFEAE8F5E08491882389
:106C400041F09091C00095FFFCCF8093C600319633
:106C5000F5CFF6018191882339F09091C00095FF1E
:106C6000FCCF8093C600F6CF8091C00085FFFCCF9B
:106C70008AE08093C600D80112961C92FE013196DC
:106C80005F01CF010E94AD2D2801F8E64F0E511C87
:106C9000C801875B9F4FD2018D939C93F601808141
:106CA0008F3209F084C06FE270E0C6010E9423B603
:106CB00001967C014AE0242EE114F10409F47DC020
:106CC0006FE270E0C7010E9423B64C01009709F4FF
:106CD00075C0E816F90608F071C03C016E187F080F
:106CE000A301B701CE0180960E944CB6E0E2F0E02D
:106CF000EC0FFD1FE60DF71D1082FE01B09681918D
:106D0000882339F09091C00095FFFCCF8093C60096
:106D1000F6CF8091C00085FFFCCF2092C600D20143
:106D20006D917C916115710519F06C5F7F4F02C008
:106D300060E070E021E0AE01405E5F4FCE0105965D
:106D40000E94831581112BC0E6E7F5E0849188232A
:106D500041F09091C00095FFFCCF8093C600319622
:106D6000F5CFFE01B0968191882339F09091C00053
:106D700095FFFCCF8093C600F6CFE4E7F5E0849161
:106D8000882341F09091C00095FFFCCF8093C6000E
:106D90003196F5CF8091C00085FFFCCF02C1F20192
:106DA000B182A0827401FFEFEF1AFF0A85CFC801FC
:106DB00086599F4FD2018D939C937601F801E8513B
:106DC000FE4F4F01332009F4B1C0D2016D917C9187
:106DD0006115710519F06C5F7F4F02C060E070E0D3
:106DE00021E0A701C4010E948315882309F474C01F
:106DF000F40181899289A389B489F801EB56FD4F8A
:106E000080839183A283B383E6E6F5E08491D80181
:106E1000AB56BD4F882349F09091C00095FFFCCF41
:106E20008093C60031968491F5CFF7018191882334
:106E300039F09091C00095FFFCCF8093C600F6CF4B
:106E4000EEE5F5E08491882341F09091C00095FF34
:106E5000FCCF8093C6003196F5CF4D915D916D9139
:106E60007C912AE030E08CE99DE00E94868A809146
:106E7000C00085FFFCCF8AE08093C600F801E3568E
:106E8000FD4F1082118212821382E0E5F5E08491B9
:106E9000882341F09091C00095FFFCCF8093C600FD
:106EA0003196F5CF8091C00085FFFCCF8AE08093BA
:106EB000C600A70160E070E0C80134DDD80151963A
:106EC0008C91882319F0C801419601C0C7010E9426
:106ED00048728EE793E08CC0ECE3F5E08491882360
:106EE00041F09091C00095FFFCCF8093C600319691
:106EF000F5CFF7018191882339F09091C00095FF7B
:106F0000FCCF8093C600F6CFEAE3F5E084918823B6
:106F100041F09091C00095FFFCCF8093C600319660
:106F2000F5CF8091C00085FFFCCF3BC0F2016081AE
:106F300071816115710519F06C5F7F4F02C060E0CF
:106F400070E026E5A701C4010E94831581112DC0C0
:106F5000E6E2F5E08491882341F09091C00095FF2E
:106F6000FCCF8093C6003196F5CFF701819188233D
:106F700039F09091C00095FFFCCF8093C600F6CF0A
:106F8000E4E2F5E08491882341F09091C00095FF00
:106F9000FCCF8093C6003196F5CF8091C00085FF6D
:106FA000FCCF8AE08093C60025C081E0D8018C9395
:106FB000E2E1F5E08491882341F09091C00095FFD3
:106FC000FCCF8093C6003196F5CFF60181918823DE
:106FD00039F09091C00095FFFCCF8093C600F6CFAA
:106FE0008091C00085FFFCCF8AE08093C600C70176
:106FF0000E944872C5010E94B72DAC960FB6F89456
:10700000DEBF0FBECDBFDF91CF911F910F91FF90DB
:10701000EF90DF90CF90BF90AF909F908F907F9038
:107020006F905F904F903F902F90089521E0FC016A
:10703000218340E0D1CCCF92DF92EF92FF920F9369
:107040001F93CF93DF93CDB7DEB76F970FB6F8944A
:10705000DEBF0FBECDBF8C016C0128E6C20ED11C75
:1070600086599F4FF60191838083E65CFD4F21E0B6
:1070700030E0318320837801FCE5EF1AFDEFFF0A51
:10708000F7011182108240E050E0BA0104960E949C
:10709000A912F601808191812BE1FC013496DE0179
:1070A000159601900D922A95E1F7FC01828193815A
:1070B0009C838B838AEB95E09A83898320E030E080
:1070C000AE014F5F5F4F62E973E0C8010E944C2E32
:1070D000CE0101960E94B72DF701808191816F96B4
:1070E0000FB6F894DEBF0FBECDBFDF91CF911F91D9
:1070F0000F91FF90EF90DF90CF900895AF92BF92E5
:10710000CF92DF92EF92FF920F931F93CF93DF9373
:10711000CDB7DEB76F970FB6F894DEBF0FBECDBF09
:107120008C017B01CE0101960E94AD2DF801EF5834
:10713000FF4F80816801811104C029E4C20ED11C77
:1071400003C08AE6C80ED11C21E0A701B6016C5F1E
:107150007F4FCE0105960E94831581112DC0EFE26D
:10716000FEE08491882341F09091C00095FFFCCF10
:107170008093C6003196F5CFE0E7F4E08491882350
:1071800041F09091C00095FFFCCF8093C6003196EE
:10719000F5CFF7018191882339F09091C00095FFD8
:1071A000FCCF8093C600F6CF8091C00085FFFCCF56
:1071B0008AE08093C60036C0F801E154FE4F80811A
:1071C00091818A30910530F59C012F5F3F4F3183CB
:1071D00020832FE1289F7001299FF00C112429E8BA
:1071E000E20EF11CE00EF11E5C01B701C7014F96E3
:1071F0000E94373081E0A81AB1082FE1E21AF108A5
:107200008FEFA816B80689F7B601C80187579F4FB8
:107210000E943730BE016F5F7F4FC80186599F4F74
:107220000E943730CE0101960E94B72D6F960FB69F
:10723000F894DEBF0FBECDBFDF91CF911F910F91AC
:10724000FF90EF90DF90CF90BF90AF900895EF92B6
:10725000FF920F931F93CF93DF93EC01C154DE4F46
:107260002881398121153105F9F0215031093983FF
:1072700028838C0107571F4FB80186599F4F0E94E2
:107280003730C80100E010E07C012FE1E20EF11C74
:10729000288139810217130738F40F5F1F4FB70198
:1072A0000E943730C701F0CFDF91CF911F910F912E
:1072B000FF90EF900895EF92FF920F931F93CF935B
:1072C000DF93EC010E943D938E010D5F1D4FF8018D
:1072D00080819E0128513E4F79018823A1F1C90187
:1072E0000E948C13F801808181508083BE01FDE8EB
:1072F0008F9F600D711D1124685F7D4F21E041E07B
:10730000CE016ADBF8018081FE0124E0829FE00D5E
:10731000F11D1124EC5FFD4F408151816281738129
:10732000FE01E356FD4F4083518362837383C7019F
:107330000E94A912CE01DF91CF911F910F91FF9072
:10734000EF900C9416310E94B393C7010E948C13E6
:107350001A8284E694E0DF91CF911F910F91FF9004
:10736000EF9081C48FEF8EBD0DB407FEFDCF8EB5BB
:1073700008958EBD0DB407FEFDCF089561E0FC01B8
:1073800080810C948AA8FC012281322F306A3695C4
:107390003CBD20FD06C031E0263009F430E0232F4B
:1073A00001C020E02DBD60E0FC0180810C948AA822
:1073B000CF92DF92EF92FF920F931F93CF93DF93C1
:1073C000EC018B017A010E9431A96B01CBDF8B8329
:1073D0008F3F49F40E9431A96C197D096D327140CB
:1073E000A8F381E144C08E3F11F08FE040C0E1146A
:1073F000F104D9F0C70101972FEF2EBDF8014FEF2F
:107400009F01201B310B2817390738F40DB407FEF4
:10741000FDCF2EB521934EBDF3CF0DB407FEFDCFAA
:107420002EB5F801E80FF91F2083D801E00EF11EF8
:10743000C12CD12CAE15BF0579F08D91ED2DFF2714
:10744000E827EE0FFF1FEC5AF94F85919491DC2C41
:10745000CC24C826D926EECF85DF082F10E0102FC8
:10746000002780DF082BC016D10631F080E2898327
:10747000CE0184DF80E003C0CE0180DF81E0DF91B8
:10748000CF911F910F91FF90EF90DF90CF900895D3
:107490000F931F93CF93DF93EB010E9431A98B01D0
:1074A00061DF8F3F49F00E9431A9601B710B6C179F
:1074B0007D07B0F380E001C081E0DF91CF911F91A3
:1074C0000F910895CF92DF92FF920F931F93CF9366
:1074D000DF9300D01F92CDB7DEB76C01F62E298363
:1074E0003A834B835C834FDF6CE271E0C601D0DFEF
:1074F0008F2D80643EDF08E110E05C814B813A8192
:107500002981DA01C901002E04C0B695A795979587
:1075100087950A94D2F729833A834B835C8329DFCA
:107520000850110929813A814B815C81083F8FEF16
:10753000180739F7FF2029F0E8E0FE1621F08FEF59
:1075400003C085E901C087E814DFFCE0FF1201C039
:1075500009DF10E007DFF601838387FF04C01F3FC8
:1075600011F01F5FF7CF0F900F900F900F90DF91EA
:10757000CF911F910F91FF90DF90CF900895BF9210
:10758000CF92DF92EF92FF920F931F93CF93DF93EF
:10759000EC01B62E1C82198248830E9431A98B010E
:1075A00061E088810E9451A8CE01E8DE60E082E3BC
:1075B0000E9451A861E083E30E9451A861E084E346
:1075C0000E9451A861E085E30E9451A861E085E333
:1075D0000E948AA885E08A8382E58CBD1DBC6AE092
:1075E000F62E8FEFC6DEFA94E1F720E030E0A90135
:1075F00060E0CE0167DFF82E8B8381E0F81649F05A
:107600000E9431A9601B710B613D774070F381E0EE
:1076100046C02AEA31E040E050E068E0CE0152DFA7
:1076200082FF02C0FC820CC054E0F52E9BDE8B83EF
:10763000FA94E1F78A3A11F082E031C082E08C835B
:107640008C81823031F4C12CD12CE12C40E4F42E19
:1076500003C0C12CD12C760120E030E0A90167E302
:10766000CE0130DFA701960169E2CE012BDF8B83CB
:10767000882349F00E9431A9601B710B613D77405E
:1076800058F38AE00CC08C818230B1F420E030E005
:10769000A9016AE3CE0116DF882329F088E08983F7
:1076A000CE016CDE14C05EDE807C803C11F483E091
:1076B0008C8358DE57DE56DECE0160DE86E08B1509
:1076C00018F488E1898303C0BA8281E001C080E0B8
:1076D000DF91CF911F910F91FF90EF90DF90CF90AE
:1076E000BF900895AF92BF92CF92DF92EF92FF9238
:1076F0000F931F93CF93DF93EC016A017B01890104
:107700008C81833039F0F9E0CC0CDD1CEE1CFF1CC1
:10771000FA95D1F773E0B72EE4E0AE2EBA94A70144
:10772000960161E1CE01CEDE882311F0A98207C067
:1077300040E052E0B801CE013BDE81110EC0CE0127
:10774000BB2049F01BDE20E030E0A9016CE0CE0157
:10775000B9DE1982E3CF12DE80E0DF91CF911F9175
:107760000F91FF90EF90DF90CF90BF90AF90089572
:10777000CF93DF93EC016EBD20E030E00DB407FE47
:10778000FDCFFA01E20FF31F80818EBD0DB407FE1D
:10779000FDCF81818EBD2E5F3F4F211582E03807DE
:1077A00069F70DB407FEFDCF8FEFE3DD8FEFE1DD6D
:1077B000D9DD8B838F71853031F083E18983CE01F0
:1077C000DDDD80E001C081E0DF91CF9108950F936E
:1077D0001F93CF93DF93EC0189018C81833039F0C3
:1077E000B9E0440F551F661F771FBA95D1F79A016C
:1077F000AB0168E1CE0166DE882311F086E01EC091
:10780000A8016EEFCE01B4DF8823C9F068E572E00D
:10781000CE013EDE182F811102C087E10FC020E0AB
:1078200030E0A9016DE0CE014DDE811106C09ADD88
:10783000811103C0CE01A2DD05C086E18983CE019E
:107840009DDD10E0812FDF91CF911F910F91089561
:10785000FC01659175918591949108952F923F92C5
:107860004F925F926F927F928F929F92AF92BF9250
:10787000CF92DF92EF92FF920F931F93CF93DF93FC
:1078800000D000D0CDB7DEB71C01FC01E051F24FB3
:1078900014919C01220F331F220F331F3E832D832F
:1078A0002C5B354F4901F90110821182128213823B
:1078B00020E53AE04CE45AE068E47AE084E49AE0B7
:1078C0000E943EA48D819E818150924FC1DF6B0149
:1078D0007C01612F772767FD7095872F972F0E9476
:1078E00042AF2B013C012D813E81215F354F590173
:1078F00020E030E040EC5FE3C701B6010E9475B1C3
:10790000A30192010E9475B1F501608371838283A6
:1079100093832D813E81215A3D4F3C832B83F90176
:107920006081718182819381609321027093220230
:10793000809323029093240220E030E040E752E459
:107940000E94A7AE20E3C22E2AE0D22E7B018C013A
:107950002BE13AE047E15AE063E17AE08FE09AE018
:107960000E94779A0E943D93F40110821182128244
:10797000138220E53AE04CE45AE068E47AE084E4DB
:107980009AE00E943EA42D813E812D50324F3A83D1
:107990002983C9015DDF9058A30192010E9475B14E
:1079A000F501608371838283938320E030E040E7B8
:1079B00052E4609121027091220280912302909101
:1079C00024020E94A7AE7B018C012BE13AE047E143
:1079D0005AE063E17AE08FE09AE00E94779A0E9491
:1079E0003D9389819A8134DF9B01AC010E94C7AD30
:1079F000A30192010E9475B1F501608371838283B6
:107A0000938320E030E040E05FE3EB81FC81608124
:107A10007181828193810E9475B16093210270937C
:107A20002202809323029093240220E030E040E77A
:107A300052E40E94A7AE7B018C012BE13AE047E1C2
:107A40005AE063E17AE08FE09AE00E94779A0E9420
:107A50003D938D819E81855F914FFADE0D811E8160
:107A6000085C154FF80120813181428153810E94C9
:107A7000C7ADF40160837183828393838D819E817E
:107A80008D5D914FE5DE2D813E812D5B3D4F79016E
:107A9000F80120813181428153810E94C7ADF701F5
:107AA00060837183828393838D819E81895E914FF0
:107AB000CFDE2D813E81295C3D4F7901F801208187
:107AC0003181428153810E94C7ADF7016083718388
:107AD00082839383F40180819181A281B381F50136
:107AE00080839183A283B383109221021092220299
:107AF00010922302109224020E94EA8BF101EB5CA7
:107B0000F54F81E0808326960FB6F894DEBF0FBE56
:107B1000CDBFDF91CF911F910F91FF90EF90DF903C
:107B2000CF90BF90AF909F908F907F906F905F901D
:107B30004F903F902F900895FC012491222341F013
:107B40003091C00035FFFCCF2093C6000196F4CFE2
:107B500022E030E08CE99DE00C94308BFC01249114
:107B6000222341F03091C00035FFFCCF2093C600A6
:107B70000196F4CF2AE030E08CE99DE00C94868AEF
:107B80002091640830916508243031050CF06AC0FA
:107B9000409166085091670860E6649F9001659F78
:107BA000300D1124BC01C9018259974F0E9437B68C
:107BB000EFE2FEE08491882341F09091C00095FFB0
:107BC000FCCF8093C6003196F5CFE5EEFDE08491C1
:107BD000882341F09091C00095FFFCCF8093C600B0
:107BE0003196F5CF809166089091670820E6289F2E
:107BF000F001299FF00D1124E259F74F819188235C
:107C000039F09091C00095FFFCCF8093C600F6CF6D
:107C1000E3EEFDE08491882341F09091C00095FF50
:107C2000FCCF8093C6003196F5CF8091C00085FFD0
:107C3000FCCF8AE08093C600809166089091670827
:107C4000019664E070E00E946BB2909367088093A5
:107C50006608809164089091650801969093650884
:107C60008093640808952091640830916508243059
:107C700031050CF06AC0409166085091670860E6D3
:107C8000649F9001659F300D1124BC01C901825988
:107C9000974F0E94A0B5EFE2FEE08491882341F067
:107CA0009091C00095FFFCCF8093C6003196F5CF30
:107CB000E8EDFDE08491882341F09091C00095FFAC
:107CC000FCCF8093C6003196F5CF809166089091E5
:107CD000670820E6289FF001299FF00D1124E25942
:107CE000F74F8191882339F09091C00095FFFCCF28
:107CF0008093C600F6CFE6EDFDE08491882341F045
:107D00009091C00095FFFCCF8093C6003196F5CFCF
:107D10008091C00085FFFCCF8AE08093C6008091EF
:107D2000660890916708019664E070E00E946BB26B
:107D30009093670880936608809164089091650825
:107D40000196909365088093640808959B9AA39880
:107D50000895FCDF40E052EC61E070E08CE99DE0CA
:107D60000E944689E0EDFDE08491882341F09091E6
:107D7000C00095FFFCCF8093C6003196F5CF80916F
:107D8000C00085FFFCCF8AE08093C6008FE29EE0B2
:107D9000FC012491222341F03091C00035FFFCCF3B
:107DA0002093C6003196F5CF24B720FF14C0E8EC2D
:107DB000FDE03491332341F04091C00045FFFCCFFA
:107DC0003093C6003196F5CF3091C00035FFFCCF1F
:107DD0003AE03093C60021FF14C0E8EBFDE0349197
:107DE000332341F04091C00045FFFCCF3093C600E3
:107DF0003196F5CF3091C00035FFFCCF3AE030939B
:107E0000C60022FF14C0E7EAFDE03491332341F0BD
:107E10004091C00045FFFCCF3093C6003196F5CFAE
:107E20003091C00035FFFCCF3AE03093C60023FF0D
:107E300014C0E7E9FDE03491332341F04091C000E4
:107E400045FFFCCF3093C6003196F5CF3091C0008E
:107E500035FFFCCF3AE03093C60025FF14C0E7E8B9
:107E6000FDE02491222341F03091C00035FFFCCF8A
:107E70002093C6003196F5CF2091C00025FFFCCF9E
:107E80002AE02093C60014BEE0E8FDE024912223FE
:107E900041F03091C00035FFFCCF2093C6003196F1
:107EA000F5CFEAE7FDE02491222341F03091C000B4
:107EB00035FFFCCF2093C6003196F5CF2091C0004E
:107EC00025FFFCCF2AE02093C600FC012491EFE2BD
:107ED000FEE0222349F03091C00035FFFCCF209313
:107EE000C60031962491F5CFEAE6FDE024912223E5
:107EF00041F03091C00035FFFCCF2093C600319691
:107F0000F5CFE5E5FDE02491222341F03091C0005A
:107F100035FFFCCF2093C6003196F5CFE9E4FDE0B4
:107F20002491222341F03091C00035FFFCCF2093F3
:107F3000C6003196F5CFE2E3FDE02491222341F023
:107F40003091C00035FFFCCF2093C6003196F5CFAD
:107F50002091C00025FFFCCF2AE02093C600E7E275
:107F6000FDE02491222341F03091C00035FFFCCF89
:107F70002093C6003196F5CFEBE1FDE0249122235A
:107F800041F03091C00035FFFCCF2093C600319600
:107F9000F5CF2091C00025FFFCCF2AE02093C6003A
:107FA000FC018491EFE2FEE0882349F09091C0004B
:107FB00095FFFCCF8093C60031968491F5CFECE01D
:107FC000FDE08491882341F09091C00095FFFCCFA3
:107FD0008093C6003196F5CF0E9458964AE050E053
:107FE000BC018CE99DE00E945A8AE5EFFCE0849197
:107FF000882341F09091C00095FFFCCF8093C6008C
:108000003196F5CF4AE050E060ED74E08CE99DE0F8
:108010000E945A8A8091C00085FFFCCF8AE080933D
:10802000C60010926A0810926B0810926C081092A9
:108030006D080E9467870E9439830E94A2200E94D7
:10804000279A0E9446950E947076FFEF23ED80E309
:10805000F15020408040E1F700C000000895809179
:108060005E0890915F0860E070E001960C94F7B2B2
:1080700080915E0890915F084AE050E060E070E017
:1080800001960C945FB4682F772767FD7095209157
:1080900068083091690840E6429FC001439F900DF7
:1080A00011248259974F0E9423B690935F088093C2
:1080B0005E0821E0892B09F420E0822F08950E94B8
:1080C00031A960935A0870935B0880935C08909381
:1080D0005D0808950E9431A960935A0870935B0867
:1080E00080935C0890935D08E0916808F0916908BE
:1080F000E659F74F8081811114C0ECEFF8E08491CC
:10810000882341F09091C00095FFFCCF8093C6007A
:108110003196F5CF8091C00085FFFCCF8AE0809337
:10812000C60008958CE99DE00E949889EFEFF8E081
:108130008491882341F09091C00095FFFCCF8093FB
:10814000C6003196F5CF4091F3095091F409609142
:10815000F5097091F6094F5F5F4F6F4F7F4F2AE02F
:1081600030E08CE99DE00E94378A8091C00085FF55
:10817000FCCF8AE08093C600ADCF8F929F92AF92E2
:10818000BF92CF92DF92EF92FF920F931F93CF9304
:10819000DF9337ECE32E34E0F32E04E41AE0CFE073
:1081A000DAE049E5C42E4AE0D42EF70181917F013F
:1081B0006ADF882311F153DF4B015C01F6018081F6
:1081C000811103C06091EE0901C061E070E080E0C0
:1081D00090E00E9442AFF8012081318142815381B9
:1081E0000E9475B19B01AC01C501B4010E94C7ADED
:1081F000688379838A839B8309C0F8018081918198
:10820000A281B38188839983AA83BB830C5F1F4FAC
:108210002496FFEFCF1ADF0A8BECE81684E0F8060D
:1082200021F686E430DF8823D1F019DF6B017C0171
:108230006093FF097093000A8093010A9093020AE9
:1082400020E030E0A9010E94A3B0181644F4C092C7
:108250002102D0922202E0922302F0922402DF91C6
:10826000CF911F910F91FF90EF90DF90CF90BF9033
:10827000AF909F908F90089580DF89E404DF88237A
:1082800051F0EDDE6093030A7093040A8093050AAF
:108290009093060A08C01092030A1092040A1092E2
:1082A000050A1092060A8AE4EEDE882351F0D7DE32
:1082B0006093070A7093080A8093090A90930A0A48
:1082C00008951092070A1092080A1092090A109253
:1082D0000A0A0895CF92DF92EF92FF92CF93DF9335
:1082E000EC01C0904302D0904402E0904502F0902F
:1082F0004602A7019601688179818A819B810E944B
:10830000A0AE87FF04C0C882D982EA82FB82C090F7
:108310004702D0904802E0904902F0904A02A7013B
:1083200096016C817D818E819F810E94A0AE87FF26
:1083300004C0CC82DD82EE82FF8220E030E0A90121
:1083400060914B0270914C0280914D0290914E02CF
:108350000E94C7AD6B017C019B01AC0168857985EA
:108360008A859B850E94A0AE87FF04C0C886D986F7
:10837000EA86FB86C0903702D0903802E09039023E
:10838000F0903A02A7019601688179818A819B81E8
:108390000E94A3B0181624F4C882D982EA82FB8214
:1083A000C0903B02D0903C02E0903D02F0903E0233
:1083B000A70196016C817D818E819F810E94A3B06F
:1083C000181624F4CC82DD82EE82FF82C0903F0238
:1083D000D0904002E0904102F0904202A701960145
:1083E000688579858A859B850E94A3B0181624F438
:1083F000C886D986EA86FB86DF91CF91FF90EF9001
:10840000DF90CF900895CF92DF92EF92FF920F937B
:108410001F938FE09AE05EDF0E9431A960935A08B3
:1084200070935B0880935C0890935D0820910F0A1D
:108430003091100A4091110A5091120A6091440A39
:108440007091450A8091460A9091470A0E94A0AE19
:10845000811179C02091130A3091140A4091150AB4
:108460005091160A6091480A7091490A80914A0A0F
:1084700090914B0A0E94A0AE811165C020E030E0CF
:1084800040E752E460912102709122028091230220
:10849000909124020E94A7AE50E3C52E5AE0D52E3B
:1084A0007B018C012BE13AE047E15AE063E17AE09D
:1084B0008FE09AE00E94779A80910F0A9091100ABB
:1084C000A091110AB091120A8093440A9093450A30
:1084D000A093460AB093470A8091130A9091140A18
:1084E000A091150AB091160A8093480A9093490A00
:1084F000A0934A0AB0934B0A8091170A9091180AE8
:10850000A091190AB0911A0A80934C0A90934D0ACF
:10851000A0934E0AB0934F0A80911B0A90911C0AB7
:10852000A0911D0AB0911E0A8093500A9093510A9F
:10853000A093520AB093530A1F910F91FF90EF90AE
:10854000DF90CF90089560915D0270915E02882760
:1085500077FD8095982F0E9442AF209121023091A3
:10856000220240912302509124020E9475B120E022
:1085700030E040E752E40E94A7AE20E030E048EC53
:1085800052E488CFCF92DF92EF92FF92CF93C62F23
:10859000E091300AF0E0882309F4C2C0DF01A45D55
:1085A000B54F8C91811196C18091440A9091450AF2
:1085B000A091460AB091470A80930F0A9093100A3F
:1085C000A093110AB093120A8091480A9091490A27
:1085D000A0914A0AB0914B0A8093130A9093140A0F
:1085E000A093150AB093160A80914C0A90914D0AF7
:1085F000A0914E0AB0914F0A8093170A9093180ADF
:10860000A093190AB0931A0AC090500AD090510A48
:10861000E090520AF090530AC0921B0AD0921C0AB2
:10862000E0921D0AF0921E0AEE0FFF1FEE0FFF1FD1
:10863000E15BFD4F2081318142815381CC2349F0A0
:1086400060912F027091300280913102909132023C
:1086500008C060913302709134028091350290918C
:1086600036020E94A7AE9B01AC01C701B6010E9471
:10867000C7AD6093500A7093510A8093520A909349
:10868000530A80E59AE00E94E3A4C0902102D090B2
:108690002202E0902302F090240220E030E040E744
:1086A00052E460912B0270912C0280912D029091E6
:1086B0002E020E9475B16093210270932202809372
:1086C000230290932402E091300AF0E0E45DF54F3C
:1086D00081E0808398DE2091280A3091290A409118
:1086E0002A0A50912B0A60914C0A70914D0A809190
:1086F0004E0A90914F0A0E94C6AD60934C0A709347
:108700004D0A80934E0A90934F0A20E53AE04CE4DC
:108710005AE068E47AE084E49AE00E943EA4D1C082
:10872000E45DF54F8081882309F4D4C08091440A28
:108730009091450AA091460AB091470A80930F0A8A
:108740009093100AA093110AB093120A8091480ADC
:108750009091490AA0914A0AB0914B0A8093130A5A
:108760009093140AA093150AB093160A60914C0ACC
:1087700070914D0A80914E0A90914F0A6093170AAA
:108780007093180A8093190A90931A0AC090500A9D
:10879000D090510AE090520AF090530AC0921B0AFE
:1087A000D0921C0AE0921D0AF0921E0A2091280A1B
:1087B0003091290A40912A0A50912B0A0E94C7AD94
:1087C00060934C0A70934D0A80934E0A90934F0A1F
:1087D00020E53AE04CE45AE068E47AE084E49AE088
:1087E0000E943EA4F090300ACC2389F02091200A08
:1087F0003091210A4091220A5091230A60912F0260
:1088000070913002809131029091320210C020911B
:10881000240A3091250A4091260A5091270A609136
:1088200033027091340280913502909136020E9499
:10883000C7AD24E0F29EF0011124E15BFD4F2081E1
:108840003181428153810E94A7AE9B01AC016091AE
:10885000500A7091510A8091520A9091530A0E94D5
:10886000C6AD6093500A7093510A8093520A909358
:10887000530A80E59AE00E94E3A4C0902102D090C0
:108880002202E0902302F090240220E030E040E752
:1088900052E4609127027091280280912902909100
:1088A0002A020E9475B16093210270932202809384
:1088B000230290932402E091300AF0E0E45DF54F4A
:1088C0001082A1DDC0922102D0922202E092230206
:1088D000F0922402CF91FF90EF90DF90CF90089517
:1088E000AF92BF92CF92DF92EF92FF920F931F93BE
:1088F000CF93DF93D82F2091070A3091080A409137
:10890000090A50910A0A6091030A7091040A809141
:10891000050A9091060A0E94B0B0C62F172F082FA3
:10892000F92E60915D0270915E02882777FD809537
:10893000982F0E9442AF2091210230912202409153
:108940002302509124020E9475B120E030E040E7FC
:1089500052E40E94A7AE20E030E048EC52E40E94CE
:10896000A7AE2091300A2F93DF93FF920F931F93AE
:10897000CF935B016C0172E0E72E01E020E043E061
:108980005AE06FE07AE084E49AE00E943B2A80910A
:108990000F0A9091100AA091110AB091120A8093C7
:1089A000440A9093450AA093460AB093470A8091DF
:1089B000130A9091140AA091150AB091160A809397
:1089C000480A9093490AA0934A0AB0934B0A8091AF
:1089D000170A9091180AA091190AB0911A0A809367
:1089E0004C0A90934D0AA0934E0AB0934F0A80917F
:1089F0001B0A90911C0AA0911D0AB0911E0A809337
:108A0000500A9093510AA093520AB093530A0E94BD
:108A100031A960935A0870935B0880935C08909327
:108A20005D080F900F900F900F900F900F90DF91B7
:108A3000CF911F910F91FF90EF90DF90CF90BF905B
:108A4000AF900895F8940E944521179A1092350A24
:108A5000169A1092360A159A1092370A149A60E004
:108A600087E40E9451A8E5E3FEE08491882341F069
:108A70009091C00095FFFCCF8093C6003196F5CF52
:108A8000EDEDF8E08491882341F09091C00095FFCE
:108A9000FCCF8093C6003196F5CF8091C00085FF52
:108AA000FCCF8AE08093C60084ED98E00E940D76AA
:108AB0007894C6E0D0E02197209749F068EC70E008
:108AC00080E090E00E9460A90E949C76F4CFF89428
:108AD000FFCF2F923F924F925F926F927F928F9231
:108AE0009F92AF92BF92CF92DF92EF92FF920F933D
:108AF0001F93CF93DF93CDB7DEB76E970FB6F89481
:108B0000DEBF0FBECDBFB0E6BB2E14E0E12EF12CD0
:108B10000BEBC02E0BE0D02E8AE0A82E9924939464
:108B200080911D0E90911E0E20911F0E3091200EEF
:108B3000821B930B8F779927892B09F41AC2809196
:108B400064089091650804970CF013C28CE99DE0CD
:108B50000E947C89809363082091610830916208AB
:108B60008A3061F08D3051F08A3321F490916008A1
:108B7000992321F02F3531050CF41DC12115310544
:108B800009F437C18091660890916708B89E30015A
:108B9000B99E700C1124F301E20FF31FE259F74F55
:108BA000108220916008211101C110926008FC011F
:108BB000E659F74F108283010259174F6EE470E0B7
:108BC000C8010E9423B60097F1F190935F0880934B
:108BD0005E08801B910B860D971D4AE050E060E017
:108BE00070E08159974F0E945FB46093F7097093CA
:108BF000F8098093F9099093FA094090F30950908D
:108C0000F4096090F5097090F6092FEF421A520AA4
:108C1000620A720A0091660810916708641575056A
:108C20008605970509F4E8C0B09EC001B19E900D7D
:108C3000112467ED7CE08259974F0E94CEB5892BB5
:108C400009F0DAC069C16AE270E0C8010E9423B687
:108C5000892B09F444C0E5E3FEE08491882341F0C8
:108C60009091C00095FFFCCF8093C6003196F5CF60
:108C7000E1E3FCE08491882341F09091C00095FFEE
:108C8000FCCF8093C6003196F5CF4091F309509107
:108C9000F4096091F5097091F6092AE030E08CE959
:108CA0009DE00E94378A8091C00085FFFCCF8AE05A
:108CB0008093C6001092620810926108C0C2809131
:108CC000F7099091F809A091F909B091FA098093F8
:108CD000F3099093F409A093F509B093F6098091F4
:108CE000660890916708B89E8001B99E100D112406
:108CF000C8018259974F3C0167E470E00E9423B697
:108D0000009781F190935F0880935E088619970918
:108D1000800F911F60E070E08159974F0E94F7B279
:108D20000E940FAF64307105E8F480914C088823ED
:108D3000C9F0F6018491EBEBFBE0882349F09091B8
:108D4000C00095FFFCCF8093C60031968491F5CF8B
:108D50008091C00085FFFCCFA092C60081EB9BE014
:108D60000E9400760091660810916708B09EC001CD
:108D7000B19E900D112463E973E08259974F0E94D0
:108D80002EB6892B09F45EDEC8010196B7010E9458
:108D90006BB2909367088093660880916408909105
:108DA00065080196909365088093640810926208A4
:108DB00010926108B5CE8B3311F4909260089091B7
:108DC00060089111ADCE4091660850916708B901D5
:108DD0006F5F7F4F7093620860936108B49EF001EB
:108DE000B59EF00D1124E20FF31FE259F74F808377
:108DF00097CE1092600823C2B09E3001B19E700CD5
:108E00001124C3018259974F1C016AE270E00E944D
:108E100023B6009789F5E5E3FEE08491882341F0CD
:108E20009091C00095FFFCCF8093C6003196F5CF9E
:108E3000EBE5FCE08491882341F09091C00095FF20
:108E4000FCCF8093C6003196F5CF4091F309509145
:108E5000F4096091F5097091F6092AE030E08CE997
:108E60009DE00E94378A8091C00085FFFCCF8AE098
:108E70008093C60057D91ECF20E010E0F301E20F27
:108E8000F11DE259F74F30813A3219F02F5F132765
:108E9000F5CF90935F0880935E0882199309860D41
:108EA000971D60E070E08159974F0E94F7B20E94D1
:108EB0000FAF212F30E02617370709F400CFE5E385
:108EC000FEE08491882341F09091C00095FFFCCF93
:108ED0008093C6003196F5CFE5E8FCE084918823C5
:108EE00041F09091C00095FFFCCF8093C600319671
:108EF000F5CF4091F3095091F4096091F509709113
:108F0000F6092AE030E08CE99DE00E94378A8091E2
:108F1000C00085FFFCCFABCFE5E3FEE08491882362
:108F200041F09091C00095FFFCCF8093C600319630
:108F3000F5CFE4EAFCE08491882341F09091C000F1
:108F400095FFFCCF8093C6003196F5CF4091F30991
:108F50005091F4096091F5097091F6092AE030E02A
:108F60008CE99DE00E94378A8091C00085FFFCCF8C
:108F70007ECF80915F0A882309F461C180916108E6
:108F800090916208892B09F05AC1809164089091F0
:108F90006508892B11F410924A08F8EE2F2EF3E0A1
:108FA0003F2E412C512CACE3CA2ED12CE12CF12CBC
:108FB0008E010F5F1F4FE0E66E2E77247394409171
:108FC000FA0C5091FB0C6091FC0C7091FD0C80919F
:108FD000F20C9091F30CA091F40CB091F50C4817A1
:108FE00059076A077B0708F02AC1809164089091AD
:108FF000650804970CF023C180914A0881111FC1B4
:1090000080914D0C90914E0CA0914F0CB091500C52
:109010008093FA0C9093FB0CA093FC0CB093FD0C86
:1090200085E49CE00E94E011482F809363088A3019
:10903000B9F04D30A9F0433229F420916008222381
:1090400079F002C04A33C9F3209161083091620877
:109050002F3531052CF48F3FFFEF9F0709F0D1C06A
:109060004091FA0C5091FB0C6091FC0C7091FD0C3E
:109070008091F20C9091F30CA091F40CB091F50C4E
:10908000481759076A077B0708F481C0EEE9FBE03F
:109090008491882341F09091C00095FFFCCF80938C
:1090A000C6003196F5CF8091C00085FFFCCFFAE075
:1090B000F093C6000E9431A960934E0870934F0848
:1090C00080935008909351088090520890905308D4
:1090D000A0905408B0905508681979098A099B092D
:1090E000A20191010E947EB249015A01CA01B9014F
:1090F000A70196010E947EB2CA01B901A70196019B
:109100000E947EB27F936F93C501B40120E13EE0DF
:1091100040E050E00E947EB23F932F93AAE8BBE06C
:10912000BF93AF931F930F930E945BB6EFE2FEE0F5
:1091300084910FB6F894DEBF0FBECDBF882349F0EF
:109140009091C00095FFFCCF8093C600319684912A
:10915000F5CFF8018191882339F09091C00095FFF7
:10916000FCCF8093C600F6CF8091C00085FFFCCF76
:109170003AE03093C600C8010E9448728DE59AE03B
:109180000E945B3961E08DE59AE00E94873380910F
:109190006308833211F470924A082091610830917B
:1091A00062082115310509F424CE8091660890915A
:1091B0006708689EF001699EF00D1124E20FF31F0D
:1091C000E259F74F1082FC01E659F74F7082209167
:1091D0006408309165082F5F3F4F309365082093F6
:1091E0006408019664E070E00E946BB29093670897
:1091F00080936608109260081092620810926108CD
:10920000DECE4B3311F4709260084091600841113A
:10921000D2CE4091660850916708B9016F5F7F4FC9
:109220007093620860936108649EF001659EF00D82
:109230001124E20FF31FE259F74F8083C0CE6E96E0
:109240000FB6F894DEBF0FBECDBFDF91CF911F9157
:109250000F91FF90EF90DF90CF90BF90AF909F90D5
:109260008F907F906F905F904F903F902F900895D8
:10927000CF92DF92EF92FF920F931F93CF93C82F5D
:10928000809164089091650803970CF422DC0E9499
:1092900031A9009156081091570820915808309133
:1092A0005908C0905A08D0905B08E0905C08F09094
:1092B0005D086C197D098E099F0906171707280795
:1092C000390728F4012B022B032B09F0BBDB40915B
:1092D0001D0250911E0260911F0270912002452BC9
:1092E000462B472B19F10E9431A900915A08109181
:1092F0005B0820915C0830915D08601B710B820B4C
:10930000930B00911D0210911E0220911F023091BB
:109310002002061717072807390740F490916D0EB1
:1093200080916C0E981302C0CC2349F0CF911F910D
:109330000F91FF90EF90DF90CF900C945B9A179A6B
:109340001092350A169A1092360A159A1092370A18
:10935000149AECCF0E94452180914C08811138C0AD
:1093600081E080934C088091F3099091F409A091D9
:10937000F509B091F6098093EF099093F009A09355
:10938000F109B093F209E5E3FEE08491882341F00E
:109390009091C00095FFFCCF8093C6003196F5CF29
:1093A000EEE5F8E08491882341F09091C00095FFAC
:1093B000FCCF8093C6003196F5CF8091C00085FF29
:1093C000FCCF8AE08093C60084E598E00C94007698
:1093D000089580914C080895CF93DF93EC0180911C
:1093E000300A80934D0884E50E944340811102C0F9
:1093F00080E075C00E942F400E9414AF60934D081A
:109400006623B1F3EFE2FEE08491882341F090916E
:10941000C00095FFFCCF8093C6003196F5CFCD36C6
:10942000D105B9F054F4C836D105B1F0C936D1052B
:1094300009F045C0EDEDF3E021C0CA3DD10531F0A2
:10944000CD3DD105E1F5E8E9F3E036C0EFEAF3E020
:1094500029C0E6ECF3E01CC0E4EFF3E0819188233F
:1094600071F19091C00095FFFCCF8093C600F6CFBC
:109470009091C00095FFFCCF8093C600819181112F
:10948000F7CF1DC09091C00095FFFCCF8093C60020
:1094900081918111F7CF13C09091C00095FFFCCF4F
:1094A0008093C60081918111F7CF09C09091C000CF
:1094B00095FFFCCF8093C60081918111F7CF40E0EA
:1094C00050E060914D088CE99DE00E94918A809166
:1094D000C00085FFFCCF8AE08093C60081E0DF9169
:1094E000CF910895CF92DF92EF92FF922091540A8C
:1094F0002223F1F020E030E040E05FE30E9475B10C
:109500006B017C0120E030E0A9010E94A0AE88231D
:1095100079F0A7019601C701B6010E9475B12BED44
:109520003FE049E450E40E9475B19B01AC0104C0E6
:1095300020E030E040E85FE360E070E080E89FE337
:109540000E94A7AEFF90EF90DF90CF9008956091BA
:109550005302709154028091550290915602C2DFDD
:1095600060934F0270935002809351029093520285
:1095700008953F924F925F926F927F928F929F9247
:10958000AF92BF92CF92DF92EF92FF920F931F9311
:10959000CF93DF93CDB7DEB7E9970FB6F894DEBF70
:1095A0000FBECDBF80E50E9443408823B1F186E421
:1095B0000E9443408823A9F0EAE1F4E081918823E6
:1095C00039F09091C00095FFFCCF8093C600F6CF94
:1095D0008091C00085FFFCCF8AE08093C6000C9488
:1095E000F46082E50E944340882311F40C94F460F7
:1095F000E0E2F4E08191882339F09091C00095FF7A
:10960000FCCF8093C600F6CF8091C00085FFFCCFD1
:109610008AE08093C6000C94F46087E40E94434083
:10962000882309F44CC20E942F400E940FAF6A3079
:10963000710509F4AFC09CF46230710509F44CC0A7
:1096400024F477FF25C00C94F4606330710509F4AD
:109650004EC06430710509F455C00C94F4606A354D
:10966000710509F4D8C154F46B30710509F498C040
:109670006C31710509F49AC00C94F4606B35710576
:1096800009F4CDC16C35710509F4CEC10C94F460B8
:1096900080914C0881110C94F4600E94BD4080912F
:1096A0002D0A8823A9F088E50E944340811110C04B
:1096B00089E50E94434081110BC08AE50E94434026
:1096C000811106C085E40E94434081110C94F7602B
:1096D0000E9403420C94F46080914C0881110C9418
:1096E000F4600E943C4181E0FBD80C94F4608091CE
:1096F0004C0881110C94F4600E943C4180E0F0D849
:109700000C94F46081E89BE00E94007680E50E9462
:109710004340882339F00E942F400E9414AF4B0130
:109720005C0103C0812C912C540183E50E944340CD
:10973000882361F00E942F4020E030E04AE754E4A3
:109740000E9475B10E9414AF4B015C010E943D93D1
:109750000E9431A96B017C01C80CD91CEA1CFB1CBE
:109760000E9431A960935A0870935B0880935C084B
:1097700090935D080E9431A96C157D058E059F05AB
:1097800010F00C94F4600E94721E80E071DD0E9463
:109790009C76F0CF60E081E00E94C2420C94F460BD
:1097A00060E080E00E94C2420C94F460809121024B
:1097B00090912202A0912302B09124028093FB0990
:1097C0009093FC09A093FD09B093FE0980915D027E
:1097D00090915E029093580A8093570A84E690E035
:1097E00090935E0280935D020E9431A960935A08B3
:1097F00070935B0880935C0890935D0881E00E9401
:10980000F18B8091440A9091450AA091460AB0914B
:10981000470A80930F0A9093100AA093110AB093FD
:10982000120A8091480A9091490AA0914A0AB0917F
:109830004B0A8093130A9093140AA093150AB093CD
:10984000160A80914C0A90914D0AA0914E0AB0914F
:109850004F0A8093170A9093180AA093190AB0939D
:109860001A0A8091500A9091510AA091520AB0911F
:10987000530A80931B0A90931C0AA0931D0AB0936D
:109880001E0A1092210210922202109223021092BC
:10989000240288E50E944340882311F090E00AC02A
:1098A00089E50E9443408111F9CF8AE50E94434037
:1098B00091E098279093250291110C94266188E5F8
:1098C0000E94434081110C942661809125028111F0
:1098D0000C942C6189E50E94434081110C942C6109
:1098E00088E50E9443408823D1F00E943840672BCE
:1098F000682B692BA1F00E942F402091380A3091EB
:10990000390A40913A0A50913B0A0E94C7AD6093D0
:10991000440A7093450A8093460A9093470A89E562
:109920000E9443408823D1F00E943840672B682B67
:10993000692BA1F00E942F4020913C0A30913D0AF2
:1099400040913E0A50913F0A0E94C7AD6093480A79
:109950007093490A80934A0A90934B0A809125029A
:1099600081110C9432618AE50E94434081110C946C
:1099700032618AE50E9443408823D1F00E9438403A
:10998000672B682B692BA1F00E942F402091400A81
:109990003091410A4091420A5091430A0E94C7AD5A
:1099A00060934C0A70934D0A80934E0A90934F0A2D
:1099B00020E53AE04CE45AE068E47AE084E49AE096
:1099C0000E943EA480E00E94F18B8091FB0990915F
:1099D000FC09A091FD09B091FE09809321029093AA
:1099E0002202A0932302B09324028091570A9091FF
:1099F000580A90935E0280935D020E9431A96093A1
:109A00005A0870935B0880935C0890935D080E94ED
:109A1000EA8B0C94F4601092EE090C94F46081E0EF
:109A20008093EE090C94F46085E40E944340811118
:109A300002C00E943D9357ECC52E54E0D52E68E33A
:109A4000E62E6AE0F62E04E41AE0B12CF6018191CC
:109A50006F010E944340882339F1F3E0BF120CC02C
:109A60000E942F40F801608371838283938380E595
:109A70009AE00E94E3A418C00E942F40F7012081C1
:109A80003181428153810E94C7ADF80160837183A7
:109A90008283938320E53AE04CE45AE068E47AE07C
:109AA00084E49AE00E943EA4B394F4E0EF0EF11C2B
:109AB0000C5F1F4F24E0B212C9CF0C94F4608DE408
:109AC0000E944340882311F40C9423600E942F408D
:109AD0000E940FAF6537710511F40C94C9550CF055
:109AE000A6C06032710509F4F0C20CF056C06731AF
:109AF000710509F445C254F56231710509F468C76E
:109B0000BCF477FF02C00C94F460623071050CF471
:109B100061C16131710511F00C94F46088E49BE03F
:109B20000E94007617981698159814980C94F46073
:109B30006531710509F418C20CF01CC2643171055D
:109B400011F00C94F460E8E3FBE0EAC16B317105BD
:109B500009F442C2B4F46931710509F429C20CF068
:109B60002DC28DE59AE00E9416310E9431A96093C2
:109B700052087093530880935408909355080C949E
:109B8000F4606E31710509F462C20CF03AC36C31B5
:109B9000710509F427C20C94F4606C35710509F461
:109BA0006AC7ECF46235710509F409C764F46035DD
:109BB000710509F4DAC60CF0E5C66A32710509F4DC
:109BC0007EC30C94F4606435710509F401C70CF48C
:109BD000FAC66535710509F433C70C94F4606B3629
:109BE000710509F4BCC664F46936710509F4DEC375
:109BF0000CF085C66836710509F4A8C30C94F460AE
:109C00006037710509F4BFC334F46D36710509F48A
:109C1000D9C40C94F4606237710509F4CEC7633778
:109C2000710511F00C94F460EEEBF9E0ADC76D3DF9
:109C3000710511F40C94D3590CF04DC06B3C7105B7
:109C400011F40C944D5844F56C38710509F49DC31A
:109C50009CF46837710511F40C94BD566937710591
:109C600011F40C94C2566737710511F00C94F4602E
:109C7000E7E2F4E00C94CD56683C710511F40C94C5
:109C8000B757693C710511F40C942C586E3B710563
:109C900011F00C94F46020C56F3C710511F40C9424
:109CA000095954F46D3C710511F40C948C5814F45A
:109CB0000C946A580C94EC58613D710511F40C94A5
:109CC000645914F40C943E596C3D710511F40C94D4
:109CD000C4590C94F460603931E0730711F40C94AA
:109CE000965B54F56E3291E0790711F40C94505B59
:109CF00084F46C32F1E07F0711F40C94545A14F0A0
:109D00000C948A5A623E710511F40C94F9590C9422
:109D1000F4606E3531E0730711F40C94905F6F3589
:109D200081E0780711F40C94C75F6F32714011F035
:109D30000C94F4600C945E5B6835E2E07E0711F4ED
:109D40000C94745CBCF4663F21E0720711F40C942F
:109D5000995B673F31E0730711F40C949C5B653F9E
:109D6000714011F00C94F4600E9467870E9439835F
:109D70000C94F4606B3893E0790711F40C946A5FEB
:109D80003CF46335734011F40C949F5B0C94F460C5
:109D9000603A23E0720709F401C2673E734011F094
:109DA0000C94F46010924C080E9413768091EF0995
:109DB0009091F009A091F109B091F2098093F30913
:109DC0009093F409A093F509B093F6090E9492408C
:109DD0000C94F46000915E0810915F080E5F1F4FB5
:109DE00080E50E944340882379F00E942F400E9422
:109DF00014AF6B017C01BB24B3946115710581051F
:109E0000910531F4B12C04C0B12CC12CD12C7601B8
:109E100083E50E944340882399F00E942F4020E070
:109E200030E04AE754E40E9475B10E9414AF6B0120
:109E30007C01AA24A394611571058105910509F49B
:109E4000A12C6AE270E0C8010E9423B6009711F0CD
:109E5000FC011082F801CF0121912032E1F3B11011
:109E600007C0A11005C0222319F00E94487204C047
:109E700080E79BE00E94007681E00E9428720E94A9
:109E80003D930E9431A960935A0870935B088093B8
:109E90005C0890935D08C114D104E104F104A9F0B9
:109EA0000E9431A94B015C018C0C9D1CAE1CBF1C97
:109EB0000E9431A9681579058A059B05B8F40E94AE
:109EC0006277811113C00C9438610E9460778823F7
:109ED00011F40C94F4600E94627781110AC00E9410
:109EE000721E80E0C5D90E949C76F5CF80E00E946A
:109EF000287280915F0A882331F081E69BE00E94FE
:109F000000760C94F46081E59BE00E9400760C944E
:109F1000F4609091C00095FFFCCF8093C60031960D
:109F200084918111F6CF8091C00085FFFCCF8AE03B
:109F30008093C6008DE59AE00E94F22FEAE2FBE0F2
:109F40008491882341F09091C00095FFFCCF8093CD
:109F5000C6003196F5CF8091C00085FFFCCF8AE026
:109F60008093C6000C94F4608DE59AE00E9447301F
:109F70000C94F4608DE59AE00E9412310C94F46028
:109F800000915E0810915F080C5F1F4F6AE270E05D
:109F9000C8010E9423B6009711F0FC01108221E055
:109FA00041E0B8018DE59AE00E94EC340C94F46035
:109FB0008DE59AE00E941D310C94F4608091600A56
:109FC000882311F40C94F46083E50E9443408111CE
:109FD0000C9441610C94F4608DE59AE00E94C132CA
:109FE0000C94F46080915E0890915F086AE270E0E2
:109FF00004960E9423B68C010097D9F0209168083E
:10A000003091690840E6429FC001439F900D1124A2
:10A010006EE470E08259974F0E9423B660E270E0D0
:10A020000E9423B6019690935F0880935E08F80122
:10A03000108260915E0870915F086C5F7F4F21E035
:10A0400040E08DE59AE00E94EC340C94F46080913D
:10A05000600A882311F40C94F46060E08DE59AE0C6
:10A060000E947D3480915E0890915F086AE270E002
:10A0700004960E9423B68C010097D9F020916808BD
:10A080003091690840E6429FC001439F900D112422
:10A090006EE470E08259974F0E9423B660E270E050
:10A0A0000E9423B6019690935F0880935E08F801A2
:10A0B000108260915E0870915F086C5F7F4F8DE544
:10A0C0009AE00E9481310C94F46080915F0A8111C2
:10A0D0000E943D9300915E0810915F080C5F1F4F36
:10A0E0006AE270E0C8010E9423B67C0161E270E080
:10A0F000C8010E9423B6009719F08C010F5F1F4F13
:10A10000E114F10411F0F701108280E50E94434050
:10A11000F82E20915E0830915F080217130708F4AB
:10A12000F12C8091600A882311F40C94F46021E0F2
:10A130002F2541E0B8018DE59AE00E94EC3483E5DB
:10A140000E9443408823B9F020915E0830915F0857
:10A150002017310780F40E943840AB01BC014093C6
:10A16000FA0C5093FB0C6093FC0C7093FD0C85E48F
:10A170009CE00E94A9128DE59AE00E941631F11030
:10A180000C94F4600E9431A96093520870935308B4
:10A1900080935408909355080C94F46080915E0865
:10A1A00090915F086AE270E005960E9423B68C01E8
:10A1B0000097D9F0209168083091690840E6429FE5
:10A1C000C001439F900D11246EE470E08259974FB7
:10A1D0000E9423B660E270E00E9423B6019690933D
:10A1E0005F0880935E08F801108260915E087091AC
:10A1F0005F086B5F7F4F8DE59AE00E9416380C94E4
:10A20000F4600E9431A960934E0870934F088093C8
:10A2100050089093510800915208109153082091D2
:10A22000540830915508601B710B820B930B28EE7C
:10A2300033E040E050E00E947EB2CA01B9012CE355
:10A2400030E040E050E00E947EB27F936F933F93F6
:10A250002F938BE19BE09F938F93CE0101969F9369
:10A260008F930E945BB6EFE2FEE084910FB6F89404
:10A27000DEBF0FBECDBF882349F09091C00095FF8F
:10A28000FCCF8093C60031968491F5CFFE013196C4
:10A290008191882339F09091C00095FFFCCF809385
:10A2A000C600F6CF8091C00085FFFCCF8AE0809386
:10A2B000C600CE0101960E9448720C94F46083E5BA
:10A2C0000E944340882311F40C94F4600E942F40B4
:10A2D0000E940FAFF62EE72E862F9E2D8C0180E573
:10A2E0000E944340882331F00F3F110509F010F41C
:10A2F0000C9452610DE010E0EFE8F4E0819191914F
:10A300008017910711F40C94F46034E0E73CF307F4
:10A31000A9F70830110539F48F2D9E2D90932F0A3F
:10A3200080932E0A04C017FF02C00C94F46061E011
:10A33000802F0E9451A86F2D802F0E948AA86F2D18
:10A340007E2D802F0E9447A70C94F46088E690E051
:10A3500043D881110C94F46083E50E944340882324
:10A3600071F000914D080E942F4010E0000F111F66
:10A37000085B174F0E940FAFF801718360830E9442
:10A3800044210C94F4600E94224583E50E944340DE
:10A39000882311F40C94F4600E942F400E940FAFA8
:10A3A00070934708609346080C94F46089E690E047
:10A3B00013D881110C94F460E5E1FBE084918823CB
:10A3C00041F09091C00095FFFCCF8093C60031967C
:10A3D000F5CFE0914D0824E0E29FF0011124E05C0C
:10A3E000F74F408151816281738121E030E08CE937
:10A3F0009DE00E94308BE2E1FBE08491882341F0F4
:10A400009091C00095FFFCCF8093C6003196F5CFA8
:10A41000E0914D08F0E0EE0FFF1FE85BF74F608121
:10A420007181882777FD8095982F0E9442AFAB01FC
:10A43000BC0121E030E08CE99DE00E94308BEEE031
:10A44000FBE08491882341F09091C00095FFFCCF00
:10A450008093C6003196F5CF40913A0850913B0861
:10A4600060913C0870913D0821E030E08CE99DE06E
:10A470000E94308BEBE0FBE08491882341F09091C7
:10A48000C00095FFFCCF8093C6003196F5CF609158
:10A49000460870914708882777FD8095982F0E947D
:10A4A00042AFAB01BC0121E030E08CE99DE00E94AD
:10A4B000308BE8E0FBE08491882341F09091C0006C
:10A4C00095FFFCCF8093C6003196F5CF4AE050E06F
:10A4D00060E070E08CE99DE00E945A8AE6E0FBE0D3
:10A4E0008491882341F09091C00095FFFCCF809328
:10A4F000C6003196F5CF40914008509141086091D7
:10A5000042087091430821E030E08CE99DE00E9410
:10A51000308BE3E0FBE08491882341F09091C00010
:10A5200095FFFCCF8093C6003196F5CF6091480827
:10A5300070914908882777FD8095982F0E9442AF37
:10A54000AB01BC0121E030E08CE99DE00E94308B42
:10A55000EFEFFAE08491882341F09091C00095FFDD
:10A56000FCCF8093C6003196F5CF80914D0890E0E6
:10A570000E943C1E4AE050E0BC018CE99DE00E9434
:10A580005A8AEAEFFAE08491882341F09091C00062
:10A5900095FFFCCF8093C6003196F5CF8FEF9FEFEC
:10A5A0000E943C1E4AE050E0BC018CE99DE00E9404
:10A5B0005A8A8091C00085FFFCCF8AE08093C60054
:10A5C0000C94B0628DE690E00E94EC4981110C94ED
:10A5D000F4608FEE9AE00E94007683E50E9443408B
:10A5E000882391F000914D080E942F4010E0000F49
:10A5F000111F085B174F0E940FAFF8017183608332
:10A6000081E080931C0215C082E50E9443408823AC
:10A6100081F000914D080E942F4010E0000F111FA3
:10A62000085B174F0E940FAFF8017183608310928F
:10A630001C020E9444210E9431A94B015C0100913F
:10A640004D0810E0F801EE0FFF1FE85BF74F608147
:10A650007181882777FD8095982F0E9442AFF8017D
:10A66000EE0FFF1FEE0FFF1FE05CF74F11E02081A0
:10A670003181428153810E94A3B018160CF010E082
:10A6800010934B0810921F0ACC24CA94DC2C76013C
:10A6900048EE442E43E0542E612C712C5AE0352EA6
:10A6A00080911F0A81110C946D62FFEFCF16DF06B7
:10A6B000EF06FF0611F40C945961F7FE02C00C94EA
:10A6C0006D620E9431A96C197D09683B7B4010F4D2
:10A6D0000C9459610C946D6289EC9AE00E940076AA
:10A6E00083E50E944340882361F00E942F400E942E
:10A6F0000FAF709347086093460881E080931C0277
:10A700000FC082E50E944340882351F00E942F40F1
:10A710000E940FAF709347086093460810921C0286
:10A720000E9431A94B015C0110921F0A60914608FA
:10A7300070914708882777FD8095982F0E9442AF37
:10A7400011E020913A0830913B0840913C0850912B
:10A750003D080E94A3B018160CF010E010934B08AF
:10A7600006EC1AE0E2ECEE2EEAE0FE2EFEEBCF2E37
:10A77000FAE0DF2EAAE07A2E80914B08609146081D
:10A7800070914708882309F48BC080911F0A8111BA
:10A7900087C0882777FD8095982F0E9442AF20912F
:10A7A0003A0830913B0840913C0850913D080E9486
:10A7B000A3B018160CF08BC00E9431A96819790952
:10A7C0008A099B09693E73408105910508F460C0C0
:10A7D000E091300A84E0E89FF0011124E05CF74F3B
:10A7E0004081518162817381F8018491E6ECFAE045
:10A7F000882349F09091C00095FFFCCF8093C6005C
:10A8000031968491F5CF22E030E08CE99DE00E9402
:10A81000308BF7018491E2ECFAE0882349F09091C3
:10A82000C00095FFFCCF8093C60031968491F5CF90
:10A830006091300A70E04AE050E08CE99DE00E94AF
:10A840005A8AF6018491EEEBFAE0882349F0909160
:10A85000C00095FFFCCF8093C60031968491F5CF60
:10A8600040913A0850913B0860913C0870913D0836
:10A8700021E030E08CE99DE00E94308B8091C000A7
:10A8800085FFFCCF7092C6000E9431A94B015C018C
:10A890000E94721E80E00E9438490E949C766CCF14
:10A8A000882777FD8095982F0E9442AF20913A0823
:10A8B00030913B0840913C0850913D080E94A0AE69
:10A8C00087FF05C080911C02882309F475CF84EBB3
:10A8D0009AE00E94007680915F0A882321F08EE73B
:10A8E00093E00E9448720E9431A960935A087093C5
:10A8F0005B0880935C0890935D080C94F46083E59A
:10A900000E944340882319F10E942F4020E030E04C
:10A91000A9010E94A0AE87FD0FC00E942F4020E039
:10A9200030E04FE753E40E94A3B0181644F00E94B1
:10A930002F400E940FAF05C060E070E002C06FEFD3
:10A9400070E070932F0A60932E0A0C94F4608FEFDE
:10A9500090E090932F0A80932E0A0C94F46010924A
:10A960002F0A10922E0A0C94F4609B9AA39881E00F
:10A970008093260284EA9AE00E9400760E949C76E8
:10A980000C94F4600E9445210E943D93149A0E9409
:10A99000A79310922F0A10922E0A68EE73E080E0BF
:10A9A00090E00E9460A99B9AA39A1092260286E9E1
:10A9B0009AE00E9400760E949C760C94F4601092BB
:10A9C0005C0A0C94F46081E080935C0A0C94F4605F
:10A9D00083E50E9443408823A1F00E942F4020E09D
:10A9E00030E04AE754E40E9475B10E9414AF6093CE
:10A9F0001D0270931E0280931F02909320020C94FC
:10AA0000F46088E50E94434081110C948E6289E5D0
:10AA10000E94434081110C948E628AE50E9443405B
:10AA200081110C948E6285E40E94434081110C9444
:10AA30008E620E943D93149A0E94A7930C94F46036
:10AA400083E50E944340882311F40C94F4600E9433
:10AA50002F4020E030E04AE754E40E9475B10E94A4
:10AA600014AF6093560870935708809358089093DA
:10AA700059080C94F46027EC34E039AF28AF01EAB0
:10AA800013E161EB862E63E1962E75E6A72E73E146
:10AA9000B72E312CE8ADF9AD8191F9AFE8AF0E9446
:10AAA0004340882309F45BC0F3E03F1251C00E9489
:10AAB0002F406B017C0120E030E040EA51E40E942D
:10AAC000A0AE87FF3FC0A7019601F80160817181A8
:10AAD000828193810E94A7AE2B013C019B01AC01B6
:10AAE0006091791370917A1380917B1390917C130C
:10AAF0000E9475B16093791370937A1380937B13DE
:10AB000090937C13A3019201F40160817181828191
:10AB100093810E9475B1F401608371838283938372
:10AB2000F50160817181828193810E9440AFA30110
:10AB300092010E9475B10E9414AFF5016083718388
:10AB400082839383F801C082D182E282F38207C0BC
:10AB50000E942F40F8016083718382839383339432
:10AB60000C5F1F4FF4E08F0E911C24E0A20EB11C6D
:10AB700034E033128FCF0C94F4609091C00095FFB5
:10AB8000FCCF8093C600319684918111F6CF0C944E
:10AB9000F46000915E0810915F080B5F1F4F6AE23E
:10ABA00070E0C8010E9423B6009711F0FC011082EA
:10ABB000C8010E9448720C94F460EBEBF9E08491B8
:10ABC000882341F09091C00095FFFCCF8093C60090
:10ABD0003196F5CF4091440A5091450A6091460A5A
:10ABE0007091470A22E030E08CE99DE00E94308BB2
:10ABF000E7EBF9E08491882341F09091C00095FF44
:10AC0000FCCF8093C6003196F5CF4091480A509111
:10AC1000490A60914A0A70914B0A22E030E08CE9BF
:10AC20009DE00E94308BE3EBF9E08491882341F0B2
:10AC30009091C00095FFFCCF8093C6003196F5CF70
:10AC400040914C0A50914D0A60914E0A70914F0A02
:10AC500022E030E08CE99DE00E94308BEFEAF9E0E1
:10AC60008491882341F09091C00095FFFCCF8093A0
:10AC7000C6003196F5CF4091500A5091510A60912B
:10AC8000520A7091530A22E030E08CE99DE00E9464
:10AC9000308BE4EAF9E08491882341F09091C00080
:10ACA00095FFFCCF8093C6003196F5CF0E94999313
:10ACB0000E9442AF2091A1133091A2134091A3139F
:10ACC0005091A4130E94A7AEAB01BC0122E030E07A
:10ACD0008CE99DE00E94308BE0EAF9E084918823C2
:10ACE00041F09091C00095FFFCCF8093C600319653
:10ACF000F5CF81E00E9499930E9442AF2091A51365
:10AD00003091A6134091A7135091A8130E94A7AEAB
:10AD1000AB01BC0122E030E08CE99DE00E94308B69
:10AD2000ECE9F9E08491882341F09091C00095FF0F
:10AD3000FCCF8093C6003196F5CF82E00E949993B4
:10AD40000E9442AF2091A9133091AA134091AB13F6
:10AD50005091AC130E94A7AEAB01BC0122E030E0E1
:10AD60008CE99DE00E94308B8091C00085FFFCCF74
:10AD70008AE08093C6000C94F46080E00E94F18B1E
:10AD80000C94F46081E00E94F18B0C94F46090913B
:10AD9000C00095FFFCCF8093C60081918111F7CF51
:10ADA0008091C00085FFFCCF8AE08093C600E4E973
:10ADB000F9E08491882341F09091C00095FFFCCF89
:10ADC0008093C6003196F5CF1E9B03C0EBE0F4E004
:10ADD00009C0E5E1F4E006C09091C00095FFFCCF0A
:10ADE0008093C60081918111F7CF8091C00085FFCB
:10ADF000FCCF8AE08093C600ECE8F9E084918823D8
:10AE000041F09091C00095FFFCCF8093C600319631
:10AE1000F5CF029903C0EBE0F4E009C0E5E1F4E00E
:10AE200006C09091C00095FFFCCF8093C600819131
:10AE30008111F7CF8091C00085FFFCCF8AE080931D
:10AE4000C600E4E8F9E08491882341F09091C000C5
:10AE500095FFFCCF8093C6003196F5CF1D9B03C0B4
:10AE6000EBE0F4E009C0E5E1F4E006C09091C00039
:10AE700095FFFCCF8093C60081918111F7CF80911F
:10AE8000C00085FFFCCF8AE08093C600ECE7F9E0C4
:10AE90008491882341F09091C00095FFFCCF80936E
:10AEA000C6003196F5CF019903C0EBE0F4E009C08C
:10AEB000E5E1F4E006C09091C00095FFFCCF8093DF
:10AEC000C60081918111F7CF8091C00085FFFCCF32
:10AED0008AE08093C600E4E7F9E08491882341F09A
:10AEE0009091C00095FFFCCF8093C6003196F5CFBE
:10AEF0001C9B03C0EBE0F4E009C0E5E1F4E006C010
:10AF00009091C00095FFFCCF8093C6008191811184
:10AF1000F7CF8091C00085FFFCCF8AE08093C60008
:10AF2000ECE6F9E08491882341F09091C00095FF10
:10AF3000FCCF8093C6003196F5CF379903C0EBE084
:10AF4000F4E009C0E5E1F4E006C09091C00095FF8F
:10AF5000FCCF8093C60081918111F7CF8091C00012
:10AF600085FFFCCF8AE08093C6000C94F46080914A
:10AF7000300A80934D0884E50E944340882319F1EC
:10AF80000E942F400E9414AF60934D086623D9F0B1
:10AF9000EFE2FEE08491882341F09091C00095FF9C
:10AFA000FCCF8093C6003196F5CFE0E4F4E08191C8
:10AFB000882311F40C94F4609091C00095FFFCCFAD
:10AFC0008093C600F4CF84E40E944340882311F4A8
:10AFD0000C94F4600E942F4020E030E0A9010E9410
:10AFE000A0AE811103C01092540A32C000914D08E6
:10AFF00010E00E942F40F801EE0FFF1FEE0FFF1F21
:10B00000ED5AFD4F6083718382839383E0905302F6
:10B01000F0905402009155021091560220E030E069
:10B02000A901B701C8010E94A0AE811104C0E12CA2
:10B03000F12C00E410E4C701D801809353029093EF
:10B040005402A0935502B093560281E08093540AB3
:10B050000E94A74A0C94F46007EC14E041E9E42E46
:10B0600043E1F42EF80181918F010E94434088232F
:10B0700049F00E942F400E9414AFF7016083718352
:10B0800082839383F4E0EF0EF11C24E00B3C120763
:10B0900049F70E9410A50C94F46007EC14E031EB22
:10B0A000E32E33E1F32EF80181918F010E9443409A
:10B0B000882339F00E942F40F701608371838283D7
:10B0C0009383F4E0EF0EF11C24E00B3C120759F7D8
:10B0D0000C94F46083E50E944340882351F00E9461
:10B0E0002F406093891370938A1380938B139093EE
:10B0F0008C1384E50E944340882311F40C94F4607F
:10B100000E942F406093851370938613809387135A
:10B11000909388130C94F46083E50E944340882345
:10B1200051F00E942F4060938D1370938E13809383
:10B130008F139093901384E50E944340882351F02D
:10B140000E942F406093751370937613809377134A
:10B150009093781382E40E944340882361F00E9418
:10B160002F400E9414AF6093C1137093C213809359
:10B17000C3139093C41388E50E944340882351F081
:10B180000E942F40609381137093821380938313E6
:10B19000909384138AE50E944340882351F00E94D3
:10B1A0002F4060937D1370937E1380937F13909351
:10B1B000801385E40E944340882311F40C94F460CA
:10B1C0000E942F406093791370937A1380937B13BE
:10B1D00090937C130C94F46007EC14E028E3E22EC7
:10B1E0002AE0F22EF80181918F010E9443408823CA
:10B1F00039F00E942F40F70160837183828393832B
:10B20000F4E0EF0EF11C24E00A3C120709F4ECC74D
:10B21000E9CF83E50E944340882351F00E942F40EC
:10B220006093330270933402809335029093360218
:10B2300086E40E944340882381F00E942F4020E052
:10B2400030E040E752E40E94A7AE60932B02709377
:10B250002C0280932D0290932E028AE50E94434097
:10B26000882309F4C1C70E942F406093280A709375
:10B27000290A80932A0A90932B0AB6C783E50E9475
:10B280004340882351F00E942F406093240A70931A
:10B29000250A8093260A9093270A86E40E94434059
:10B2A000882309F4A1C70E942F4020E030E040E746
:10B2B00052E40E94A7AE6093270270932802809305
:10B2C000290290932A0290C783E50E944340882375
:10B2D00009F48AC70E942F400E940FAF61157105C3
:10B2E00049F06130710559F481E080932D0A109284
:10B2F0002C0A7AC710922D0A10922C0A75C7EFE219
:10B30000FEE08491882341F09091C00095FFFCCF2E
:10B310008093C6003196F5CFE9E5F9E08491882362
:10B3200041F09091C00095FFFCCF8093C60031960C
:10B33000F5CF809168089091690820E6289FF00178
:10B34000299FF00D1124E259F74F8191882339F09C
:10B350009091C00095FFFCCF8093C600F6CFE7E543
:10B36000F9E08491882341F09091C00095FFFCCFD3
:10B370008093C6003196F5CF8091C00085FFFCCF49
:10B380008AE08093C60030C783E50E94434088234B
:10B3900009F42AC70E942F400E940FAF70935E02EB
:10B3A00060935D0221C783E50E944340882309F42E
:10B3B0001BC70E942F400E940FAF6B017C0184E5E8
:10B3C0000E944340882381F08DED90E00E94EC497B
:10B3D00081110AC7E0914D08F0E0EE0FFF1FE75A18
:10B3E000FD4FD182C08200C7D0925C02C0925B0246
:10B3F000FBC680E50E944340882309F4F5C60E94FD
:10B400002F400E940FAFD62E062F172F83E50E94E4
:10B410004340882331F00E942F400E940FAF7B01F0
:10B4200003C0EE24EA94FE2CC7010196039708F0AE
:10B43000DBC6EFE8F4E0819191918017910709F460
:10B44000D3C634E0E73CF307B1F717FDCDC60E9441
:10B450003D93CD2C60E08D2D0E9451A88FEFE81612
:10B46000F80631F0EA94EF2871F000E010E00DC02A
:10B470008D2D0E94BFA831E020E0892B09F030E03B
:10B48000032F122F02C001E010E08C2D0E94BFA8F4
:10B490008017910709F4A8C60E94721E80E00E94DE
:10B4A00038490E949C76F1CF83E50E94434088236F
:10B4B00031F00E942F400E940FAF8B0102C00EE6B8
:10B4C00010E080E50E944340882331F00E942F4025
:10B4D0000E940FAFCB0102C088EE93E06C01EE2416
:10B4E000D7FCE094FE2C101611067CF420E030E02E
:10B4F000A901B80184E50E94FDA9C701B6010E9417
:10B5000060A984E50E940EAD6FC6C701B6010E9416
:10B5100060A96AC680E50E944340882351F00E94DA
:10B520002F40609318027093190280931A0290932F
:10B530001B0289E40E944340882361F00E942F404F
:10B540000E94B7276093140270931502809316022D
:10B550009093170284E40E944340882361F00E9484
:10B560002F400E94C32760931002709311028093B2
:10B5700012029093130283E40E944340882351F007
:10B580000E942F4060930C0270930D0280930E0274
:10B5900090930F020E94251EE7E5F4E08191882335
:10B5A00039F09091C00095FFFCCF8093C600F6CF94
:10B5B000EAE5F4E08191882339F09091C00095FF8D
:10B5C000FCCF8093C600F6CF40911802509119022B
:10B5D00060911A0270911B0222E030E08CE99DE03C
:10B5E0000E94308BEEE5F4E08191882339F0909150
:10B5F000C00095FFFCCF8093C600F6CF6091140287
:10B600007091150280911602909117020E94BD2739
:10B61000AB01BC0122E030E08CE99DE00E94308B60
:10B62000E2E6F4E08191882339F09091C00095FF23
:10B63000FCCF8093C600F6CF60911002709111028A
:10B6400080911202909113020E94C927AB01BC01A4
:10B6500022E030E08CE99DE00E94308BE6E6F4E0E9
:10B660008191882339F09091C00095FFFCCF8093A1
:10B67000C600F6CF40910C0250910D0260910E026F
:10B6800070910F0222E030E08CE99DE00E94308B47
:10B690008091C00085FFFCCF8AE08093C600A4C5DE
:10B6A00083E50E944340882319F00E942F4003C085
:10B6B00060E070E0CB010E9407A596C585E40E947A
:10B6C0004340882341F00E942F400E940FAF8B011E
:10B6D00077FF03C009C000E010E0C12CD12CB6E117
:10B6E000EB2EB3E4FB2E06C0C12CD12CACE8EA2E25
:10B6F000A2E4FA2E83E50E944340882321F00E94B1
:10B700002F406B017C0183E40E944340882331F089
:10B710000E942F400E940FAF9B0102C025E030E045
:10B72000A801C701B6010E9458215EC50E943D9341
:10B730005BC50E94678758C50E94398355C58AE555
:10B740000E944340882309F497C00E942F406B0158
:10B750007C0120E030E040E751EC0E94A3B087FD7F
:10B760003FC020E030E040EA50ECC701B6010E9443
:10B77000A0AE1816ACF1F7FAF094F7F8F094C09276
:10B78000310AD092320AE092330AF092340AEFE2A0
:10B79000FEE08491882341F09091C00095FFFCCF9A
:10B7A0008093C6003196F5CFEBE4F9E084918823CD
:10B7B00041F09091C00095FFFCCF8093C600319678
:10B7C000F5CF8091C00085FFFCCF8AE08093C60052
:10B7D0008091C00085FFFCCF8AE08093C60004C53D
:10B7E000EFE2FEE08491882341F09091C00095FF44
:10B7F000FCCF8093C6003196F5CFE2E4F9E0849166
:10B80000882341F09091C00095FFFCCF8093C60043
:10B810003196F5CFEAE3F9E08491882341F09091E5
:10B82000C00095FFFCCF8093C6003196F5CF4AE06B
:10B8300050E061EF7FEF8CE99DE00E945A8AE2E3DD
:10B84000F9E08491882341F09091C00095FFFCCFEE
:10B850008093C6003196F5CF4AE050E06BEF7FEF62
:10B860008CE99DE00E945A8A8091C00085FFFCCF40
:10B870008AE08093C600B8C4EFE2FEE0849188239A
:10B8800041F09091C00095FFFCCF8093C6003196A7
:10B89000F5CFE6E2F9E08491882341F09091C00071
:10B8A00095FFFCCF8093C6003196F5CF8091C00004
:10B8B00085FFFCCF8AE08093C6004091310A509109
:10B8C000320A6091330A7091340A705822E030E0F5
:10B8D0008CE99DE00E94308B8091C00085FFFCCFF9
:10B8E0008AE08093C60080C480915D0290915E02E0
:10B8F0009093580280935702C090440AD090450A12
:10B90000E090460AF090470ACF8ED8A2E9A2FAA2A8
:10B910000091480A1091490A20914A0A30914B0A35
:10B920000BA31CA32DA33EA340914C0A50914D0A9A
:10B9300060914E0A70914F0A4FA358A769A77AA742
:10B940008091500A9091510AA091520AB091530AE5
:10B950008BA79CA7ADA7BEA7C982DA82EB82FC8227
:10B960000D831E832F83388749875A876B877C878F
:10B970008D879E87AF87B88B85E40E9443408823DC
:10B9800059F00E942F409B01AC016BA57CA58DA5B1
:10B990009EA50E94C7AD0AC020E030E040E050E420
:10B9A0006BA57CA58DA59EA50E94C6AD6BA77CA7A7
:10B9B0008DA79EA7E0E3CE2EEAE0DE2EE12CF12C4F
:10B9C00008EC13E49E01255D3F4FAE01495D5F4FDA
:10B9D000BE016D5D7F4FCE014F960E94779A8AE53A
:10B9E0000E944340882349F00E942F409B01AC01F4
:10B9F0006FA178A589A59AA51EC020E030E040E09F
:10BA000050E46FA178A589A59AA50E94C7AD6B01E6
:10BA10007C016FA378A789A79AA720E030E040E2D5
:10BA200051E40E94A0AE87FF0CC020E030E040E26D
:10BA300051E4C701B6010E94C7AD6FA378A789A7DB
:10BA40009AA760E3C62E6AE0D62EE12CF12C06E917
:10BA500013E49E01255D3F4FAE01495D5F4FBE017E
:10BA60006D5D7F4FCE014F960E94779A88E50E94C8
:10BA70004340882379F00E942F409B01AC016F8DD9
:10BA800078A189A19AA10E94C7AD6F8F78A389A3DD
:10BA90009AA308C080E090E0A3E5B3E48F8F98A359
:10BAA000A9A3BAA389E50E944340882339F00E94E4
:10BAB0002F406BA37CA38DA39EA304C01BA21CA23A
:10BAC0001DA21EA240E3C42E4AE0D42EE12CF12C8C
:10BAD0000CE812E49E01255D3F4FAE01495D5F4FCA
:10BAE000BE016D5D7F4FCE014F960E94779A8CE428
:10BAF0000E944340882359F00E942F409B01AC01D3
:10BB00006BA57CA58DA59EA50E94C7AD0AC020E0AF
:10BB100030E040EA52E46BA57CA58DA59EA50E946D
:10BB2000C6AD6BA77CA78DA79EA720E3C22E2AE0F7
:10BB3000D22EE12CF12C00EA11E49E01255D3F4F4D
:10BB4000AE01495D5F4FBE016D5D7F4FCE014F96E7
:10BB50000E94779A0E943D93149A64E670E080E018
:10BB600090E00E9460A90E94827100E010E0F12C38
:10BB70000E94627781112AC0F3940E94721E81E0B4
:10BB80000E943849F110F4CF043FE1E01E0711F4A0
:10BB900000E010E0809101018460809301010115B3
:10BBA000110531F49FB7F89480910201846008C0B8
:10BBB0000431110541F49FB7F894809102018B7F05
:10BBC000809302019FBF0F5F1F4FD2CF9FB7F894A2
:10BBD000809102018B7F809302019FBF20E030E0C3
:10BBE0004CE852E46BA57CA58DA59EA50E94C7AD2F
:10BBF0006BA77CA78DA79EA710E3C12E1AE0D12EBC
:10BC0000E12CF12C00EA11E49E01255D3F4FAE01CD
:10BC1000495D5F4FBE016D5D7F4FCE014F960E9423
:10BC2000779A20E030E048E452E46BA57CA58DA52E
:10BC30009EA50E94C7AD6BA77CA78DA79EA7E12CF0
:10BC4000F12C00E010E49E01255D3F4FAE01495DFF
:10BC50005F4FBE016D5D7F4FCE014F960E94779A78
:10BC60001092560A1092550A0E94E8718091550A66
:10BC70009091560A019709F47CC01092560A1092CE
:10BC8000550A0E9468778091550A9091560A823031
:10BC9000910549F1039709F069C020E030E048E4DC
:10BCA00052E46BA57CA58DA59EA50E94C7AD6BA790
:10BCB0007CA78DA79EA770E3C72E7AE0D72EE12C34
:10BCC000F12C00E010E49E01255D3F4FAE01495D7F
:10BCD0005F4FBE016D5D7F4FCE014F960E94779AF8
:10BCE0000E94A871C3CF20E030E04CE852E46BA57D
:10BCF0007CA58DA59EA50E94C7AD6BA77CA78DA72F
:10BD00009EA7F0E3CF2EFAE0DF2EE12CF12C00EA23
:10BD100011E49E01255D3F4FAE01495D5F4FBE01BD
:10BD20006D5D7F4FCE014F960E94779A20E030E004
:10BD300048E452E46BA57CA58DA59EA50E94C7ADE5
:10BD40006BA77CA78DA79EA7E12CF12C00E010E447
:10BD50009E01255D3F4FAE01495D5F4FBE016D5DA8
:10BD60007F4FCE014F960E94779A7ECF0E949B71A3
:10BD70007DCF20E030E040EA50E46BA57CA58DA5A6
:10BD80009EA50E94C7AD6BA77CA78DA79EA790E339
:10BD9000C92E9AE0D92EE12CF12C00E010E49E018E
:10BDA000255D3F4FAE01495D5F4FBE016D5D7F4F29
:10BDB000CE014F960E94779AA80197016BA57CA5AA
:10BDC0008DA59EA50E94C6AD6BA77CA78DA79EA73B
:10BDD000E12CF12C08EC13E49E01255D3F4FAE01F0
:10BDE000495D5F4FBE016D5D7F4FCE014F960E9452
:10BDF000779AE12CF12C0CE812E49E01255D3F4F6F
:10BE0000AE01495D5F4FBE016D5D7F4FCE014F9624
:10BE10000E94779A9E01255D3F4FAE01495D5F4FBD
:10BE2000BE016B5F7F4FCE0101960E94779AE12C95
:10BE3000F12C08E413E49E01255D3F4FAE01475FFE
:10BE40005F4FBE016B5F7F4FCE0101960E94779AD4
:10BE500020E030E040E050E46BA57CA58DA59EA5D8
:10BE60000E94C7AD6BA77CA78DA79EA7E12CF12CE4
:10BE700000EA10E49E01255D3F4FAE01475F5F4F32
:10BE8000BE016B5F7F4FCE0101960E94779ACE0173
:10BE90000D960E94E3A480915702909158028093DE
:10BEA0005D0290935E029F938F938DE199E09F9343
:10BEB0008F938E01015D1F4F1F930F930E945BB6FE
:10BEC000C8010E94C03D0F900F900F900F900F90EF
:10BED0000F908AC188E50E944340882339F00E9470
:10BEE0002F400E940FAF80E00E9445948AE50E9497
:10BEF0004340882339F00E942F400E940FAF81E019
:10BF00000E94459485E40E944340882309F46CC153
:10BF10000E942F400E940FAF82E00E94459464C1AE
:10BF200083E50E944340811104C007EC14E0F12C2A
:10BF300010C010E00E942F400E9414AF812F0E9479
:10BF4000E4941F5F1530B1F7F0CFF394F4E0FF16DF
:10BF500079F0F80181918F010E9443408823A9F371
:10BF60000E942F400E9414AF8F2D0E94E494EDCFC9
:10BF700082E40E944340882339F00E942F400E94AF
:10BF800014AF84E00E94E4940E94AA952DC183E539
:10BF90000E944340882309F453C00E942F400E940E
:10BFA0000FAF6130710541F06230710509F048C092
:10BFB00007EC14E0F12C25C007EC14E0F12CF8019B
:10BFC00081918F010E944340882341F00E942F40BD
:10BFD0000E940FAF4FEF8F2D0E94A694F394F4E0D0
:10BFE000FF12EDCF82E40E944340882349F10E9472
:10BFF0002F400E940FAF4FEF20C0F394F4E0FF16E4
:10C0000089F0F80181918F010E9443408823A9F3B0
:10C010000E942F400E940FAF462F6FEF8F2D0E947E
:10C02000A694EBCF82E40E944340882349F00E940B
:10C030002F400E940FAF462F6FEF84E00E94A6941E
:10C040000E94AA95D1C084E50E944340882309F448
:10C0500087C00E942F400E9414AF60934D08662352
:10C06000A9F1EFE2FEE08491882341F09091C000B5
:10C0700095FFFCCF8093C6003196F5CFEAE6F4E059
:10C080008191882339F09091C00095FFFCCF809377
:10C09000C600F6CF40E050E060914D088CE99DE08D
:10C0A0000E94918AECE6F4E08191882339F0909126
:10C0B000C00095FFFCCF8093C600F6CF8091C000F2
:10C0C00085FFFCCF8AE08093C6008EC086E40E9484
:10C0D00043408823D9F00E942F406B017C0160937C
:10C0E000FF097093000A8093010A9093020A20E0EE
:10C0F00030E0A9010E94A3B0181644F4C0922102B6
:10C10000D0922202E0922302F0922402EFE2FEE0BB
:10C110008491882341F09091C00095FFFCCF8093DB
:10C12000C6003196F5CFEDE7F4E08191882339F030
:10C130009091C00095FFFCCF8093C600F6CF609130
:10C14000300A70E04AE050E08CE99DE00E945A8A93
:10C150008091C00085FFFCCF8AE08093C60044C078
:10C16000EFE2FEE08491882341F09091C00095FFBA
:10C17000FCCF8093C6003196F5CFEAE0F9E08491D8
:10C18000882341F09091C00095FFFCCF8093C600BA
:10C190003196F5CF809168089091690820E6289F34
:10C1A000F001299FF00D1124E259F74F8191882366
:10C1B00039F09091C00095FFFCCF8093C600F6CF78
:10C1C000E8E0F9E08491882341F09091C00095FF68
:10C1D000FCCF8093C6003196F5CF8091C00085FFDB
:10C1E000FCCF8AE08093C6000E946A40B9C1C0902B
:10C1F0001B0AD0901C0AE0901D0AF0901E0A2091A4
:10C20000500A3091510A4091520A5091530AC70185
:10C21000B6010E94C6AD2DEC3CEC4CEC5DE30E94F7
:10C22000A3B0181614F00C94684BC092500AD09228
:10C23000510AE092520AF092530A80E59AE00E9475
:10C24000E3A460E080E00E94C2428AC180E090E006
:10C250000E942E3C0C94654C81E090E00E942E3CA4
:10C260000C94704C82E090E00E942E3C0C94B94CEF
:10C270000E94721E80E00E9438490E949C760C94B5
:10C28000584F0E943840AB01BC014093FA0C5093C8
:10C29000FB0C6093FC0C7093FD0C85E49CE00E9409
:10C2A000A912A2CF0E942F400E940FAF8B010C94C5
:10C2B0007C510E9431A9681979098A099B09693E54
:10C2C00073408105910508F479C0ECEEFAE08491A1
:10C2D000882341F09091C00095FFFCCF8093C60069
:10C2E0003196F5CFE0914D0824E0E29FF001112452
:10C2F000E05CF74F408151816281738121E030E041
:10C300008CE99DE00E94308BE8EEFAE0849188236E
:10C3100041F09091C00095FFFCCF8093C60031960C
:10C32000F5CF60914D0870E04AE050E08CE99DE067
:10C330000E945A8AE4EEFAE08491882341F09091B9
:10C34000C00095FFFCCF8093C6003196F5CFF7FE75
:10C3500003C0E6E7F5E025C00E9431A98B019C01EE
:10C36000C701B6016854744F8F4F9F4F601B710B0C
:10C37000820B930BA30192010E947EB2BA01A90124
:10C380002AE030E08CE99DE00E94868A8091C0001E
:10C3900085FFFCCF0DC09091C00095FFFCCF80932E
:10C3A000C60081918111F7CF8091C00085FFFCCF3D
:10C3B0003092C6000E9431A94B015C010E94721E9E
:10C3C00080E00E9438490E949C76FFEFCF16DF067E
:10C3D000EF06FF0609F046C080914B08E0914D083A
:10C3E000F0E08F01000F111F000F111F005C174FAD
:10C3F000EE0FFF1FE85BF74F608171818823C9F062
:10C40000882777FD8095982F0E9442AF20E030E08A
:10C4100040E85FE30E94C6AD9B01AC01F80160817A
:10C420007181828193810E94A3B087FF50C00C94D8
:10C430005053882777FD8095982F0E9442AF20E0C7
:10C4400030E040E85FE30E94C7AD9B01AC01F8011A
:10C4500060817181828193810E94A0AE1816BCF523
:10C460000C945053F7FE02C00C945053E0914D08C9
:10C47000F0E08F01000F111F000F111F005C174F1C
:10C48000EE0FFF1FE85BF74F60817181882777FD12
:10C490008095982F0E9442AF9B01AC01F80160810A
:10C4A0007181828193810E94C6AD0E940FAF97FF78
:10C4B00007C090958095709561957F4F8F4F9F4FE6
:10C4C000663071058105910514F40C9450530E9457
:10C4D00031A96B017C010C94505386ED9AE00E94C7
:10C4E000007680915F0A882321F08EE793E00E9416
:10C4F00048720E9431A96093520870935308809348
:10C500005408909355080E9431A960935A0870937B
:10C510005B0880935C0890935D0866CE0E943D9313
:10C5200088E50E944340882319F0179A1092350A33
:10C5300089E50E944340882319F0169A1092360A22
:10C540008AE50E944340882319F0159A1092370A11
:10C5500085E40E944340882309F446CE149A44CED1
:10C56000E9960FB6F894DEBF0FBECDBFDF91CF9135
:10C570001F910F91FF90EF90DF90CF90BF90AF9001
:10C580009F908F907F906F905F904F903F90089515
:10C59000CF93DF938091640890916508039714F41A
:10C5A0000E94694560E08DE59AE00E9487338091A2
:10C5B000640890916508892B09F464C080915D0A34
:10C5C0008823E1F0809168089091690820E6289F0F
:10C5D000E001299FD00D1124C259D74F61EF7CE0B3
:10C5E000CE010E94CEB5892BF1F4BE018DE59AE013
:10C5F0000E94163380915E0A882319F00E94B94A7E
:10C600002BC0EEEEFCE08491882341F09091C000B5
:10C6100095FFFCCF8093C6003196F5CF8091C00086
:10C6200085FFFCCF16C060E08DE59AE00E947D3466
:10C63000ECEDFCE08491882341F09091C00095FFDF
:10C64000FCCF8093C6003196F5CF8091C00085FF66
:10C65000FCCF8AE08093C6008091640890916508C1
:10C660000197909365088093640880916808909181
:10C670006908019664E070E00E946BB290936908CB
:10C68000809368080E94721E80E00E9438490E94D0
:10C690004F8BDF91CF910C949C768F929F92AF92AB
:10C6A000BF92CF92DF92EF92FF920F931F93CF939F
:10C6B000DF938C018C519E4F0E94B72D680189E851
:10C6C000C80ED11C21F1780181E4E81A8EEFF80A36
:10C6D000E70157018FE1A81AB1087AEB872E75E0C0
:10C6E000972ECC15DD0599F0FE01EE19FF09EA0D34
:10C6F000FB1D91828082FE0178978081811102C0AA
:10C700006F97EFCFCE014B970E948C13F9CFC801E2
:10C7100086599F4F0E94B72DC801875B9F4FDF91BD
:10C72000CF911F910F91FF90EF90DF90CF90BF902E
:10C73000AF909F908F900C94B72D8DE59AE00C945C
:10C74000C32D8DE59AE0A9CFFB0160917002709135
:10C75000710270932C0D60932B0D6091350D7091CB
:10C76000360D70932A0D6093290D62E060936F027D
:10C7700064EC7EE770937102609370029093280DD1
:10C780008093270DF093260DE093250D662757FD26
:10C790006095762F4093210D5093220D6093230DC9
:10C7A0007093240DC901AA2797FDA095BA2F841B69
:10C7B000950BA60BB70B80931D0D90931E0DA093A8
:10C7C0001F0DB093200D80819181AA2797FDA09520
:10C7D000BA2F841B950BA60BB70B8093350D909346
:10C7E000360DA093370DB093380D08950F931F9316
:10C7F000CF93DF93EB01142F022F482F60E080E4EA
:10C800009DE00E947E28612F80E49DE00E94BFADE4
:10C8100011E1FE016491662311F0111117C011237B
:10C8200039F060E280E49DE00E94BFAD1150F7CF87
:10C83000602F80E49DE00E94BFAD60E280E49DE057
:10C84000DF91CF911F910F910C94BFAD80E49DE0DB
:10C850000E94BFAD21961150DCCFEF92FF920F9353
:10C860001F93CF93DF93EB01E42E8901F90101902F
:10C870000020E9F7F22EFE1A92E1F90E482F60E04F
:10C8800080E49DE00E947E286E2D80E49DE00E9461
:10C89000BFADFE016491662311F0F11019C06AE387
:10C8A00080E49DE00E94BFADFF2039F060E280E4AB
:10C8B0009DE00E94BFADFA94F7CFB80180E49DE0FF
:10C8C000DF91CF911F910F91FF90EF900C94BEAD2F
:10C8D00080E49DE00E94BFAD2196FA94DACF1092D9
:10C8E000990D8DE59AE00E94273910923E0D08952A
:10C8F0008DE59AE00C9416318DE59AE00C941D318B
:10C90000CF93DF93CDB7DEB7C054D1090FB6F894FB
:10C91000DEBF0FBECDBF88E0EFEAF2E0DE01D996C0
:10C9200001900D928A95E1F788E0E7EBF2E0DE01F5
:10C93000D19601900D928A95E1F788E0EFEBF2E055
:10C94000DE01999601900D928A95E1F788E0E7EC77
:10C95000F2E0DE01919601900D928A95E1F788E070
:10C96000EFECF2E0DE01599601900D928A95E1F725
:10C9700088E0E7EDF2E0DE01519601900D928A9594
:10C98000E1F788E0EFEDF2E0DE01199601900D92FB
:10C990008A95E1F788E0E7EEF2E0DE01119601907A
:10C9A0000D928A95E1F7AE01475C5F4F60E080E44D
:10C9B0009DE00E94FC29AE014F5C5F4F61E080E486
:10C9C0009DE00E94FC29AE01475D5F4F62E080E47C
:10C9D0009DE00E94FC29AE014F5D5F4F63E080E463
:10C9E0009DE00E94FC29AE01475E5F4F64E080E459
:10C9F0009DE00E94FC29AE014F5E5F4F65E080E440
:10CA00009DE00E94FC29AE01475F5F4F66E080E435
:10CA10009DE00E94FC29AE014F5F5F4F67E080E41C
:10CA20009DE00E94FC29C05CDF4F0FB6F894DEBF8A
:10CA30000FBECDBFDF91CF910895CF9382E0809359
:10CA40006F020E9431A96C507E4F8F4F9F4F6093B1
:10CA50003A0D70933B0D80933C0D90933D0D80916A
:10CA60000101846080930101CAE09FB7F89480912E
:10CA700002018460809302019FBF84E690E00E94DF
:10CA800084A99FB7F894809102018B7F8093020163
:10CA90009FBF84E690E00E9484A9C15031F7CF91F6
:10CAA0000895E0917002F0917102E817F90771F0B2
:10CAB00090937102809370024093350D5093360D20
:10CAC0006093370D7093380D2111B7CF089521E091
:10CAD00040E050E0BA01E5CF21E040E050E0BA018B
:10CAE000E0CF8F929F92AF92BF92CF92DF92EF9260
:10CAF000FF920F931F93CF93DF938091350D909109
:10CB0000360DA091370DB091380D81309048A105B8
:10CB1000B10540F01092350D1092360D1092370D80
:10CB20001092380D6091350D7091360D8091370D52
:10CB30009091380D25E030E040E050E00E947EB258
:10CB400080913E0D90E0A0E0B0E0281739074A0739
:10CB50005B0710F420933E0DD0913E0D10913F0DD8
:10CB600012FB112710F9C0E085E0C82ED12CE12C72
:10CB7000F12C9DE1892E912CA12CB12C01E060912A
:10CB8000350D7091360D8091370D9091380DD11182
:10CB900031C020916F02222369F023E065307105D6
:10CBA0008105910510F443E001C040E266E870E1C0
:10CBB0008C2F1CDE112309F400C18091350D90915A
:10CBC000360DA091370DB091380D0597A105B1052F
:10CBD00008F0F3C032DF8CE692E7DF91CF911F912E
:10CBE0000F91FF90EF90DF90CF90BF90AF909F900C
:10CBF0008F906DCFD13061F520916F02222391F09B
:10CC0000A70196010E947EB22130310541055105F0
:10CC100019F423E043E002C023E040E265E770E15D
:10CC20008C2FE4DD112309F4C8C06091350D70919B
:10CC3000360D8091370D9091380DA70196010E9415
:10CC40007EB2213031054105510509F0B6C0C2CF91
:10CC5000D23061F520916F02222391F0A701960155
:10CC60000E947EB2223031054105510519F423E0BE
:10CC700043E002C023E040E269E670E18C2FB6DDBC
:10CC8000112309F49AC06091350D7091360D809191
:10CC9000370D9091380DA70196010E947EB2223087
:10CCA00031054105510509F088C094CFD33061F5B5
:10CCB00020916F02222391F0A70196010E947EB27B
:10CCC000233031054105510519F423E043E002C04A
:10CCD00023E040E267E570E18C2F88DD112309F441
:10CCE0006CC06091350D7091360D8091370D90912B
:10CCF000380DA70196010E947EB22330310541050F
:10CD0000510509F05AC066CFD43059F520916F0211
:10CD1000222391F0A70196010E947EB224303105B2
:10CD20004105510519F423E043E002C023E040E24D
:10CD300065E470E18C2F5ADD112309F43EC0609147
:10CD4000350D7091360D8091370D9091380DA701FA
:10CD500096010E947EB2243031054105510569F5E6
:10CD600039CFD53051F520916F02222391F0A701E0
:10CD700096010E947EB2253031054105510519F416
:10CD800023E043E002C023E040E269E370E18C2F3E
:10CD90002DDD112391F06091350D7091360D80914C
:10CDA000370D9091380DA70196010E947EB2253073
:10CDB00031054105510509F40DCF8091350D909154
:10CDC000360DA091370DB091380D4E97A105B105E4
:10CDD00040F08092350D9092360DA092370DB092B2
:10CDE000380D6091350D7091360D8091370D909111
:10CDF000380DA70196010E947EB280913E0D90E011
:10CE00000396422F50E0841795074CF48DEF820F64
:10CE100080933E0D00936F02DCEFD20FCFEFCF5F18
:10CE2000DF5FC43008F4ABCEDF91CF911F910F913B
:10CE3000FF90EF90DF90CF90BF90AF909F908F903A
:10CE400008958F929F92AF92BF92CF92DF92EF920E
:10CE5000FF920F931F93CF93DF938091350D9091A5
:10CE6000360DA091370DB091380D81309048A10555
:10CE7000B10540F01092350D1092360D1092370D1D
:10CE80001092380D6091350D7091360D8091370DEF
:10CE90009091380D25E030E040E050E00E947EB2F5
:10CEA00080913E0D90E0A0E0B0E0281739074A07D6
:10CEB0005B0710F420933E0DD0913E0D10913F0D75
:10CEC00012FB112710F9C0E025E0C22ED12CE12C75
:10CED000F12C3DE1832E912CA12CB12C01E060912D
:10CEE000350D7091360D8091370D9091380DD1111F
:10CEF00031C020916F02222369F023E06530710573
:10CF00008105910510F443E001C040E264E370E163
:10CF10008C2F6CDC112309F429C18091350D90917F
:10CF2000360DA091370DB091380D0597A105B105CB
:10CF300008F01CC182DD8CE692E7DF91CF911F9152
:10CF40000F91FF90EF90DF90CF90BF90AF909F90A8
:10CF50008F90BDCDD13079F520916F02222391F0D1
:10CF6000A70196010E947EB221303105410551058D
:10CF700019F42EE74EE302C02EE740E268E270E1CA
:10CF80008C2F34DC112309F4F1C06091350D7091C0
:10CF9000360D8091370D9091380DA70196010E94B2
:10CFA0007EB2213031054105510509F0DFC045DD74
:10CFB0008BEA99E730C0D230D9F520916F02222355
:10CFC00091F0A70196010E947EB222303105410501
:10CFD000510519F42EE74EE302C02EE740E26EE160
:10CFE00070E18C2F03DC112309F4C0C06091350D72
:10CFF0007091360D8091370D9091380DA7019601F3
:10D000000E947EB2223031054105510509F0AEC0C3
:10D0100014DD8FEA9AE6DF91CF911F910F91FF9077
:10D02000EF90DF90CF90BF90AF909F908F9054CDB6
:10D03000D33079F520916F02222391F0A701960158
:10D040000E947EB2233031054105510519F420E2DA
:10D050004EE302C020E240E262E170E18C2FC6DBC9
:10D06000112309F483C06091350D7091360D8091C4
:10D07000370D9091380DA70196010E947EB22330A2
:10D0800031054105510509F071C0D7DC8CE090E114
:10D090005FC0D43079F520916F02222391F0A7016F
:10D0A00096010E947EB2243031054105510519F4E4
:10D0B00020E24EE302C020E240E26BEF7FE08C2FE3
:10D0C00095DB112309F452C06091350D7091360D36
:10D0D0008091370D9091380DA70196010E947EB284
:10D0E000243031054105510509F040C0A6DC87EF29
:10D0F0009FE02EC0D530D1F520916F02222391F010
:10D10000A70196010E947EB22530310541055105E7
:10D1100019F420E24EE302C020E240E26DEE7FE02F
:10D120008C2F64DB112311F16091350D7091360D58
:10D130008091370D9091380DA70196010E947EB223
:10D14000253031054105510589F477DC89EE9FE0F2
:10D15000DF91CF911F910F91FF90EF90DF90CF90D3
:10D16000BF90AF909F908F900C94333E8091350D7F
:10D170009091360DA091370DB091380D4E97A105C5
:10D18000B10540F08092350D9092360DA092370D8A
:10D19000B092380D6091350D7091360D8091370D3C
:10D1A0009091380DA70196010E947EB280913E0DAC
:10D1B00090E00396422F50E0841795074CF48DEFD2
:10D1C000820F80933E0D00936F02DCEFD20FCFEF02
:10D1D000CF5FDF5FC43008F482CEDF91CF911F9123
:10D1E0000F91FF90EF90DF90CF90BF90AF909F9006
:10D1F0008F900895BF92CF92DF92EF92FF920F939C
:10D200001F93CF93DF938091350D9091360DA091B0
:10D21000370DB091380D81309048A105B10540F02F
:10D220001092350D1092360D1092370D1092380D68
:10D230006091350D7091360D8091370D9091380DBC
:10D2400025E030E040E050E00E947EB280913E0D4B
:10D2500090E0A0E0B0E0281739074A075B0710F418
:10D2600020933E0DD0913E0D10913F0D12FB1127E2
:10D2700010F9C0E065E0C62ED12CE12CF12C01E0C4
:10D280006091350D7091360D8091370D9091380D6C
:10D29000D1112EC020916F02222369F023E0653066
:10D2A00071058105910510F443E001C040E260EE94
:10D2B0007FE08C2F9BDA112309F479C08091350D22
:10D2C0009091360DA091370DB091380D0597A105BD
:10D2D000B10508F06CC0B1DB81E297E6DF91CF9138
:10D2E0001F910F91FF90EF90DF90CF90BF90EFCB09
:10D2F000D13071F520916F02222391F0A7019601A0
:10D300000E947EB2213031054105510519F42EE706
:10D310004EE302C02EE740E269ED7FE08C2F66DA33
:10D32000112309F444C06091350D7091360D809140
:10D33000370D9091380DA70196010E947EB22130E1
:10D3400031054105510599F578DB8FE090E8A8C0DB
:10D35000D23069F520916F02222391F0A701960146
:10D360000E947EB2223031054105510519F42EE7A5
:10D370004EE302C02EE740E262ED7FE08C2F36DA0A
:10D380001123A9F06091350D7091360D8091370D04
:10D390009091380DA70196010E947EB2223031058E
:10D3A0004105510521F449DB86E190E879C020E090
:10D3B00030E040E251E46091110D7091120D8091C6
:10D3C000130D9091140D0E94A0AE87FF73C0609161
:10D3D000350D7091360D8091370D9091380DD33009
:10D3E00081F520916F02222391F0A70196010E94FE
:10D3F0007EB2233031054105510519F42EE74EE385
:10D4000002C02EE740E26BEC7FE08C2FEFD91111C8
:10D4100003C055E0B52E50C06091350D7091360DAA
:10D420008091370D9091380DA70196010E947EB230
:10D43000233031054105510561F7FFDA8DE190E8B0
:10D440002FC0D43031F720916F02222391F0A70131
:10D4500096010E947EB2243031054105510519F430
:10D460002EE74EE302C02EE740E262EC7FE08C2F15
:10D47000BDD9112371F26091350D7091360D8091F7
:10D48000370D9091380DA70196010E947EB224308D
:10D4900031054105510509F0BCCFCFDA8BE49EE799
:10D4A000DF91CF911F910F91FF90EF90DF90CF9080
:10D4B000BF9012CB43E0B42E6091350D7091360DC4
:10D4C0008091370D9091380DA70196010E947EB290
:10D4D0008B2D90E0A0E0B0E0281739074A075B07E2
:10D4E00088F025E0B29EC00111240197AA2797FD7C
:10D4F000A095BA2F8093350D9093360DA093370DDC
:10D50000B093380D6091350D7091360D8091370DC7
:10D510009091380DA70196010E947EB280913E0D38
:10D5200090E00396422F50E0841795074CF48DEF5E
:10D53000820F80933E0D00936F02DCEFD20FCFEF8E
:10D54000CF5FDF5FC43008F49BCEDF91CF911F9196
:10D550000F91FF90EF90DF90CF90BF90089580E003
:10D5600090E0A0E8BFE38093110D9093120DA0937B
:10D57000130DB093140D3ECE20E044E064E180E44E
:10D580009DE00E94B128BCD980E49DE00C947228F3
:10D59000F3DF20E040E050E0BA0184E290E881CA85
:10D5A00010924908109248081092470810924608B5
:10D5B00010922F0A10922E0AEBCF80E49DE00C947B
:10D5C000722820E030E04EE353E46091400870910F
:10D5D000410880914208909143080E94A3B0181618
:10D5E0004CF480E89EE00E94333E83E79EE00E9478
:10D5F000333E20C0E2DF40E060E080E49DE00E9436
:10D600007E286BEC74E080E49DE00E94BEAD42E0B9
:10D6100060E080E49DE00E947E2862ED74E080E49A
:10D620009DE00E94BEAD60ED77E080E090E00E945A
:10D6300060A9C3DFADCF20E030E04EE353E460915A
:10D6400040087091410880914208909143080E94DF
:10D65000A3B018166CF48FE69EE00E94333E83E67A
:10D660009EE00E94333E87E59EE00E94333E20C04C
:10D67000A4DF40E060E080E49DE00E947E286BEC47
:10D6800074E080E49DE00E94BEAD42E060E080E492
:10D690009DE00E947E2862ED74E080E49DE00E949F
:10D6A000BEAD60ED77E080E090E00E9460A985DF8C
:10D6B0006FCF8091970D9091980D9093490880932A
:10D6C00048088091950D9091960D9093470880930E
:10D6D000460810922F0A10922E0A5ADF0C94442109
:10D6E0008091910D9091920D9093490880934808F4
:10D6F00080918F0D9091900D9093470880934608EC
:10D7000010922F0A10922E0A43DF0C94442180912C
:10D7100095029091960290934908809348088091D1
:10D720009302909194029093470880934608109238
:10D730002F0A10922E0A2CDF0C9444218091910222
:10D7400090919202909349088093480880918F02AB
:10D7500090919002909347088093460810922F0A68
:10D7600010922E0A15DF0C94442180918D02909125
:10D770008E02909349088093480880918B02909183
:10D780008C02909347088093460810922F0A1092BB
:10D790002E0AFEDE0C9444218091890290918A0227
:10D7A000909349088093480880918702909188025D
:10D7B000909347088093460810922F0A10922E0AE1
:10D7C000E7DE0C9444212F923F924F925F926F922A
:10D7D0007F928F929F92AF92BF92CF92DF92EF9201
:10D7E000FF920F931F93CF93DF93CDB7DEB7A89728
:10D7F0000FB6F894DEBF0FBECDBF80916F028111CE
:10D8000004C080913F0D82FFEBC28DE59AE00E943B
:10D810001B389DA38CA38091350D9091360DA0915E
:10D82000370DB091380D81309048A105B10540F019
:10D830001092350D1092360D1092370D1092380D52
:10D840006091350D7091360D8091370D9091380DA6
:10D8500025E030E040E050E00E947EB280913E0D35
:10D8600090E0A0E0B0E0281739074A075B0710F402
:10D8700020933E0D40903E0D80913F0D82FB882706
:10D8800080F98F8F512C35E0C32ED12CE12CF12C57
:10D8900041102DC080916F028823A9F08091350D31
:10D8A0009091360DA091370DB091380D23E005977A
:10D8B000A105B10510F443E001C040E26BE77FE051
:10D8C000852D0E94F6632F8D222389F08091350DDE
:10D8D0009091360DA091370DB091380D0597A105A7
:10D8E000B10528F4AAD88CE692E7F1D879C261E6AE
:10D8F0007AE08BEC9AE00E9440108091610A8F32AE
:10D9000031F041E0441671F022E0722E02C077241B
:10D9100073940CA11DA101501109842C912CA12CF0
:10D92000B12C52C080916F028823D9F06091350DDF
:10D930007091360D8091370D9091380DA7019601A9
:10D940000E947EB2213031054105510519F420E2D3
:10D950004EE302C020E240E267E77FE0852D0E94AF
:10D96000F6638F8D882381F26091350D7091360DAD
:10D970008091370D9091380DA70196010E947EB2DB
:10D98000213031054105510509F0BECF56D80E941E
:10D990006F6426C2741088C140E050E0B8018DE584
:10D9A0009AE00E9492349091A30A80916F02992389
:10D9B00009F4A1C081110DC09F8D911179C0772408
:10D9C0007394740C015011090F3FFFEF1F0711F7FB
:10D9D0006DC16091350D7091360D8091370D90912C
:10D9E000380DA70196010E947EB2281539054A0517
:10D9F0005B0579F5452D60E080E49DE00E947E287E
:10DA00006EE380E49DE00E94BFAD65E080E49DE0B0
:10DA10000E94BFAD80916E0A882329F01092800A7F
:10DA20008EE69AE002C081E69AE03C0192E1392E4E
:10DA3000F30161913F01662311F0311085C133205C
:10DA400009F4BACF60E280E49DE00E94BFAD3A9451
:10DA5000F6CF452D60E080E49DE00E947E2860E2E4
:10DA600080E49DE00E94BFAD65E080E49DE00E94FF
:10DA7000BFAD80916E0A882329F01092800A8EE64D
:10DA80009AE002C081E69AE03C0182E1382EF3017F
:10DA900061913F01662311F031105CC1332009F41C
:10DAA0008BCF60E280E49DE00E94BFAD3A94F6CF58
:10DAB0006091350D7091360D8091370D9091380D34
:10DAC000A70196010E947EB2281539054A055B051B
:10DAD00009F075CF0E941D6561E67AE08DE59AE058
:10DAE0000E947E381092350D1092360D1092370D2F
:10DAF0001092380D75C1811104C0FF8DF11191C0D4
:10DB00005ECF6091350D7091360D8091370D9091FB
:10DB1000380DA70196010E947EB2281539054A05E5
:10DB20005B0509F054C020919B0D2EA3712C472D4D
:10DB300060E080E49DE00E947E2860E280E49DE059
:10DB40000E94BFAD739444E07412F1CF452D60E0A4
:10DB500080E49DE00E947E286EE380E49DE00E94C8
:10DB6000BFADBFE62B2EBAE03B2E2EE63AE0612C8D
:10DB7000712C39A328A361E070E0E8A1F9A12191FB
:10DB8000F9A3E8A32223B1F0CB0101969BA38AA3BA
:10DB9000452D80E49DE028A76114710409F4E0C0DC
:10DBA0000E947E2828A5622F80E49DE00E94BFADE0
:10DBB0006AA17BA1F4E17F2E761A772009F49DCF2C
:10DBC00060E280E49DE00E94BFAD7A94F6CF452DDF
:10DBD00060E080E49DE00E947E2860E280E49DE0B9
:10DBE0000E94BFAD80916E0A882329F01092810AAD
:10DBF0008EE69AE002C081E69AE03C01E3E13E2E27
:10DC0000F30161913F01662311F03110E3C033202D
:10DC100009F473CF60E280E49DE00E94BFAD3A94C6
:10DC2000F6CF6091350D7091360D8091370D909142
:10DC3000380DA70196010E947EB2281539054A05C4
:10DC40005B0509F0BCCE0E941D6581E69AE09F93BA
:10DC50008F9380E79FE09F938F938E010F5F1F4FFD
:10DC60001F930F930E945BB60F900F900F900F9031
:10DC70000F900F907E01F5E0EF0EF11CF70180810F
:10DC8000882349F0992787FD90950E9498B5F70160
:10DC900081937F01F3CFC8010E94C03D8CE69FE0D5
:10DCA0000E94333E75DC9CC073948CCE6091350D20
:10DCB0007091360D8091370D9091380DA701960126
:10DCC0000E947EB2872D90E0A0E0B0E028173907CF
:10DCD0004A075B0788F025E0729EC0011124019776
:10DCE000AA2797FDA095BA2F8093350D9093360DF6
:10DCF000A093370DB093380D6091350D7091360DAE
:10DD00008091370D9091380DA70196010E947EB247
:10DD100080913E0D90E00396422F50E084179507C6
:10DD200064F48DEF820F80933E0D81E080936F024B
:10DD30007CEF472E420E55245A945394439443E06B
:10DD4000451508F0A5CD4CC080E49DE00E94BFAD14
:10DD50003A946ECE80E49DE00E94BFAD3A9497CE97
:10DD60000E947E2828A5622F80E49DE00E94BFAD1E
:10DD70006AA17BA16431710509F0FFCE9101ACE28B
:10DD80006A2E7724739480913F0D82FD05C08091A7
:10DD90009B0D9EA1981789F081E090E0E1E06E1A5A
:10DDA00071086114710421F0892B69F381E090E01E
:10DDB000FFEF2F1A3F0A3C01DCCE61E070E080E00B
:10DDC00090E028A73FA30E9460A980E090E028A5EA
:10DDD0003FA1E4CF80E49DE00E94BFAD3A9410CF14
:10DDE000A8960FB6F894DEBF0FBECDBFDF91CF91DE
:10DDF0001F910F91FF90EF90DF90CF90BF90AF9069
:10DE00009F908F907F906F905F904F903F902F905A
:10DE100008958F929F92AF92BF92CF92DF92EF922E
:10DE2000FF920F931F93CF93DF938091350D9091C5
:10DE3000360DA091370DB091380D81309048A10575
:10DE4000B10540F01092350D1092360D1092370D3D
:10DE50001092380D6091350D7091360D8091370D0F
:10DE60009091380D25E030E040E050E00E947EB215
:10DE700080913E0D90E0A0E0B0E0281739074A07F6
:10DE80005B0710F420933E0DD0913E0D10913F0D95
:10DE900012FB112710F9C0E045E0C42ED12CE12C73
:10DEA000F12C57E2852E912CA12CB12C01E0609130
:10DEB000350D7091360D8091370D9091380DD1113F
:10DEC00034C020916F02222371F023E06530710588
:10DED0008105910510F443E001C040E267E57FE071
:10DEE0008C2F0E94F663112309F4C8C18091350D6F
:10DEF0009091360DA091370DB091380D0597A10581
:10DF0000B10508F0BBC10E941D658CE692E7DF9168
:10DF1000CF911F910F91FF90EF90DF90CF90BF9026
:10DF2000AF909F908F900C946765D130D9F5209178
:10DF30006F02222399F0A70196010E947EB2213040
:10DF400031054105510519F420E24EE302C020E2FB
:10DF500040E267E47FE08C2F0E94F663112309F40E
:10DF60008DC16091350D7091360D8091370D909176
:10DF7000380DA70196010E947EB22130310541057E
:10DF8000510509F07BC10E941D65DF91CF911F9162
:10DF90000F91FF90EF90DF90CF90BF90AF909F9048
:10DFA0008F909ECBD230D9F520916F02222399F029
:10DFB000A70196010E947EB222303105410551052C
:10DFC00019F420E24EE302C020E240E268E37FE081
:10DFD0008C2F0E94F663112309F450C16091350D16
:10DFE0007091360D8091370D9091380DA7019601F3
:10DFF0000E947EB2223031054105510509F03EC133
:10E000000E941D65DF91CF911F910F91FF90EF90BE
:10E01000DF90CF90BF90AF909F908F904ACBD3303E
:10E02000D9F520916F02222399F0A70196010E9451
:10E030007EB2233031054105510519F420E24EE34B
:10E0400002C020E240E269E27FE08C2F0E94F6638A
:10E05000112309F413C16091350D7091360D809133
:10E06000370D9091380DA70196010E947EB22330A2
:10E0700031054105510509F001C10E941D65DF917F
:10E08000CF911F910F91FF90EF90DF90CF90BF90B5
:10E09000AF909F908F9052CBD430D9F520916F02E2
:10E0A000222399F0A70196010E947EB22430310507
:10E0B0004105510519F420E24EE302C020E240E29E
:10E0C00069E17FE08C2F0E94F663112309F4D6C02A
:10E0D0006091350D7091360D8091370D9091380D0E
:10E0E000A70196010E947EB22430310541055105F9
:10E0F00009F0C4C00E941D65DF91CF911F910F915F
:10E10000FF90EF90DF90CF90BF90AF909F908F9057
:10E110002CCBD530D9F520916F02222399F0A7019D
:10E1200096010E947EB2253031054105510519F452
:10E1300020E24EE302C020E240E269E07FE08C2F63
:10E140000E94F663112309F499C06091350D709116
:10E15000360D8091370D9091380DA70196010E94E0
:10E160007EB2253031054105510509F087C00E9476
:10E170001D65DF91CF911F910F91FF90EF90DF9080
:10E18000CF90BF90AF909F908F90C1CAD630D9F5F5
:10E1900020916F02222399F0A70196010E947EB27E
:10E1A000263031054105510519F420E24EE302C045
:10E1B00020E240E26AEF7EE08C2F0E94F66311239A
:10E1C00009F45CC06091350D7091360D8091370D6A
:10E1D0009091380DA70196010E947EB2263031053C
:10E1E0004105510509F04AC00E941D65DF91CF919C
:10E1F0001F910F91FF90EF90DF90CF90BF90AF9065
:10E200009F908F90C9CAD730C9F520916F02222301
:10E2100099F0A70196010E947EB227303105410591
:10E22000510519F420E24EE302C020E240E261EF22
:10E230007EE08C2F0E94F663112301F16091350D71
:10E240007091360D8091370D9091380DA701960190
:10E250000E947EB2273031054105510579F40E94B4
:10E260001D65DF91CF911F910F91FF90EF90DF908F
:10E27000CF90BF90AF909F908F9092C98091350DB5
:10E280009091360DA091370DB091380D8897A1056A
:10E29000B10540F08092350D9092360DA092370D69
:10E2A000B092380D6091350D7091360D8091370D1B
:10E2B0009091380DA70196010E947EB280913E0D8B
:10E2C00090E00396422F50E0841795074CF48DEFB1
:10E2D000820F80933E0D00936F02DCEFD20FCFEFE1
:10E2E000CF5FDF5FC43008F4E2CDDF91CF911F91A3
:10E2F0000F91FF90EF90DF90CF90BF90AF909F90E5
:10E300008F9008955AD941E060E080E49DE00E943A
:10E310007E2869EF74E080E49DE00E94BEAD42E09B
:10E3200060E080E49DE00E947E2869E075E080E482
:10E330009DE00C94BEAD41D942E060E080E49DE0F8
:10E340000E947E286CE175E080E49DE00C94BEADF7
:10E350001F93CF93DF9331D940E060E080E49DE0EC
:10E360000E947E286CE275E080E49DE00E94BEADD4
:10E3700042E060E080E49DE00E947E286AE375E070
:10E3800080E49DE00E94BEAD10E043E0612F80E498
:10E390009DE00E947E286FE573E080E49DE00E948E
:10E3A000BEADCAE0D0E00E94721E81E00E943849F2
:10E3B00065E570E080E090E00E9460A921972097D9
:10E3C00091F71F5F143109F7DF91CF911F910895E5
:10E3D0001F93CF93DF93F1D840E060E080E49DE0AD
:10E3E0000E947E2866E475E080E49DE00E94BEAD58
:10E3F00042E060E080E49DE00E947E286AE375E0F0
:10E4000080E49DE00E94BEAD10E043E0612F80E417
:10E410009DE00E947E286FE573E080E49DE00E940D
:10E42000BEADCAE0D0E00E94721E81E00E94384971
:10E430006EE670E080E090E00E9460A9219720974E
:10E4400091F71F5F143109F7DF91CF911F91089564
:10E4500080932E0D10922D0D0895E2E7F2E00190C9
:10E460000020E9F73197E257F2401E161F0634F0FC
:10E470001092860282E080936F02089580E2E43178
:10E48000F105B4F7DF01AE58BD4F8C933196F7CF4D
:10E4900020918C0D211108C044E150E0BC0182E7BD
:10E4A00092E00E944CB6D9CF089510925F0A60E0C6
:10E4B0008DE59AE00E947D340E94B39380E69FE050
:10E4C0000E94333E81E080931F0A87E595E0E0DFFC
:10E4D0008CE59FE00C94333EAF92BF92CF92DF92D7
:10E4E000EF92FF920F931F93CF93DF931092990DAA
:10E4F0008091350D9091360DA091370DB091380D6A
:10E5000081309048A105B10540F01092350D109270
:10E51000360D1092370D1092380D6091350D7091B7
:10E52000360D8091370D9091380D25E030E040E0B8
:10E5300050E00E947EB280913E0D90E0A0E0B0E0FD
:10E54000281739074A075B0710F420933E0DD09136
:10E550003E0D10913F0D12FB112710F9C0E075E040
:10E56000C72ED12CE12CF12CAA24A394D11137C0B1
:10E5700080916F028823A9F08091350D9091360D1E
:10E58000A091370DB091380D23E00597A105B10595
:10E5900010F443E001C040E264E071E18C2F0E947E
:10E5A000F6631123E1F08091350D9091360DA09125
:10E5B000370DB091380D0597A105B10580F40E9483
:10E5C0001D6584E290E8DF91CF911F910F91FF903C
:10E5D000EF90DF90CF90BF90AF900C9467650E9452
:10E5E00000A54091350D5091360D6091370D709119
:10E5F000380D811104C080915F0A882399F1D130D0
:10E60000C9F580916F028823A9F0CB01BA01A70157
:10E6100096010E947EB2213031054105510519F461
:10E620002EE74EE302C02EE740E26FEF70E18C2F41
:10E630000E94F6631123F1F06091350D7091360D53
:10E640008091370D9091380DA70196010E947EB2FE
:10E65000213031054105510569F40E941D6582E6AE
:10E660009BE73EC2D13031F480916F0281119BC291
:10E670001111AFC22091600A6091350D7091360D75
:10E680008091370D9091380D222309F4F1C020912B
:10E69000480C222309F4B9C020915F0A2223E9F132
:10E6A000D23009F076C020916F02222399F0A701A1
:10E6B00096010E947EB2223031054105510519F4C0
:10E6C00020E24EE302C020E240E26BEE70E18C2FCC
:10E6D0000E94F663112309F4E2C06091350D709138
:10E6E000360D8091370D9091380DA70196010E944B
:10E6F0007EB2223031054105510509F0D0C00E949B
:10E700001D65DF91CF911F910F91FF90EF90DF90EA
:10E71000CF90BF90AF900C947C64D230D1F5209113
:10E720006F02222399F0A70196010E947EB2223047
:10E7300031054105510519F420E24EE302C020E203
:10E7400040E26EED70E18C2F0E94F663112309F414
:10E75000A6C06091350D7091360D8091370D909166
:10E76000380DA70196010E947EB222303105410585
:10E77000510509F094C00E941D65DF91CF911F9152
:10E780000F91FF90EF90DF90CF90BF90AF900C94DF
:10E790007864D33009F083C020916F02222399F06E
:10E7A000A70196010E947EB2233031054105510533
:10E7B00019F420E24EE302C020E240E263ED70E192
:10E7C0008C2F0E94F663112309F469C06091350D06
:10E7D0007091360D8091370D9091380DA7019601FB
:10E7E0000E947EB2233031054105510509F057C022
:10E7F0000E941D65DF91CF911F910F91FF90EF90C7
:10E80000DF90CF90BF90AF9050CED23011F003E0A8
:10E8100047C020916F02222399F0A70196010E9420
:10E820007EB2223031054105510519F42EE74EE341
:10E8300002C02EE740E265EC70E18C2F0E94F66387
:10E84000112329F36091350D7091360D8091370DAC
:10E850009091380DA70196010E947EB222303105B9
:10E8600041055105A1F60E941D6583EE9BE638C166
:10E87000D23069F620916F02222311F3A70196018D
:10E880000E947EB2223031054105510519F42EE770
:10E890004EE302C02EE740E26AEB70E1CECF04E027
:10E8A00080915F0A8111DCC00D1348C080916F0216
:10E8B0008823F9F06091350D7091360D8091370DF8
:10E8C0009091380DA70196010E947EB2802F90E0B2
:10E8D000A0E0B0E0281739074A075B0719F420E2E7
:10E8E0004EE302C020E240E26CEA70E18C2F0E940D
:10E8F000F663112319F16091350D7091360D8091F9
:10E90000370D9091380DA70196010E947EB2802F9D
:10E9100090E0A0E0B0E0281739074A075B0771F4E0
:10E920000E941D65DF91CF911F910F91FF90EF9095
:10E93000DF90CF90BF90AF900C941B6BBB24B3942F
:10E94000B00EBD1248C080916F028823F9F060912B
:10E95000350D7091360D8091370D9091380DA701CE
:10E9600096010E947EB28D2F90E0A0E0B0E02817C3
:10E9700039074A075B0719F420E24EE302C020E2A0
:10E9800040E26CE970E18C2F0E94F663112319F1CB
:10E990006091350D7091360D8091370D9091380D45
:10E9A000A70196010E947EB28B2D90E0A0E0B0E01E
:10E9B000281739074A075B0771F40E941D65DF912C
:10E9C000CF911F910F91FF90EF90DF90CF90BF906C
:10E9D000AF900C94E16A62E0B62EB00EBD123FC05B
:10E9E00080916F028823F9F06091350D7091360D9A
:10E9F0008091370D9091380DA70196010E947EB24B
:10EA00008D2F90E0A0E0B0E0281739074A075B0798
:10EA100019F42EE74EE302C02EE740E263E970E10D
:10EA20008C2F0E94F6631123D1F06091350D709107
:10EA3000360D8091370D9091380DA70196010E94F7
:10EA40007EB28B2D90E0A0E0B0E0281739074A078E
:10EA50005B0729F40E941D6581E297E641C00D5FC6
:10EA60000D134AC080916F028823F9F06091350D33
:10EA70007091360D8091370D9091380DA701960158
:10EA80000E947EB2802F90E0A0E0B0E02817390706
:10EA90004A075B0719F42EE74EE302C02EE740E277
:10EAA0006BE870E18C2F0E94F663112329F16091CD
:10EAB000350D7091360D8091370D9091380DA7016D
:10EAC00096010E947EB2802F90E0A0E0B0E028176F
:10EAD00039074A075B0781F40E941D6581E795E6C7
:10EAE000DF91CF911F910F91FF90EF90DF90CF902A
:10EAF000BF90AF900C946C65BB24B394B00E609142
:10EB0000350D7091360D8091370D9091380DA7011C
:10EB100096010E947EB28B2D90E0A0E0B0E0281715
:10EB200039074A075B0788F025E0B29EC00111242F
:10EB30000197AA2797FDA095BA2F8093350D909342
:10EB4000360DA093370DB093380D6091350D70914F
:10EB5000360D8091370D9091380DA70196010E94D6
:10EB60007EB280913E0D90E00396422F50E08417D4
:10EB700095074CF48DEF820F80933E0DA0926F02AB
:10EB8000DCEFD20FCFEFCF5FDF5FC43008F4EECC05
:10EB9000DF91CF911F910F91FF90EF90DF90CF9079
:10EBA000BF90AF900895CB01BA01A70196010E94D2
:10EBB0007EB2213031054105510519F42EE74EE3AF
:10EBC00002C02EE740E267EF70E18C2F0E94F663EF
:10EBD0004FCD6091350D7091360D8091370D90912C
:10EBE000380DA70196010E947EB221303105410502
:10EBF000510509F03FCD0E941D6589E09FE670CF69
:10EC000020918C0D211108C044E150E0BC0182E745
:10EC100092E00E94BFB521CC0895F2DF81E080939D
:10EC20008C0D0C94C86A10928C0D0895CF92DF92CF
:10EC3000EF92FF92CF93CCB1C095CC1FCC27CC1FC5
:10EC40008091030183FFC260C0903A0DD0903B0DCC
:10EC5000E0903C0DF0903D0D0E9431A9C616D706FC
:10EC6000E806F90610F4489B39C0C0933F0D809127
:10EC70003F0D817090913F0D91FD82609091390D13
:10EC8000891721F18130F1F028F0823089F083304A
:10EC9000A1F01CC0913021F490919B0D9F5F05C0A5
:10ECA0009230A1F490919B0D915090939B0D0EC0CA
:10ECB000992391F3933051F4F5CF923069F3913069
:10ECC00029F4F0CF933041F3992361F38093390D08
:10ECD000CF91FF90EF90DF90CF900895C460C5CFA3
:10ECE0000E94BC6A6F98E4E0F1E08081877F8083B6
:10ECF000779A9FB7F894E5E0F1E08081886080839F
:10ED00009FBF5098589A60E088E40E9451A89FB72E
:10ED1000F894E5E0F1E08081846080839FBF80917A
:10ED2000030182FB882780F991E089278093340DC5
:10ED30007DDF10929B0D0895CF92DF92EF92FF92AC
:10ED400075DF8091030191E082FB882780F9892794
:10ED50002091340D8217C9F082E080936F02809178
:10ED6000030182FB882780F989278093340D0E9454
:10ED7000BC6A8091340D882309F490C08DE59AE037
:10ED80000E94473089E49EE03BDFC090300DD09078
:10ED9000310DE090320DF090330D0E9431A9C6166E
:10EDA000D706E806F90608F086C040919B0D44237B
:10EDB00061F181E080936F02552747FD5095652FE3
:10EDC000752F8091350D9091360DA091370DB09132
:10EDD000380D840F951FA61FB71F8093350D909394
:10EDE000360DA093370DB093380D10929B0D0E94F5
:10EDF00031A96856754C8F4F9F4F6093050D7093E6
:10EE0000060D8093070D9093080D80913F0D82FFB2
:10EE10000EC00E9431A96856754C8F4F9F4F60936A
:10EE2000050D7093060D8093070D9093080DE091EA
:10EE30007002F09171021995C090050DD090060DE9
:10EE4000E090070DF090080D0E9431A9C616D70674
:10EE5000E806F90638F480917002909171028452AC
:10EE6000904819F580916F02823011F40E94DD6A9A
:10EE700080916F02882319F0815080936F020E9465
:10EE800031A96C597F4F8F4F9F4F6093300D709316
:10EE9000310D8093320D9093330D0DC08DE59AE0C6
:10EEA0000E9412318CE39EE06FCF0E94C86A82E01C
:10EEB00080936F02D7CFFF90EF90DF90CF900895AF
:10EEC00081E0089580913F0D82FB882780F90895A5
:10EED0000F931F93CF93DF930E94DD6A40E060E0C1
:10EEE00080E49DE00E947E2865E675E080E49DE078
:10EEF0000E94BEAD41E061E080E49DE00E947E287A
:10EF000068E775E080E49DE00E94BEAD42E061E00C
:10EF100080E49DE00E947E286CE775E080E49DE03F
:10EF20000E94BEAD43E061E080E49DE00E947E2847
:10EF300060E975E080E49DE00E94BEAD41E060E0E4
:10EF400080E49DE00E947E2860EA75E080E49DE018
:10EF50000E94BEAD00919B0D112707FD1095C1E0E9
:10EF6000D0E08091550A9091560A892B09F076C01D
:10EF70000E94721E81E00E94384980919B0D992762
:10EF800087FD90950817190709F459C09801281BA7
:10EF9000390B37FF03C031952195310922303105F6
:10EFA0000CF44DC0801791070CF42197081719072E
:10EFB0000CF42196C430D1052CF4209729F4C1E03B
:10EFC000D0E002C0C3E0D0E041E060E080E49DE03A
:10EFD0000E947E2861E973E080E49DE00E94BEAD5E
:10EFE00042E060E080E49DE00E947E2861E973E0F9
:10EFF00080E49DE00E94BEAD43E060E080E49DE0DF
:10F000000E947E2861E973E080E49DE00E94BEAD2D
:10F010004C2F60E080E49DE00E947E2860EA75E06D
:10F0200080E49DE00E94BEAD00919B0D112707FD7D
:10F03000109564E670E080E090E00E9460A942DFF5
:10F04000882309F48ECFD093560AC093550A64EFF3
:10F0500071E080E090E00E9460A983CF0E94DD6AA9
:10F06000DF91CF911F910F910C94C86AFC018081B0
:10F0700090E02AE030E0B9010E946BB2482FCB014A
:10F08000B9010E946BB2805D8093090D405D409391
:10F090000A0D10920B0D89E09DE0089520E030E00C
:10F0A00040E251E4FC0160817181828193810E9480
:10F0B00075B10E940FAF77FD02C02BE201C02DE2B7
:10F0C0002093090D9B0177FF04C022273327261BBD
:10F0D000370BC90168EE73E00E946BB2CB01EAE026
:10F0E000F0E0BF010E946BB2805D80930A0DC90100
:10F0F00064E670E00E946BB2CB01BF010E946BB26C
:10F10000805D80930B0DC901BF010E946BB2282F57
:10F11000CB01BF010E946BB2805D80930C0D8EE22B
:10F1200080930D0D205D20930E0D10920F0D89E040
:10F130009DE008958F929F92AF92BF92CF92DF92FF
:10F14000EF92FF92FC0180809180A280B38020E04A
:10F1500030E048EC52E4C501B4010E9475B16B0186
:10F160007C0120E030E0A9010E94A3B018161CF435
:10F17000C701B60103C0C701B60190580E940FAF86
:10F180006B017C0120E030E0A901C501B4010E94BF
:10F19000A0AE87FF12C08DE28093090DC701B601B2
:10F1A00028EE33E040E050E00E94A0B2CA01B9016D
:10F1B0002AE030E040E050E036C0C701B60120E16F
:10F1C00037E240E050E00E94A0B28AE0882E912C05
:10F1D000A12CB12CCA01B901A50194010E94A0B2D1
:10F1E000662391F0605D6093090DC701B60128EEBA
:10F1F00033E040E050E00E94A0B2CA01B901A5018D
:10F2000094010E94A0B213C080E28093090DC7014F
:10F21000B60128EE33E040E050E00E94A0B2CA01FF
:10F22000B901A50194010E94A0B2662311F0605DAE
:10F2300001C060E260930A0DC701B60124E630E028
:10F2400040E050E00E94A0B2BAE08B2E912CA12C9D
:10F25000B12CCA01B901A50194010E94A0B2605D60
:10F2600060930B0DC701B601A50194010E94A0B2E5
:10F27000662381F0605D60930E0DCA01B901A5019E
:10F2800094010E94A0B2605D60930D0D8EE28093A8
:10F290000C0D15C0CA01B901A50194010E94A0B2CC
:10F2A000662329F0605D60930D0D8EE203C080E25D
:10F2B00080930D0D80930C0D80E280930E0D1092C3
:10F2C0000F0D89E09DE0FF90EF90DF90CF90BF9011
:10F2D000AF909F908F900895FC012081318137FF7E
:10F2E00007C08DE28093090D31952195310914C035
:10F2F0002436310574F0C90164E670E00E946BB2F7
:10F30000CB016AE070E00E946BB2805D8093090DD2
:10F3100006C080E28093090D2A30310564F0EAE0EE
:10F32000F0E0C901BF010E946BB2CB01BF010E9496
:10F330006BB2805D01C080E280930A0DC9016AE072
:10F3400070E00E946BB2805D80930B0D10920C0DEB
:10F3500089E09DE008958F929F92AF92BF92CF92E5
:10F36000DF92EF92FF920F931F93CF93DF93609101
:10F3700014027091150280911602909117020E945A
:10F38000BD276093190D70931A0D80931B0D9093F8
:10F390001C0D6091100270911102809112029091E7
:10F3A00013020E94C9276093150D7093160D809368
:10F3B000170D9093180D8091350D9091360DA091F9
:10F3C000370DB091380D81309048A105B10540F05E
:10F3D0001092350D1092360D1092370D1092380D97
:10F3E0006091350D7091360D8091370D9091380DEB
:10F3F00025E030E040E050E00E947EB280913E0D7A
:10F4000090E0A0E0B0E0281739074A075B0710F446
:10F4100020933E0DD0913E0D10913F0D12FB112710
:10F4200010F9C0E095E0C92ED12CE12CF12C23E19C
:10F43000822E912CA12CB12C01E06091350D7091A0
:10F44000360D8091370D9091380DD11134C0209137
:10F450006F02222371F023E065307105810591056B
:10F4600010F443E001C040E26AEA7FE08C2F0E9482
:10F47000F663112309F4E2C08091350D9091360DA9
:10F48000A091370DB091380D0597A105B10508F091
:10F49000D5C00E941D6581E297E6DF91CF911F9153
:10F4A0000F91FF90EF90DF90CF90BF90AF909F9023
:10F4B0008F900C946765D130D9F520916F0222238B
:10F4C000B9F0A70196010E947EB288E498E021304D
:10F4D00031054105510521F4FFDE9C014EE303C0D7
:10F4E000FBDE9C0140E263EA7FE08C2F0E942D64EA
:10F4F000112309F4A3C06091350D7091360D8091F0
:10F50000370D9091380DA70196010E947EB22130EF
:10F5100031054105510509F091C00E941D6528E3A0
:10F5200031E040E050E068E478E08CE99FE078C0AA
:10F53000D230D9F520916F022223B9F0A7019601AC
:10F540000E947EB286E498E02230310541055105E3
:10F5500021F4C2DE9C014EE303C0BEDE9C0140E20A
:10F5600068E97FE08C2F0E942D64112309F466C0A6
:10F570006091350D7091360D8091370D9091380D59
:10F58000A70196010E947EB2223031054105510546
:10F5900009F054C00E941D6523E930E040E050E0CE
:10F5A00066E478E084E99FE03BC0D33009F046C0D0
:10F5B00020916F022223B9F0A70196010E947EB22A
:10F5C0008EE29AE0233031054105510521F484DEB5
:10F5D0009C014EE303C080DE9C0140E26AE87FE0CC
:10F5E0008C2F0E942D64112349F16091350D70918B
:10F5F000360D8091370D9091380DA70196010E942C
:10F600007EB22330310541055105C1F40E941D65CC
:10F610002FEF30E040E050E06EE27AE080E89FE0DB
:10F62000DF91CF911F910F91FF90EF90DF90CF90DE
:10F63000BF90AF909F908F900C94A4638091350DF4
:10F640009091360DA091370DB091380D4497A105DA
:10F65000B10540F08092350D9092360DA092370D95
:10F66000B092380D6091350D7091360D8091370D47
:10F670009091380DA70196010E947EB280913E0DB7
:10F6800090E00396422F50E0841795074CF48DEFDD
:10F69000820F80933E0D00936F02DCEFD20FCFEF0D
:10F6A000CF5FDF5FC43008F4C8CEDF91CF911F91E8
:10F6B0000F91FF90EF90DF90CF90BF90AF909F9011
:10F6C0008F9008958F929F92AF92BF92CF92DF92C8
:10F6D000EF92FF920F931F93CF93DF938091350D9D
:10F6E0009091360DA091370DB091380D8130904832
:10F6F000A105B10540F01092350D1092360D109213
:10F70000370D1092380D6091350D7091360D809146
:10F71000370D9091380D25E030E040E050E00E9438
:10F720007EB280913E0D90E0A0E0B0E0281739074E
:10F730004A075B0710F420933E0DD0913E0D1091C7
:10F740003F0D12FB112710F9C0E035E0C32ED12C7C
:10F75000E12CF12C42E2842E912CA12CB12C01E061
:10F760006091350D7091360D8091370D9091380D67
:10F77000D11134C020916F02222371F023E0653053
:10F7800071058105910510F443E001C040E26CEE83
:10F790007EE08C2F0E94F663112309F49CC18091B6
:10F7A000350D9091360DA091370DB091380D05971C
:10F7B000A105B10508F08FC10E941D658CE692E796
:10F7C000DF91CF911F910F91FF90EF90DF90CF903D
:10F7D000BF90AF909F908F900C946765D130D9F512
:10F7E00020916F022223B9F0A70196010E947EB2F8
:10F7F0008DE592E0213031054105510521F46CDDA4
:10F800009C014EE303C068DD9C0140E266EE7EE0B1
:10F810008C2F0E942D64112309F45DC16091350D78
:10F820007091360D8091370D9091380DA70196019A
:10F830000E947EB2213031054105510509F04BC1CE
:10F840000E941D6527EE33E04AE050E06DE572E06E
:10F8500080EE9EE03DC0D23009F048C020916F029A
:10F860002223B9F0A70196010E947EB288E498E0B5
:10F87000223031054105510521F42EDD9C014EE376
:10F8800003C02ADD9C0140E269ED7EE08C2F0E94DE
:10F890002D64112309F41FC16091350D7091360D4F
:10F8A0008091370D9091380DA70196010E947EB28C
:10F8B000223031054105510509F00DC10E941D6539
:10F8C00028E331E040E050E068E478E082ED9EE03B
:10F8D000DF91CF911F910F91FF90EF90DF90CF902C
:10F8E000BF90AF909F908F900C94A463D330D9F5C4
:10F8F00020916F022223B9F0A70196010E947EB2E7
:10F9000086E498E0233031054105510521F4E4DC1B
:10F910009C014EE303C0E0DC9C0140E26EEC7EE023
:10F920008C2F0E942D64112309F4D5C06091350DF0
:10F930007091360D8091370D9091380DA701960189
:10F940000E947EB2233031054105510509F0C3C044
:10F950000E941D6523E930E040E050E066E478E075
:10F960008AEC9EE0B5CFD430D9F520916F022223E6
:10F97000B9F0A70196010E947EB28EE29AE024308F
:10F9800031054105510521F4A7DC9C014EE303C07C
:10F99000A3DC9C0140E260EC7EE08C2F0E942D6491
:10F9A000112309F498C06091350D7091360D809146
:10F9B000370D9091380DA70196010E947EB2243038
:10F9C00031054105510509F086C00E941D652FEFE4
:10F9D00030E040E050E06EE27AE086EB9EE078CFE7
:10F9E000D530D9F520916F022223B9F0A7019601F5
:10F9F0000E947EB28BE592E025303105410551052C
:10FA000021F46ADC9C014EE303C066DC9C0140E209
:10FA100061EB7EE08C2F0E942D64112309F45BC002
:10FA20006091350D7091360D8091370D9091380DA4
:10FA3000A70196010E947EB225303105410551058E
:10FA400009F049C00E941D6527EE33E04AE050E00E
:10FA50006BE572E08CEA9EE03BCFD630E1F5209179
:10FA60006F02222399F0A70196010E947EB22630F0
:10FA700031054105510519F420E24EE302C020E2B0
:10FA800040E26CE97EE08C2F0E94F663112319F1AD
:10FA90006091350D7091360D8091370D9091380D34
:10FAA000A70196010E947EB226303105410551051D
:10FAB00091F40E941D6587E99EE0DF91CF911F912F
:10FAC0000F91FF90EF90DF90CF90BF90AF909F90FD
:10FAD0008F900C94333E8091350D9091360DA0910E
:10FAE000370DB091380D8397A105B10540F0809294
:10FAF000350D9092360DA092370DB092380D609171
:10FB0000350D7091360D8091370D9091380DA7010C
:10FB100096010E947EB280913E0D90E00396422FA6
:10FB200050E0841795074CF48DEF820F80933E0DC3
:10FB300000936F02DCEFD20FCFEFCF5FDF5FC430F7
:10FB400008F40ECEDF91CF911F910F91FF90EF90AF
:10FB5000DF90CF90BF90AF909F908F900895FC0161
:10FB6000808191818436910524F164E670E00E94E1
:10FB70006BB2CB012AE030E0B9010E946BB2805D2C
:10FB80008093090D80819181B9010E946BB2CB01F4
:10FB9000B9010E946BB2805D80930A0D80819181D2
:10FBA000B9010E946BB2805D80930B0D10920C0D19
:10FBB00023C08A309105BCF02AE030E0B9010E94F0
:10FBC0006BB2CB01B9010E946BB2805D8093090DCD
:10FBD00080819181B9010E946BB2805D80930A0D92
:10FBE00010920B0D09C06AE070E00E946BB2805D5C
:10FBF0008093090D10920A0D89E09DE00895CF923F
:10FC0000EF920F93EFE1CE2EF0E2EF2E0FE02EE019
:10FC100045E066E280E49DE00E9459290F91EF9053
:10FC2000CF900895CF93DF93FC016491EC0121966E
:10FC3000662331F080E49DE00E94362ACE01F4CFA5
:10FC4000DF91CF9108950F931F93CF93DF938C0192
:10FC5000EB0141E061E080E49DE00E947E28C80164
:10FC6000E1DF6AE380E49DE00E94BFADFE01019008
:10FC70000020E9F76C2F6E1B6C5E41E080E49DE094
:10FC80000E947E28BE0180E49DE0DF91CF911F910C
:10FC90000F910C94BEADCF92DF92EF92FF920F9333
:10FCA0001F938091350D9091360DA091370DB09135
:10FCB000380D0097A105B10509F442C0BC018827A1
:10FCC00077FD8095982F0E9442AF2091110D3091C1
:10FCD000120D4091130D5091140D0E9475B19B01AE
:10FCE000AC016091500A7091510A8091520A909132
:10FCF000530A0E94C7AD6093500A7093510A8093D3
:10FD0000520A9093530A1092350D1092360D1092AC
:10FD1000370D1092380DA0E3CA2EAAE0DA2EE12C9E
:10FD2000F12C00E81FE320E53AE04CE45AE068E4F7
:10FD30007AE084E49AE00E94779A81E080936F02EF
:10FD400080916F02882339F080E59AE0A7D9BC0141
:10FD500089EB9FE078DF80913F0D82FF0EC021E0AC
:10FD600040E050E0BA018AEF98E61F910F91FF90B2
:10FD7000EF90DF90CF900C9451651F910F91FF9001
:10FD8000EF90DF90CF900895CF93DF931F921F9253
:10FD9000CDB7DEB78091350D9091360DA091370D1E
:10FDA000B091380DB7FF08C01092350D1092360D86
:10FDB0001092370D1092380D80911D0D90911E0DEF
:10FDC000A0911F0DB091200D4091350D5091360D31
:10FDD0006091370D7091380D84179507A607B70706
:10FDE00044F48093350D9093360DA093370DB09366
:10FDF000380D80916F028823A9F08091210D909198
:10FE0000220D2091350D3091360D820F931F9A836C
:10FE10008983CE01019660DABC018091270D909113
:10FE2000280D11DF80913F0D82FF1DC0E091250D4F
:10FE3000F091260D8091210D9091220D2091350D8C
:10FE40003091360D820F931F918380834091290D4D
:10FE500050912A0D60E070E021E080912B0D90918F
:10FE60002C0D0E9451650F900F90DF91CF91089556
:10FE70004F925F926F927F928F929F92AF92BF92BA
:10FE8000CF92DF92EF92FF920F931F93CF93DF9366
:10FE90004C015B017A018091350D9091360DA09156
:10FEA000370DB091380D892B8A2B8B2B09F47BC031
:10FEB0000E945F40E501CC0FDD1FCC0FDD1F8E01DE
:10FEC0000C5B154F6091350D7091360D882777FDCD
:10FED0008095982F0E9442AF2091110D3091120D04
:10FEE0004091130D5091140D0E9475B1F8012081BD
:10FEF0003181428153810E94C7AD2B013C0120E03A
:10FF000030E0A9010E94A0AEF80187FD05C0408243
:10FF100051826282738204C0108211821282138223
:10FF2000B701882777FD8095982F0E9442AF6B011B
:10FF30007C018E010C5B154F9B01AC01F8016081C7
:10FF40007181828193810E94A3B018162CF4F8016C
:10FF5000C082D182E282F3821092350D1092360D6A
:10FF60001092370D1092380DCA55DA4F20E030E06C
:10FF700040E752E4688179818A819B810E94A7AE23
:10FF8000D0E3CD2EDAE0DD2E7B018C0120E53AE0D6
:10FF90004CE45AE068E47AE084E49AE00E94779ABC
:10FFA00081E080936F0280916F02882359F0C50130
:10FFB000880F991F880F991F8C5B954F6FD8BC01D4
:10FFC000C40141DE80913F0D82FF18C021E040E076
:10FFD00050E0BA018AEF98E6DF91CF911F910F911F
:10FFE000FF90EF90DF90CF90BF90AF909F908F9059
:10FFF0007F906F905F904F900C945165DF91CF91FF
:020000021000EC
:100000001F910F91FF90EF90DF90CF90BF90AF9036
:100010009F908F907F906F905F904F90089546EDE6
:1000200050E060E070E083EB9FE022CF46EC50E0D0
:1000300061E070E085EB9FE01BCF49EC50E062E0AF
:1000400070E087EB9FE014CF8F929F92AF92BF92A8
:10005000CF92DF92EF92FF920F931F93CF93DF9394
:10006000CDB7DEB728970FB6F894DEBF0FBECDBF71
:1000700080912F0D882321F0815080932F0D03C094
:1000800081E080936F0280916F02882309F456C249
:1000900080919A0D8F5F80939A0D8E3129F40E9482
:1000A000BC6A10929A0D0EC06AE00E944AB2911189
:1000B00009C020E044E064E180E49DE00E947E29E4
:1000C0000E94806420E030E040E05FE360914008FF
:1000D0007091410880914208909143080E94C7ADF9
:1000E0000E940FAF78876F8360914808709149082C
:1000F000882777FD8095982F0E9442AF20E030E05E
:1001000040E05FE30E94C7AD0E940FAF7E836D8326
:1001100040E060E080E49DE00E947E2862E080E4B0
:100120009DE00E94BFADCE010796D6D8BC0180E409
:100130009DE00E94BEAD6FE280E49DE00E94BFADF5
:10014000CE0105960CDDBC0180E49DE00E94BEADB1
:1001500084E99EE067DD60E973E080E49DE00E9451
:10016000BEAD40E06AE080E49DE00E947E2862EA45
:1001700075E080E49DE00E94BEAD2CEA35EC47E2DC
:1001800057E360914C0A70914D0A80914E0A90910C
:100190004F0A0E94C7AD69837A838B839C83CE010B
:1001A00001960E949A78BC0180E49DE00E94BEAD59
:1001B00060E280E49DE00E94BFAD41E060E080E449
:1001C0009DE00E947E2820E030E040E05FE3609107
:1001D0003A0870913B0880913C0890913D080E943C
:1001E000C7AD0E940FAF78876F836091460870910A
:1001F0004708882777FD8095982F0E9442AF20E01E
:1002000030E040E05FE30E94C7AD0E940FAF7E8305
:100210006D8360E080E49DE00E94BFADCE01079653
:100220005BD8BC0180E49DE00E94BEAD6FE280E43B
:100230009DE00E94BFADCE01059691DCBC0180E43B
:100240009DE00E94BEAD81E99EE0ECDC60E973E0D8
:1002500080E49DE00E94BEAD41E06AE080E49DE064
:100260000E947E2860E973E080E49DE00E94BEADBC
:1002700066E080E49DE00E94BFAD8DE592E02CD861
:10028000BC0180E49DE00E94BEAD65E280E49DE09B
:100290000E94BFAD6DE873E080E49DE00E94BEADBA
:1002A00042E060E080E49DE00E947E288EE89EE0CF
:1002B000B9DC80915F0A8823A9F18091480C8823DA
:1002C00019F18091F20C9091F30CA091F40CB09183
:1002D000F50C0097A105B105B9F0BC01CD016D5930
:1002E0007F4F8F4F9F4F24E630E040E050E00E9468
:1002F0007EB26091FA0C7091FB0C8091FC0C909195
:10030000FD0C0E947EB201C020E030E03A832983D8
:10031000CE0101960E946C79BC0180E49DE00E94B0
:10032000BEAD03C08AE89EE07DDC65E280E49DE02E
:100330000E94BFAD6CE873E080E49DE00E94BEAD1A
:1003400042E06AE080E49DE00E947E2860E973E07C
:1003500080E49DE00E94BEAD67E080E49DE00E94E5
:10036000BFAD8091520890915308A0915408B0916C
:100370005508892B8A2B8B2BE1F10E9431A920E6AD
:10038000C22E2AEED22EE12CF12CA70196010E945A
:100390007EB249015A0160915208709153088091D0
:1003A000540890915508A70196010E947EB2C4019D
:1003B000821B930B6CE370E00E9457B2182F698385
:1003C000CE0101960E943678BC0180E49DE00E9437
:1003D000BEAD6AE380E49DE00E94BFAD1983CE010B
:1003E00001960E943678BC0180E49DE00E94BEAD7B
:1003F00003C084E89EE016DC60E973E080E49DE0E1
:100400000E94BEAD43E060E080E49DE00E947E2853
:100410006EE773E082E792E00E942EB6892B09F026
:1004200074C06EE67AE085E59DE00E942EB6892BC9
:10043000D1F0E5E5FDE0DF010D900020E9F7AD0129
:100440004150510945555D4060E070E0CF010E9488
:10045000FEB56EE67AE085E59DE00E9437B6109223
:100460008B0D10928A0DEEE6FAE001900020E9F77C
:10047000EF56FA40759708F445C000918A0D109127
:100480008B0DC12CD12C80918A0D90918B0D9801F0
:10049000281B390B2431310534F0019690938B0DD4
:1004A00080938A0D38C0C114D104B9F7F801E35A1A
:1004B000F54F7F019189602F681B43E0911115C0B2
:1004C00080E49DE00E947E28D70150966C9180E4E4
:1004D0009DE00E94BFAD10928B0D10928A0D00E03E
:1004E00010E0CC24C394D12CCECF80E49DE00E94B8
:1004F0007E28F701608980E49DE00E94BFAD0F5F18
:100500001F4FC1CF65E57DE002C062E772E080E485
:100510009DE00E94BEAD02E712E0D8018D918D01F1
:1005200080322CF460E280E49DE00E94BFADB2E036
:1005300006381B0791F78AE080932F0D80913F0DBD
:1005400082FB882780F990912E0D992399F0909144
:100550002D0D992339F0811119C010922D0D109293
:100560002E0D14C0882391F00E941D6581E08093B8
:100570002D0D0CC0882351F021E040E050E0BA017D
:100580008CE692E70E9451650E94BC6A80915D02F0
:1005900090915E022091350D3091360D8436910593
:1005A00034F4820F931F853691054CF416C08436BF
:1005B000910599F0820F931F8436910574F410927F
:1005C000350D1092360D1092370D1092380D84E6CD
:1005D00090E090935E0280935D0220915D023091E5
:1005E0005E028091350D9091360D2436310569F407
:1005F0008B3091051CF0865A9F4F09C0863FEFEF64
:100600009E078CF482599F4F02C0820F931F9093D4
:100610005E0280935D021092350D1092360D10929D
:10062000370D1092380D80915D0290915E028A30F4
:1006300091051CF48AE090E005C0883E934034F0B8
:1006400087EE93E090935E0280935D0228960FB64A
:10065000F894DEBF0FBECDBFDF91CF911F910F91F8
:10066000FF90EF90DF90CF90BF90AF909F908F90D2
:100670000895CF93DF93CFE2DEE0FE0184918823DB
:1006800041F09091C00095FFFCCF8093C600319659
:10069000F5CFE4E0F4E18491882341F09091C0002B
:1006A00095FFFCCF8093C6003196F5CF8091C000B6
:1006B00085FFFCCF8AE08093C600FE018491EFE2C3
:1006C000FEE0882349F09091C00095FFFCCF809315
:1006D000C60031968491F5CF4091A1135091A21399
:1006E0006091A3137091A4138CEF93E10E949C3D41
:1006F0004091A5135091A6136091A7137091A81370
:1007000089EF93E10E949C3D4091A9135091AA1357
:100710006091AB137091AC1386EF93E10E949C3D06
:100720004091AD135091AE136091AF137091B0131F
:1007300083EF93E10E949C3D8091C00085FFFCCF38
:100740008AE08093C600FE018491EFE2FEE08823F8
:1007500049F09091C00095FFFCCF8093C600319680
:100760008491F5CFE9EDF3E18491882341F09091F4
:10077000C00095FFFCCF8093C6003196F5CF8091E5
:10078000C00085FFFCCF8AE08093C600FE01849103
:10079000EFE2FEE0882349F09091C00095FFFCCF86
:1007A0008093C60031968491F5CF4091B11350915A
:1007B000B2136091B3137091B41380ED93E10E9472
:1007C0009C3D4091B5135091B6136091B713709151
:1007D000B8138DEC93E10E949C3D4091B913509168
:1007E000BA136091BB137091BC138AEC93E10E9421
:1007F0009C3D4091BD135091BE136091BF13709109
:10080000C01387EC93E10E949C3D8091C00085FF5E
:10081000FCCF8AE08093C600FE018491EFE2FEE007
:10082000882349F09091C00095FFFCCF8093C600CB
:1008300031968491F5CFE9EAF3E18491882341F080
:100840009091C00095FFFCCF8093C6003196F5CF04
:100850008091C00085FFFCCF8AE08093C600FE0136
:100860008491EFE2FEE0882349F09091C00095FF6B
:10087000FCCF8093C60031968491F5CF40919113BF
:1008800050919213609193137091941380EA93E1C5
:100890000E94AE3D4091951350919613609197132D
:1008A000709198138DE993E10E94AE3D40919913A8
:1008B00050919A1360919B1370919C138AE993E174
:1008C0000E94AE3D40919D1350919E1360919F13E5
:1008D0007091A01387E993E10E94AE3D8091C00022
:1008E00085FFFCCF8AE08093C600FE018491EFE291
:1008F000FEE0882349F09091C00095FFFCCF8093E3
:10090000C60031968491F5CFE2E6F3E18491882325
:1009100041F09091C00095FFFCCF8093C6003196C6
:10092000F5CF8091C00085FFFCCF8AE08093C600A0
:10093000FE018491EFE2FEE0882349F09091C0002F
:1009400095FFFCCF8093C60031968491F5CF4091FE
:10095000891350918A1360918B1370918C1389E5E0
:1009600093E10E949C3D40918513509186136091C4
:1009700087137091881386E593E10E949C3D8091D6
:10098000C00085FFFCCF8AE08093C600FE01849101
:10099000EFE2FEE0882349F09091C00095FFFCCF84
:1009A0008093C60031968491F5CFE3EAF2E1849119
:1009B000882341F09091C00095FFFCCF8093C60042
:1009C0003196F5CF8091C00085FFFCCF8AE08093FF
:1009D000C600FE018491EFE2FEE0882349F0909189
:1009E000C00095FFFCCF8093C60031968491F5CF6F
:1009F00040918D1350918E1360918F1370919013CD
:100A00008AE992E10E949C3D4091751350917613C2
:100A1000609177137091781387E992E10E949C3D71
:100A20004091C1135091C2136091C3137091C413CC
:100A300084E992E10E94AE3D40918113509182136E
:100A4000609183137091841381E992E10E949C3D2F
:100A500040917D1350917E1360917F1370918013AC
:100A60008EE892E10E949C3D4091791350917A1357
:100A700060917B1370917C138BE892E10E949C3D06
:100A80008091C00085FFFCCF8AE08093C600FE0104
:100A90008491EFE2FEE0882349F09091C00095FF39
:100AA000FCCF8093C60031968491F5CFE9E7F2E15F
:100AB0008491882341F09091C00095FFFCCF8093F2
:100AC000C6003196F5CF8091C00085FFFCCF8AE04B
:100AD0008093C600FE018491EFE2FEE0882349F096
:100AE0009091C00095FFFCCF8093C6003196849111
:100AF000F5CF4091380A5091390A60913A0A7091C5
:100B00003B0A80E792E10E949C3D40913C0A509153
:100B10003D0A60913E0A70913F0A8DE692E10E9483
:100B20009C3D4091400A5091410A6091420A709167
:100B3000430A8AE692E10E949C3D8091C00085FFB5
:100B4000FCCF8AE08093C600FE018491EFE2FEE0D4
:100B5000882349F09091C00095FFFCCF8093C60098
:100B600031968491F5CFECE5F2E18491882341F050
:100B70009091C00095FFFCCF8093C6003196F5CFD1
:100B80008091C00085FFFCCF8AE08093C600FE0103
:100B90008491EFE2FEE0882349F09091C00095FF38
:100BA000FCCF8093C60031968491F5CF4091180216
:100BB0005091190260911A0270911B0282E592E134
:100BC0000E949C3D60911402709115028091160262
:100BD000909117020E94BD27AB01BC018FE492E106
:100BE0000E949C3D6091100270911102809112024E
:100BF000909113020E94C927AB01BC018CE492E1E1
:100C00000E949C3D8091C00085FFFCCF8AE08093CC
:100C1000C600FE018491EFE2FEE0882349F0909146
:100C2000C00095FFFCCF8093C60031968491F5CF2C
:100C3000E8E1F2E18491882341F09091C00095FFB2
:100C4000FCCF8093C6003196F5CF8091C00085FF20
:100C5000FCCF8AE08093C600FE018491EFE2FEE0C3
:100C6000882349F09091C00095FFFCCF8093C60087
:100C700031968491F5CF40913302509134026091C6
:100C80003502709136028EE092E10E949C3D20E098
:100C900030E040E752E460912B0270912C02809189
:100CA0002D0290912E020E9475B1AB01BC018BE028
:100CB00092E10E949C3D4091280A5091290A60913E
:100CC0002A0A70912B0A88E092E10E949C3D809153
:100CD000C00085FFFCCF8AE08093C600FE018491AE
:100CE000EFE2FEE0882349F09091C00095FFFCCF31
:100CF0008093C60031968491F5CFECEDF1E18491BB
:100D0000882341F09091C00095FFFCCF8093C600EE
:100D10003196F5CF8091C00085FFFCCF8AE08093AB
:100D2000C600FE018491EFE2FEE0882349F0909135
:100D3000C00095FFFCCF8093C60031968491F5CF1B
:100D40004091240A5091250A6091260A7091270A41
:100D500082ED91E10E949C3D20E030E040E752E4CA
:100D600060912702709128028091290290912A02B5
:100D70000E9475B1AB01BC018FEC91E10E949C3DDA
:100D80008091C00085FFFCCF8AE08093C600FE0101
:100D90008491EFE2FEE0882349F09091C00095FF36
:100DA000FCCF8093C60031968491F5CFE5E7F1E161
:100DB0008491882341F09091C00095FFFCCF8093EF
:100DC000C6003196F5CF8091C00085FFFCCF8AE048
:100DD0008093C600FE018491EFE2FEE0882349F093
:100DE0009091C00095FFFCCF8093C600319684910E
:100DF000F5CF40912D0A50E060E070E08BE691E184
:100E00000E94AE3D8091C00085FFFCCF8AE08093B8
:100E1000C600FE018491EFE2FEE0882349F0909144
:100E2000C00095FFFCCF8093C60031968491F5CF2A
:100E30008091540A8823A1F1E8E5F1E184918823A7
:100E400041F09091C00095FFFCCF8093C600319691
:100E5000F5CF8091C00085FFFCCF8AE08093C6006B
:100E6000FE01C491EFE2FEE0CC2349F08091C00086
:100E700085FFFCCFC093C6003196C491F5CF409159
:100E800053025091540260915502709156028EE4C3
:100E900091E10E949C3D8091C00085FFFCCF11C074
:100EA000E2E3F1E18491882341F09091C00095FF45
:100EB000FCCF8093C6003196F5CF8091C00085FFAE
:100EC000FCCF8AE08093C600DF91CF910895AF9266
:100ED000BF92CF92DF92EF92FF920F931F93CF9327
:100EE000DF93CDB7DEB7E0970FB6F894DEBF0FBE45
:100EF000CDBF80E1EFEEF2E0DE01919601900D9220
:100F00008A95E1F780E1EFEFF2E0DE015196019082
:100F10000D928A95E1F780E1EFE0F3E0DE011196B2
:100F200001900D928A95E1F76E0181E2C80ED11C05
:100F300081EAE82E83E1F82E8E010F5E1F4F61EBF0
:100F400073E1AE014F5F5F4F91E9A92E93E1B92E96
:100F500020E030E0F60181919191A191B1916F0172
:100F6000F70181939193A193B1937F01F80181914E
:100F70009191A191B1918F01FB0181939193A193E3
:100F8000B193BF01FA0181919191A191B191AF010A
:100F9000F50181939193A193B1935F012F5F3F4F2F
:100FA00024303105B9F60E9410A580E090E8ABE34B
:100FB000B5E48093891390938A13A0938B13B09315
:100FC0008C138093851390938613A0938713B0930B
:100FD000881310928D1310928E1310928F1310920B
:100FE000901380E29EE4A0E0B0E08093C113909360
:100FF000C213A093C313B093C4131092751310922D
:101000007613109277131092781380E090E0A0EAA4
:10101000B1E48093811390938213A0938313B093D0
:1010200084138DEC9CECACECBEE380937D13909329
:101030007E13A0937F13B093801380E090E0A0EA2A
:10104000B0E48093791390937A13A0937B13B093B9
:101050007C131092400A1092410A1092420A109298
:10106000430A10923C0A10923D0A10923E0A1092D6
:101070003F0A1092380A1092390A10923A0A1092D6
:101080003B0A8CED90E09093980D8093970D82E34E
:1010900090E09093960D8093950D8FEF90E0909354
:1010A000940D8093930D2DE131E03093920D2093B8
:1010B000910D24E630E03093900D20938F0D9093A6
:1010C0008E0D80938D0D83E393E3ABE4B1E48093C5
:1010D000180290931902A0931A02B0931B026FE1B9
:1010E00075E88BE89FE30E94B72760931402709322
:1010F000150280931602909317026AE979E985E157
:1011000092E40E94C32760931002709311028093AF
:101110001202909313020E94251E80E090E0A0E846
:10112000BFE380930C0290930D02A0930E02B09344
:101130000F0210922D0A80E090E0A0E4B0E48093CA
:10114000330290933402A0933502B093360240E00C
:1011500050E064E372E440932B0250932C026093BE
:101160002D0270932E021092280A1092290A1092D2
:101170002A0A10922B0A1092240A1092250A109221
:10118000260A1092270A40E050E060E071E44093A4
:101190002702509328026093290270932A0210922A
:1011A000540A8093530290935402A0935502B09333
:1011B00056020E94A74AEFE2FEE08491882341F0A4
:1011C0009091C00095FFFCCF8093C6003196F5CF7B
:1011D000E0E1F1E18491882341F09091C00095FF16
:1011E000FCCF8093C6003196F5CF8091C00085FF7B
:1011F000FCCF8AE08093C600E0960FB6F894DEBF7D
:101200000FBECDBFDF91CF911F910F91FF90EF9057
:10121000DF90CF90BF90AF9008951F920F920FB6BE
:101220000F9211240BB60F922F933F934F935F931E
:101230006F938F939F93EF93FF936091C6002091DC
:101240001D0E30911E0EC90101968F77992740918E
:101250001F0E5091200E8417950741F0F901E356B7
:10126000F24F608390931E0E80931D0EFF91EF91BD
:101270009F918F916F915F914F913F912F910F901F
:101280000BBE0F900FBE0F901F9018959A01AB01E7
:10129000211581EE38074105510549F182E080931F
:1012A000C00060E079E08DE390E00E94A0B22150A0
:1012B000310941095109CA01B90122E030E040E099
:1012C00050E00E94A0B23093C5002093C4008091EA
:1012D000C10080618093C1008091C10088608093CB
:1012E000C1008091C10080688093C1000895109270
:1012F000C00020E130E0E7CF20911F0E3091200E9A
:1013000080911D0E90911E0E8217930771F0F901C6
:10131000E356F24F80812F5F3F4F2F773327309373
:10132000200E20931F0E90E008958FEF9FEF0895F9
:1013300080911F0E9091200E90931E0E80931D0E93
:1013400008954F925F926F927F928F929F92AF9289
:10135000BF92CF92DF92EF92FF920F931F93CF93A2
:10136000DF93CDB7DEB7A0970FB6F894DEBF0FBE00
:10137000CDBF5C014115510561057105E9F420E01F
:1013800030E040E350E060E070E0A0960FB6F894E3
:10139000DEBF0FBECDBFDF91CF911F910F91FF90A8
:1013A000EF90DF90CF90BF90AF909F908F907F9005
:1013B0006F905F904F905BC08E010F5F1F4FC12CED
:1013C000D12C76014801422E512C612C712C8FEFCB
:1013D000C81AD80AE80AF80ACB01BA01A301920197
:1013E0000E947EB2CA01F80161938F01A901BC017C
:1013F000411551056105710551F7F1E0CF1AD1088A
:10140000E108F108F401EC0DFD1D80818A3010F433
:1014100040E301C047E3480F552747FD5095652F2E
:10142000752F20E030E0C50122D081E0C81AD10834
:10143000E108F108EFEFCE16DE06EE06FE0611F724
:10144000A0960FB6F894DEBF0FBECDBFDF91CF914F
:101450001F910F91FF90EF90DF90CF90BF90AF90D2
:101460009F908F907F906F905F904F90089521157F
:10147000310539F48091C00085FFFCCF4093C60050
:1014800008952A30310509F41CC05BCFCF93DF9358
:10149000EC0120E030E04DE050E060E070E0E7DF9C
:1014A00020E030E04AE050E060E070E0CE01DF9103
:1014B000CF91DDCF9A01AB01662757FD6095762F5E
:1014C000D6CFCF92DF92EF92FF92CF93DF93EC01D2
:1014D0006A017B0177FF0FC020E030E04DE250E071
:1014E00060E070E0C4DFF094E094D094C094C11C3C
:1014F000D11CE11CF11C2AE0B701A601CE01DF914D
:10150000CF91FF90EF90DF90CF901BCF2115310549
:1015100039F48091C00085FFFCCF4093C600089548
:1015200010CF9A01462F50E060E070E0EFCFCF93EC
:10153000DF93EC019A01AB0160E070E0E7DFCE01E0
:10154000DF91CF91A3CF8F929F92AF92BF92CF9214
:10155000DF92EF92FF921F93CF93DF93EC016A012A
:101560007B01122F20E030E0A901C701B6010E94E3
:10157000A0AE87FF0CC020E030E04DE250E060E01C
:1015800070E0CE0174DFF7FAF094F7F8F094B12C24
:1015900060E070E080E09FE3B11641F020E030E0D1
:1015A00040E251E40E94A7AEB394F6CF9B01AC0198
:1015B000C701B6010E94C7AD6B017C010E9414AF48
:1015C0004B015C010E9440AF9B01AC01C701B60119
:1015D0000E94C6AD6B017C012AE0B501A401CE01D9
:1015E000B0DE112361F0EFE5F3E08191882339F05B
:1015F0009091C00095FFFCCF8093C600F6CF1123D9
:1016000019F120E030E040E251E4C701B6010E9448
:1016100075B16B017C010E940FAF4B01AA2497FCAE
:10162000A094BA2CB501A401CE014BDFC501B401D1
:101630000E9442AF9B01AC01C701B6010E94C6AD3A
:101640006B017C011150DBCFDF91CF911F91FF9097
:10165000EF90DF90CF90BF90AF909F908F900895C4
:1016600072CFCF93DF931F92CDB7DEB7698341E08E
:1016700050E0BE016F5F7F4F04960E9481160F906D
:10168000DF91CF910895FB0101900020E9F7AF01B0
:1016900041505109461B570B04960C9481168091BA
:1016A000390E811109C08091380E811105C08091D9
:1016B000370E811101C00895EFE2FEE08491882386
:1016C00041F09091C00095FFFCCF8093C600319609
:1016D000F5CFEFE6F4E18491882341F09091C000CA
:1016E00095FFFCCF8093C6003196F5CF8091390EDF
:1016F0008823F1F060913A0E70913B0E80913C0E80
:1017000090913D0E0E9442AF2091A1133091A213FF
:101710004091A3135091A4130E94A7AEAB01BC014A
:101720008BE694E10E949C3D8BE594E10E9400765B
:101730008091380E8823F1F060913E0E70913F0E3B
:101740008091400E9091410E0E9442AF2091A513CE
:101750003091A6134091A7135091A8130E94A7AEF1
:10176000AB01BC0187E594E10E949C3D87E494E1D4
:101770000E9400768091370E8823F1F06091420E2E
:101780007091430E8091440E9091450E0E9442AF9D
:101790002091A9133091AA134091AB135091AC132F
:1017A0000E94A7AEAB01BC0183E494E10E949C3D82
:1017B00083E394E10E9400768091C00085FFFCCF16
:1017C0008AE08093C6001092390E1092380E109263
:1017D000370E08951092390E1092380E1092370E6F
:1017E000089580939B020895EFE6F0E08081826087
:1017F000808308951F920F920FB60F9211240BB69B
:101800000F920F931F932F933F934F935F936F9379
:101810007F938F939F93AF93BF93EF93FF938091A9
:101820006A0E90916B0E892B09F084C190916D0E18
:1018300080916C0E981771F0E0916C0E8DE4E89F2A
:10184000F0011124E259F14FDF01A45BBF4F81E0A9
:101850008C9302C0E0E0F0E0F0936B0EE0936A0E30
:10186000309709F461C1DF01A45BBF4F81E08C9325
:1018700010924D0E10924E0E10924F0E1092500E6E
:1018800060AD71AD61349CE9790728F461329EE462
:10189000790748F002C060E47CE976956795769513
:1018A000679584E007C0613197E2790730F076955B
:1018B000679582E080934A0E07C080934A0E60329B
:1018C000710510F460E270E060527109611588E002
:1018D0007807D0F0872F9927880F991F880F991FB5
:1018E0008258974EFC01329645915491AA27659FE4
:1018F0009001649F210D3A1F06942A1F3A1F11245C
:10190000FC01859194911DC0CB01969587958C7FA4
:1019100082589B4EFC01459154910296FC018591A1
:101920009491FB01E770FF278E9F90018F9F300DF0
:101930009E9F300D1124E3E036952795EA95E1F757
:10194000CA01821B930B8436910598F4EEEBF5E007
:101950008191882339F09091C00095FFFCCF80934E
:10196000C600F6CF4AE050E08CE99DE0E0DD84E679
:1019700090E09093490E8093480E80914A0E9927EB
:1019800087FD90959093470E8093460EE0916A0EE6
:10199000F0916B0E64AD75AD70934C0E60934B0E71
:1019A00061349CE9790728F461328EE4780748F0C5
:1019B00002C060E47CE9769567957695679584E04A
:1019C00007C0613197E2790730F07695679582E03C
:1019D00080934A0E08C081E080934A0E6032710500
:1019E00010F460E270E060527109611588E07807D8
:1019F000E0F0872F9927880F991F880F991F825829
:101A0000974EFC01329625913491AA27639FA0013D
:101A1000629F410D5A1F06944A1F5A1F1124FC0150
:101A200025913491241B350B1EC0CB0196958795CB
:101A30008C7F82589B4EFC01259134910296FC01CB
:101A400045915491FB01E770FF274E9FC0014F9FC6
:101A5000900D5E9F900D1124F3E096958795FA9571
:101A6000E1F7281B390B2436310598F4EEEBF5E04D
:101A70008191882339F09091C00095FFFCCF80932D
:101A8000C600F6CF4AE050E08CE99DE050DD24E648
:101A900030E0C901A0E0B0E08093510E9093520E67
:101AA000A093530EB093540E309389002093880076
:101AB000E0916A0EF0916B0E80899189A289B389B9
:101AC000B695A79597958795B095A0959095819592
:101AD0009F4FAF4FBF4F8093650E9093660EA093BC
:101AE000670EB093680E8093610E9093620EA09380
:101AF000630EB093640E80935D0E90935E0EA09380
:101B00005F0EB093600E8093590E90935A0EA0937F
:101B10005B0EB0935C0E1092550E1092560E109202
:101B2000570E1092580E06C080ED97E090938900F2
:101B300080938800E0916A0EF0916B0E309709F463
:101B400087C580A18093690E9FB780FF09C0F89474
:101B500080910B018D7F80930B019FBF8FEF08C099
:101B6000F89480910B01826080930B019FBF81E00C
:101B7000809397028091690E9FB781FF09C0F89406
:101B800080910B018E7F80930B019FBF8FEF08C068
:101B9000F89480910B01816080930B019FBF81E0DD
:101BA000809398022091690E30919B0220FF3BC0E8
:101BB000332309F472C01E9902C080E031C08091C5
:101BC000360E882361F1E0916A0EF0916B0E8081F0
:101BD0009181A281B381181619061A061B06FCF41E
:101BE0008091210E9091220EA091230EB091240E8F
:101BF00080933A0E90933B0EA0933C0EB0933D0E13
:101C000081E08093390E80899189A289B38980937C
